:100000000C9400210C9431210C9431210C94312159
:100010000C9431210C9431210C9431210C94312118
:100020000C9431210C9431210C9431210C94312108
:100030000C9431210D94FE370C9431210C94312114
:100040000C9431210C943CD80C9431210C94312126
:100050000C9431210C9431210C9403D50D94B437B8
:100060000C9431210C94304C0C94264C0C9431217E
:100070000C9431210C9431210C9431210C943121B8
:100080000C9431210C9431210C9431210C943121A8
:100090000C9431210C9431210C9431210C94312198
:1000A0000C9431210C9431210C9431210C94312188
:1000B0000C9431210C9431210C9431210C94312178
:1000C0000C9431210C9431210C9431210C94312168
:1000D0000C9431210C9431210C9431210C94312158
:1000E0000C943121084AD73B3BCE016E84BCBFFD46
:1000F000C12F3D6C74319ABD56833DDA3D00C77FF8
:1001000011BED9E4BB4C3E916BAAAABE0000008090
:100110003F05A84CCDB2D44EB93836A9020C50B91F
:10012000918688083CA6AAAA2ABE000000803F004B
:100130000C942E7F0C94F6840C94A27A0C949D4C13
:100140000C94D3AF0C94F44C0C9480C80C9403869C
:100150000C9426C30C9406860C94F9A60D94F531E4
:100160000C948B830C94FF840C9431780C9420793C
:100170000C94C1AF0C9409820C949CC90D9420314D
:100180000C94B37C0C94EBAF0D94A4310C94BE7E14
:100190000C941BBD0D9439310C94AF7C0C948D786C
:1001A0000C94237D0D942C310C94997A0C94A3AF6C
:1001B0000C947A7A0C94DFC80C9466810C94DA4C17
:1001C0000C94A99E0C94C64C0C94BB4C0C943C22F1
:1001D0000D94D7310D942C320D9424310C945FC8BA
:1001E0000C94B17C0C9400BC0C9433210C94369686
:1001F0000C94C4C80C94B5AF0D94D3120C943BB3BB
:100200000D943F310C94D7330C94AC4C0C94089D56
:100210000C9472810C94CDAF0C94F1BC0D94E1312F
:100220000D9432130C9455820C9463790C940D86C2
:100230000C94F7850C943B760C9452810C94F5AF9A
:100240000C94ECB00C94687E0C945E810C945DC9A7
:100250000D9436320C9413860C94A0820C948782F1
:100260000C9440A00D9434440C9431B30C9466CAA1
:100270000C94A6780C944C790C94FCC40C94FD85D9
:100280000C94E5AF0C9419820D940E310C942A7ADB
:100290000C9441250D9455310C94458E0C94C7AFA8
:1002A0000C94D24C0D9418320C9491BC0C94A9C3AC
:1002B0000C9436B30C9445380C94E4980D940432A5
:1002C0000C942E830C94187B0C941FBC0C94CC784B
:1002D0000D940E320C94AFAF0C949D7A0C94362191
:1002E0000C94AC970C94B0210C9421820C94037B59
:1002F0000C94AB7C0D9435310C94BA7E0C940D7635
:100300000C9416970D94CF310C9476810C94DA826C
:100310000D94E1430C94F4850C944A780C946C860B
:100320000C942AA80C94DFAF0C94298D0C94EC4CFF
:100330000C94BBAF0D9452440C9418250C94FE7889
:100340000C94B17A0C942D7B0C940B860C94B9828E
:100350000C94C68B0D9409310C94D64C0C94667C8D
:100360000C94867A0C941C7C0C9424220C94917925
:100370000C94FB820C94C1990C949B7A0C94CAC780
:100380000C94A9AF0C94AD7C0C94C24C0C9472BC30
:100390000C9430760C94E8880C9410860D945F31A0
:1003A0000C94E7900C94A77C0C94157B0C94CB7B5D
:1003B0000D94BD310C94EE840C9463780C9412A2CD
:1003C0000D94B3310D945B310C947A790C945D7C6F
:1003D0000C94127B0D94C7310C94CDB30C94D2BC09
:1003E0000C94AC940C94B67E0C94B9780C94628105
:1003F0000D9429140D942F310C9440B30C94E7C73D
:100400000D9422320C94FA850C9426B70D94513138
:100410000C9458B30C940D790C944B980C94A32520
:100420000C94CE4C0C9456810C94367B0C944C84DA
:100430000C94E14C0C94327B0C94B39E0C946FC9D9
:100440000D9443310C94AC7A0C945A810C948786A9
:100450000C94A8C30D9400130C94C4820C9472786D
:100460000C946E810C941B7B0C9400860C94E97A9E
:100470000C94A97C0D944D310C944BC70C94D9AFBE
:100480000C94A77A0C94AA920C94329B0C94A879A1
:100490000C94A57C0C94717A0C940A850C9411A58B
:1004A0000D9428310D94A9310C947A760C94BB8A62
:1004B0000C946E820C94AEAC0C94E5780D94EB31F8
:1004C0000C946E4C0C94E6850C9433790D94473162
:1004D0000C9445830C94E8840C946A810C9407B4C2
:1004E0000C94CA4C0C9493760C94A1760C945C7E7C
:1004F0000D949C310C9469860C940D7C0C94F185C0
:100500004E414E494E495459494E46CDCCCC3D0AF8
:10051000D7233C17B7D13877CC2B329595E6241FDB
:10052000B14F0A000020410000C84200401C462094
:10053000BCBE4CCA1B0E5AAEC59D7400407A10F367
:100540005A00A0724E18090010A5D4E80000E87601
:1005500048170000E40B54020000CA9A3B00000058
:10056000E1F505000080969800000040420F000071
:1005700000A08601000000102700000000E8030032
:100580000000006400000000000A000000000001FC
:1005900000000000002C76D888DC674F0823DFC1FC
:1005A000DFAE59E1B1B796E5E3E453C63AE65199B7
:1005B0007696E8E6C28426EB898C9B62ED407C6FE0
:1005C000FCEFBC9C9F40F2BAA56FA5F490055A2A97
:1005D000F75C936B6CF9676DC11BFCE0E40D47FEA3
:1005E000F520E6B500D0ED902E0300943577050098
:1005F00080841E080000204E0A000000C80C33331F
:1006000033330F986E12831141EF8D2114893BE62D
:100610005516CFFEE6DB18D1844B381BF77C1D90B6
:100620001DA4BBE424203284725E228100C9F1241F
:10063000ECA1E53D27434F4D4D554E4943415449AB
:100640004F4E0044525952554E004552524F52534C
:1006500000494E464F004543484F004572726F7245
:100660002077726974696E6720746F204545505217
:100670004F4D210A0053544F505045442E200050F6
:1006800072696E7465722073746F70706564206433
:10069000756520746F206572726F72732E204669C3
:1006A0007820746865206572726F7220616E6420B4
:1006B000757365204D39393920746F2072657374F4
:1006C0006172742E202854656D7065726174757244
:1006D000652069732072657365742E2053657420DC
:1006E00069742061667465722072657374617274D6
:1006F000696E67290A004E6F20436865636B7375E6
:100700006D2077697468206C696E65206E756D6206
:1007100065722C204C617374204C696E653A200020
:100720004E6F20436865636B73756D2077697468DD
:10073000206C696E65206E756D6265722C204C614F
:100740007374204C696E653A2000636865636B734F
:10075000756D206D69736D617463682C204C6173D5
:1007600074204C696E653A20004C696E65204E75A8
:100770006D626572206973206E6F74204C617374B2
:10078000204C696E65204E756D6265722B312C2090
:100790004C617374204C696E653A20004D313130E4
:1007A0000053657269616C20737461747573206D98
:1007B00069736D617463680A00776169740A005334
:1007C000442072656164206572726F720A00486F1E
:1007D00074656E642049646C652054696D656F753D
:1007E0007400486F74656E642049646C65205469B8
:1007F0006D656F75740A002121204B494C4C2063B4
:100800006175736564206279204B494C4C20627598
:1008100074746F6E2F70696E0A002121204B494C51
:100820004C2063617573656420627920746F6F205A
:100830006D75636820696E6163746976652074699B
:100840006D65202D2063757272656E7420636F6D07
:100850006D616E643A20007061757365004D3630CD
:1008600030002066696C616D656E745F72756E6FC5
:100870007574200066696C616D656E745F72756E6B
:100880006F757420540046696C616D656E745275A5
:100890006E6F75742054004D656469612052656DFA
:1008A0006F766564004D6564696120496E73657299
:1008B000746564004D313030305300627573793A9D
:1008C0002070617573656420666F7220696E707543
:1008D000740A00627573793A2070617573656420DB
:1008E000666F7220757365720A00627573793A20BB
:1008F00070726F63657373696E670A00506C65612F
:100900007365205265736574005052494E544552C8
:100910002048414C5445440025533A20255300704B
:100920006F7765726F6666004B494C4C45442E20CC
:10093000005072696E7465722068616C7465642E13
:10094000206B696C6C28292063616C6C6564210ADA
:10095000006563686F3A004572726F723A000A4D23
:100960006561737572656420706F696E74733A0A9D
:1009700000357835206D6573682E205A206F6666C5
:100980007365743A20005072696E74696E67204F07
:10099000626A656374002553202569002F2F616307
:1009A00074696F6E3A0073746172740070726F6D67
:1009B00070745F00656E6400486F74656E642074C7
:1009C0006F6F20636F6C640A0053656E64204D3155
:1009D000303820746F20726573756D650A00496E3A
:1009E000736572742066696C616D656E7420616EEA
:1009F000642073656E64204D3130380A005265689A
:100A000065617420446F6E65005265686561746944
:100A10006E672E2E2E005265686561740048656110
:100A20007465722054696D656F75740053656E64EA
:100A3000204D31303820746F2068656174206E6FEE
:100A40007A7A6C650A004E6F7A7A6C652050617212
:100A50006B656400706175736564005061757365E2
:100A600000726573756D656400526573756D696EAE
:100A700067004732362043616E63656C65640047EA
:100A800032362048656174696E67204E6F7A7A6CE1
:100A900065004732362048656174696E672042659B
:100AA000640057616974696E6720666F72206865BB
:100AB000617475702E0A004669786564204C656E15
:100AC000677468205072696D6500446F6E652050D0
:100AD00072696D696E67004D616E75616C20707230
:100AE000696D696E672E2E2E004C656176696E67A2
:100AF00020473236003F537065636966696564203C
:100B0000582C5920636F6F7264696E617465206F31
:100B10007574206F6620626F756E64732E0A003FD5
:100B200028522965706561742076616C7565206E48
:100B30006F7420706C61757369626C653B206D75B4
:100B40007374206265206174206C65617374203158
:100B50002E0A003F537065636966696564206E6F95
:100B60007A7A6C652074656D7065726174757265F2
:100B7000206E6F7420706C61757369626C652E0AEB
:100B8000003F5370656369666965642066696C61DE
:100B90006D656E742073697A65206E6F7420706C59
:100BA00061757369626C652E0A003F5370656369F5
:100BB00066696564207072696D65206C656E677426
:100BC00068206E6F7420706C61757369626C652E3D
:100BD0000A003F537065636966696564206E6F7AC9
:100BE0007A6C652073697A65206E6F7420706C6111
:100BF000757369626C652E0A003F52657472616399
:100C000074696F6E204D756C7469706C69657220C3
:100C10006D757374206265207370656369666965BC
:100C2000642E0A003F5370656369666965642052EB
:100C3000657472616374696F6E204D756C74697050
:100C40006C696572206E6F7420706C617573696277
:100C50006C652E0A003F53706563696669656420A0
:100C60006C6179657220686569676874206E6F745D
:100C700020706C61757369626C652E0A0043292EC1
:100C80000A003F5370656369666965642062656444
:100C90002074656D7065726174757265206E6F7415
:100CA00020706C61757369626C65202834302D008A
:100CB000473236207374617274696E672E2E2E0A65
:100CC000004F46460A0046616465204865696768CA
:100CD000742000426564204C6576656C696E6720FF
:100CE000004661696C656420746F20656E61626C9A
:100CF0006520426564204C6576656C696E670A0004
:100D00004D65736820426564204C6576656C20648F
:100D10006174613A0A00496E76616C6964206D65A0
:100D200073682E0A00206E6F7420656E746572659C
:100D3000642E0A0050726F62696E6720506F696E90
:100D4000740025532025692F256900206F66200037
:100D50004D424C2047323920706F696E7420002953
:100D60000A004A206F7574206F662072616E676595
:100D70002028302D00290A0049206F7574206F66E5
:100D80002072616E67652028302D004732384C3064
:100D9000004D6573682070726F62696E6720646FC2
:100DA0006E65004D6573682070726F62696E6720B2
:100DB000646F6E652E0A005374617274206D6573E2
:100DC000682070726F62696E67207769746820228C
:100DD000473239205331222066697273742E0A001B
:100DE0004732395332004732384C300A4732395390
:100DF0003200686173206E6F20646174612E0A0096
:100E00004D65736820426564204C6576656C696E3B
:100E100067200053206F7574206F662072616E67C3
:100E2000652028302D35292E0A004D657368207005
:100E30006F696E74206F7574206F662072616E67C3
:100E4000650A004D34323120696E636F72726563DA
:100E50007420706172616D6574657220757361676D
:100E6000650A004F4646004F4E0020204D61783AFB
:100E70002000200020204D696E3A2000536F6674D8
:100E800020656E6473746F70733A20004D323420A5
:100E900053256C642054256C64004739322E392068
:100EA00045257300473120462564004739322E39E5
:100EB000205A2573004731205A3020463230300006
:100EC0004731205825732059257320463330303060
:100ED000004D34323020532569205A2573004D319E
:100EE00030362050256920532569004D323030209E
:100EF0004425730047323852305859004739322E52
:100F000039204530205A300A47315A2573004D3177
:100F1000303920532569004D31393020532569007F
:100F20004D343230205330205A300020496E7661E3
:100F30006C6964206578747275646572200047324C
:100F40002F47332062616420706172616D65746542
:100F500072730A00536C6565702E2E2E004D6573FA
:100F60006820706F696E74206F7574206F662072D0
:100F7000616E67650A004D302053746F70004D310B
:100F80002053746F7000436C69636B20746F205240
:100F90006573756D652E2E2E004E6F204D6F766534
:100FA0002E00456E642066696C65206C6973740A56
:100FB00000426567696E2066696C65206C697374B0
:100FC0000A004E6F206D656469610A005265737591
:100FD0006D696E6720534400286E6F2066696C65EA
:100FE000290043757272656E742066696C653A20DB
:100FF000005072696E742074696D653A20000A535E
:10100000746174733A2046696C616D656E74207505
:101010007365643A20002C204C6F6E6765737420F2
:101020006A6F623A2000546F74616C2074696D6558
:101030003A200053746174733A20002C2046616991
:101040006C65643A20002C2046696E69736865649B
:101050003A20005072696E74733A200053746174C0
:10106000733A2000436F6F6C696E672E2E2E004816
:10107000656174696E672E2E2E0045202553006F22
:101080006B006F666600560651064A064306350633
:1010900044454255473A004D3131332053004265B3
:1010A0006420436F6F6C696E672E2E2E004265645C
:1010B0002048656174696E672E2E2E00544D3344AE
:1010C00020435231305632204F46462E002F2F00FB
:1010D0004D31343520533C696E6465783E206F7520
:1010E00074206F662072616E67652028302D31296B
:1010F0000A00205200416363656C65726174696F18
:101100006E3A2050005741524E494E4721204C6FB5
:1011100077205A204A65726B206D6179206C656179
:101120006420746F20756E77616E746564207061E1
:10113000757365732E0A004D3230362058004652C2
:101140003A0020466C6F773A20004D424C204164B3
:101150006A757374205A0020643A0020693A0020AE
:10116000703A00496E76616C6964206578747275B6
:101170006465720A0020643A0020693A0020703ADF
:101180000064697300656E0043290A0061626C6542
:101190006420286D696E2074656D702000436F6C4B
:1011A00064206578747275646573206172652000CF
:1011B00046696C616D656E742072756E6F75742012
:1011C00064697374616E636520286D6D293A20002F
:1011D00046696C616D656E742072756E6F757420F2
:1011E000004F666673657473204170706C69656446
:1011F000004572723A20546F6F206661722100546C
:101200006F6F206661722066726F6D207265666511
:1012100072656E636520706F696E740A0045455093
:10122000524F4D204F4B0A00506F7765722D6C6FF7
:101230007373207265636F7665727920004D383460
:1012400000446F6E65207072696E74696E67206607
:10125000696C650A004D3737004D333100436170CA
:101260003A004D4541545041434B00434F4F4C458C
:10127000525F54454D5045524154555245004348E4
:10128000414D4245525F54454D504552415455528F
:101290004500424142595354455050494E47004140
:1012A000524353004D4F54494F4E5F4D4F444553A9
:1012B00000544845524D414C5F50524F54454354A1
:1012C000494F4E004C4F4E475F46494C454E414DAD
:1012D00045004155544F5245504F52545F53445F5F
:1012E0005354415455530053445F57524954450099
:1012F00052455045415400534443415244005052DA
:101300004F4D50545F535550504F525400454D452A
:101310005247454E43595F50415253455200434155
:1013200053455F4C494748545F4252494748544EE1
:1013300045535300544F47474C455F4C4947485429
:101340005300534F4654574152455F504F574552F3
:10135000004255494C445F50455243454E54004C61
:101360004556454C494E475F44415441005A5F50F1
:10137000524F42450052554E4F5554004155544F1F
:101380004C4556454C005052494E545F4A4F42001E
:1013900050524F4752455353004155544F524550B8
:1013A0004F52545F54454D5000564F4C554D455487
:1013B00052494300454550524F4D0042494E41521B
:1013C000595F46494C455F5452414E534645520081
:1013D00053455249414C5F584F4E5F584F46460067
:1013E0004649524D574152455F4E414D453A4D6138
:1013F000726C696E20322E302E375F4457372E3391
:1014000020544D33442053534D444E4E20284170B8
:101410007220323420323032312032323A33383A8C
:1014200032302920534F555243455F434F44455F67
:1014300055524C3A68747470733A2F2F6769746808
:1014400075622E636F6D2F496E73616E6974794199
:1014500075746F6D6174696F6E2F4D61726C696E1A
:101460002F747265652F437265616C697479447776
:10147000696E5F322E302050524F544F434F4C5FB5
:1014800056455253494F4E3A312E30204D41434834
:10149000494E455F545950453A544D3344204352C8
:1014A000313056322045585452554445525F434FCF
:1014B000554E543A3120555549443A636564653276
:1014C0006132662D343161322D343734382D396232
:1014D00031322D6335356336326633363766660A08
:1014E0000043616E6E6F74206F70656E207375625D
:1014F00064697220002569730025696D2025697370
:10150000002569682025696D2025697300256964B7
:10151000202569682025696D202569730025697972
:1015200020256964202569682025696D2025697357
:101530000023646566696E652044454641554C54F8
:101540005F00626564004B6420004B6920004B70B3
:101550002000504944204175746F74756E65206693
:10156000696E6973686564212050757420746865BC
:10157000206C617374204B702C204B6920616E6469
:10158000204B6420636F6E7374616E747320667297
:101590006F6D2062656C6F7720696E746F20436F8A
:1015A0006E66696775726174696F6E2E680A0050A5
:1015B0004944204175746F74756E65206661696C6D
:1015C0006564212074696D656F75740A0050494423
:1015D000204175746F74756E65206661696C656411
:1015E000212054656D706572617475726520746F29
:1015F0006F20686967680A00204B643A2000204B1E
:10160000693A2000204B703A200020436C617373CC
:10161000696320504944200A00204E6F206F766590
:101620007273686F6F740A002054753A2000204B63
:10163000753A2000206D61783A2000206D696E3A7D
:10164000200020643A200020626961733A20005033
:101650004944204175746F74756E652073746172AE
:10166000740A00504944204175746F74756E65208A
:101670006661696C6564212054656D706572617482
:1016800075726520746F6F20686967680A00504939
:1016900044204175746F74756E6500504944204153
:1016A00075746F74756E65206661696C6564212060
:1016B000426164206865617465722069640A00454E
:1016C00072723A207574663820666F6E74206E6F81
:1016D0007420696E697469616C697A65642E00456D
:1016E00072723A207574663820666F6E74206E6F61
:1016F0007420696E697469616C697A65642E00454D
:1017000072723A207574663820666F6E74206E6F40
:101710007420696E697469616C697A65642E000071
:101720000C0F00FE07022503BB017FFE08FE08FE2A
:1017300005080806000040F0C88888987810050859
:1017400008060000C0F88888888888F8050505061E
:1017500000012030F830200508080600002070F84D
:1017600020202020E00509090600FF2070A8A8B865
:1017700088887020070505070001D86C366CD805ED
:1017800009090600FFF8A88888888888A8F8050A4B
:101790000A0600FE205050505088A8A88870030305
:1017A0000306000340A040FFFFFFFFFFFFFFFFFF16
:1017B000FFFFFFFFFFFFFFFFFFFFFFFFFF00000036
:1017C0000605FF01070706020080808080800080F8
:1017D000030303060105A0A0A005060606000050AD
:1017E000F85050F8500509090600FF2070A8A070B5
:1017F00028A87020050707060000C8C810204098D8
:101800009805070706000040A0A040A890680103C3
:10181000030602058080800309090601FF2040407D
:101820008080804040200309090601FF804040205D
:10183000202040408005070706000020A870207087
:10184000A8200505050600012020F820200203033A
:101850000601FFC04080050101060003F8020202F4
:10186000060100C0C0050707060000081010204050
:101870004080050707060000708898A8C888700394
:10188000070706010040C040404040E0050707064A
:101890000000708808102040F8050707060000F8CF
:1018A00008103008887005070706000010305090B7
:1018B000F81010050707060000F880F00808887087
:1018C000050707060000304080F08888700507078C
:1018D000060000F808101020202005070706000069
:1018E00070888870888870050707060000708888EF
:1018F00078081060020505060100C0C000C0C002E3
:1019000006060601FFC0C000C040800305050601B1
:10191000012040804020050303060002F800F80380
:1019200005050601018040204080050707060000EC
:10193000708810202000200507070600007088B876
:10194000A8B88070050707060000708888F88888A6
:1019500088050707060000F04848704848F005076A
:1019600007060000708880808088700507070600E1
:1019700000F04848484848F0050707060000F8808E
:1019800080F08080F8050707060000F88080F0806E
:1019900080800507070600007088808098887005A1
:1019A0000707060000888888F888888803070706E4
:1019B0000100E04040404040E005070706000038D5
:1019C0001010101090600507070600008890A0C056
:1019D000A09088050707060000808080808080F83E
:1019E00005070706000088D8A888888888050707A3
:1019F0000600008888C8A8988888050707060000A0
:101A000070888888888870050707060000F0888835
:101A1000F080808005070706000070888888A890FD
:101A200068050707060000F08888F0A09088050781
:101A30000706000070888070088870050707060098
:101A400000F82020202020200507070600008888B5
:101A5000888888887005070706000088888888506D
:101A6000502005070706000088888888A8A8500528
:101A70000707060000888850205088880507070659
:101A8000000088885020202020050707060000F865
:101A90000810204080F80309090601FFE0808080DB
:101AA00080808080E005070706000080404020100D
:101AB00010080309090601FFE02020202020202033
:101AC000E00503030600052050880501010600FE1D
:101AD000F803030306010580402005050506000004
:101AE00070087888780507070600008080F08888ED
:101AF00088F00505050600007080808870050707DE
:101B00000600000808788888887805050506000022
:101B10007088F08070050707060000304840E040FC
:101B200040400507070600FE708888887808700521
:101B300007070600008080F088888888030707066A
:101B400001004000C0404040E00409090601FE10C9
:101B5000003010101010906005070706000080800C
:101B60008890E09088030707060100C0404040408D
:101B700040E0050505060000D0A8A8A8A8050505B1
:101B8000060000B0C8888888050505060000708832
:101B90008888700507070600FEF0888888F0808036
:101BA0000507070600FE7888888878080805050577
:101BB000060000B0C880808005050506000078801A
:101BC0007008F00507070600002020F820202018E4
:101BD0000505050600008888889868050505060043
:101BE0000088888850200505050600008888A8A878
:101BF0005005050506000088502050880507070697
:101C000000FE88888850204080050505060000F801
:101C1000102040F80309090601FF204040408040A1
:101C20004040200109090602FF808080808080807A
:101C300080800309090601FF804040402040404069
:101C40008005030306000248A890FF554E4C4F4103
:101C5000442046494C414D454E54004C4F41442090
:101C600046494C414D454E540046494C414D454E28
:101C700054204348414E47450042656400456E6329
:101C80006C6F73757265002568753A25303268751A
:101C90000025303268753A253032687500202020E2
:101CA000202020200020202020001FE020102010D5
:101CB0002010102010202010201030300840048008
:101CC00003001FE03FF03FF03FF01FE01FE03FF058
:101CD0003FF03FF00FC0078003003FFFF038007077
:101CE00030FC3020FC102078102030102C00D02E3A
:101CF00031D02F7BD02F7BD02E31D02C00D0203074
:101D00001020781020FC1030FC303800703FFFF0BD
:101D10003FFFF03800703186302387102787902FDF
:101D200087D02F03D020301020781020781020305A
:101D3000102F03D02F87D02787902387103186302C
:101D40003800703FFFF01FFFF81FFFF8041040023B
:101D50000820020820041040082080104100104193
:101D6000000820800410400000001FFFF81FFFF84B
:101D7000FFFFFF8000018E00E19F01F19381399FF9
:101D800081F99F81F99FB9F98F28F180380180008E
:101D9000019FFFF99174999B06A99B54A99B56A991
:101DA0009B54999FFFF9FFFFFF6E6F74696669632B
:101DB0006174696F6E200063616E63656C005072C0
:101DC000696E742041626F72746564004469736D5A
:101DD0006973730055492041626F72746564004DE8
:101DE000323520500A4D323400526573756D6500EE
:101DF00055492050617573650050617573696E6750
:101E00002E2E2E00726573756D65004D32340052B2
:101E1000756E6F75742044697374206D6D004C6F1E
:101E20006164206D6D00556E6C6F6164206D6D0096
:101E300046696C2E204469612E004520696E206D34
:101E40006D5E33004D3330332055312045256920F8
:101E500053256900504944204175746F74756E654F
:101E6000202A005049442D44202A005049442D493D
:101E7000202A005049442D50202A00200820466185
:101E80006374002008204D6178002008204D696EA1
:101E9000004F6666004F6E004175746F74656D701B
:101EA000005654726176204D696E00566D696E0061
:101EB000566D6178204500566D6178205A00566D48
:101EC0006178205900566D6178205800416D617825
:101ED000204500416D6178205A00416D617820599C
:101EE00000416D6178205800412D54726176656C17
:101EF00000412D5265747261637400416363656CC7
:101F00000056652D4A65726B00565A2D4A65726BF4
:101F10000056592D4A65726B0056582D4A65726BF2
:101F200000452073746570732F6D6D005A205374D3
:101F30006570732F6D6D00592053746570732F6D2C
:101F40006D00582053746570732F6D6D0041647679
:101F5000616E6365642053657474696E6773003FD6
:101F60000043616E63656C00496E6974004D3432E4
:101F70003800496E697469616C697A65204545501D
:101F8000524F4D0046696C616D656E740054656D0D
:101F900070657261747572650053746570732F6D2E
:101FA0006D004A65726B00416363656C65726174B4
:101FB000696F6E0056656C6F636974790053657460
:101FC00020486F6D65204F66667365747300436FBC
:101FD0006E66696775726174696F6E003F004E6569
:101FE000787420506F696E7400446F6E65004E65A2
:101FF0007874004C6576656C696E6720446F6E6519
:1020000021004D6F7665205A004732395332004E19
:1020100065787420506F696E74002569202F202523
:102020007500473239533100473239533200436C1F
:1020300069636B20746F20426567696E00486F6D3D
:10204000696E672058595A005A2056616C756500B0
:10205000496E646578205900496E6465782058009F
:1020600053746F72652053657474696E6773004CA6
:102070006F61642053657474696E6773004C657694
:10208000656C20436F726E65727300426564205AFE
:10209000004661646520486569676874004F66663C
:1020A000004F6E00426564204C6576656C696E6712
:1020B0000045646974204D657368004C6576656CF5
:1020C00020426564004D6F74696F6E003F0043618C
:1020D0006E63656C204F626A656374004E4F0059F1
:1020E00045530043616E63656C204F626A6563749B
:1020F000203D004D61696E00426564004E6F7A7A42
:102100006C650046616E20537065656400436F6EB8
:1021100066696775726174696F6E004C6F616420E7
:1021200053657474696E677300526573746F72657A
:102130002044656661756C74730053746F7265201A
:1021400053657474696E6773005072656865617475
:10215000202420436F6E6600506F776572204F75A4
:1021600074616765004F6666004F6E0052756E6F52
:1021700075742053656E736F7200416476616E638F
:1021800065642053657474696E6773004D61696E90
:10219000004D37303220542564004D363030204217
:1021A0003020542564004D373032203B2564004DEB
:1021B00037303120542564004D373032004D3730F0
:1021C00031004D363030204230004D61696E0043A1
:1021D0006F6E74696E7565004F6666004F6E0052D3
:1021E000756E6F75742053656E736F7200507572E3
:1021F0006765206D6F726500524553554D45204F00
:102200005054494F4E533A005052494E5420504179
:10221000555345440020204E6F7A7A6C653A200071
:102220005061726B696E672E2E2E00000057616937
:102230007420666F720066696C616D656E742063F0
:1022400068616E676500746F207374617274005703
:1022500061697420666F720066696C616D656E7489
:1022600020756E6C6F616400004E6F7A7A6C652029
:1022700068656174696E6700506C6561736520778D
:102280006169742E2E2E0000507265737320627582
:1022900074746F6E00746F2068656174206E6F7A5D
:1022A0007A6C650000496E736572742066696C61B2
:1022B0006D656E7400616E64207072657373206268
:1022C0007574746F6E00746F20636F6E74696E75D1
:1022D00065005761697420666F720066696C616D94
:1022E000656E74206C6F61640000507265737320BA
:1022F000427574746F6E00746F20726573756D65CE
:10230000207072696E7400005761697420666F7284
:10231000207072696E7400746F20726573756D65DC
:102320002E2E2E00005761697420666F7200666958
:102330006C616D656E7420707572676500003E207B
:1023400000256C642E25696D00457874727564658E
:102350006420546F74616C003E20004C6F6E6765A2
:102360007374204A6F622054696D65003E200054EA
:102370006F74616C205072696E742054696D6500D1
:10238000436F6D706C65746564003A20005072692B
:102390006E7420436F756E74003A20003135300042
:1023A00035004245443A20415443203130344754AB
:1023B0002D320052756E61776179205761746368C0
:1023C0003A204F4E004D61782054656D70003435D1
:1023D00030004D696E2054656D7000350045313A0E
:1023E00020536C696365456E6720343530C2B04355
:1023F000005053550047656E657269630050726FF7
:10240000746F636F6C00312E30004261756400326E
:10241000353030303000437265616C697479334413
:102420002052414D5053004D657368204C657665D0
:102430006C696E67004578747275646572730031FB
:102440000074696E796D616368696E657333642EBB
:10245000636F6D00544D3344204352313056320087
:10246000323032312D30342D313800322E302E378B
:102470005F4457372E33004D61726C696E005072A5
:10248000696E746572205374617473005468657268
:102490006D6973746F727300426F61726420496E6C
:1024A000666F005072696E74657220496E666F00C7
:1024B0004D61696E004D313030300053746F7020C3
:1024C0005072696E7400526573756D652050726943
:1024D0006E7400506F776572204F75746167650088
:1024E0003F004261636B0053746F70005072696EFD
:1024F000742066726F6D204D656469610043686188
:102500006E6765204D65646961004D32310041623E
:102510006F7574205072696E746572004368616EE5
:1025200067652046696C616D656E7400436F6E6609
:10253000696775726174696F6E0054656D7065725C
:102540006174757265004D6F74696F6E00486F73CA
:102550007420537461727400526573756D652050F8
:1025600072696E74004E6F204D656469610043614D
:102570006E63656C204F626A6563740054756E65A6
:102580000053746F70205072696E740050617573DF
:1025900065205072696E7400496E666F20536372D5
:1025A00065656E003F005374617274205072696EED
:1025B000740043616E63656C005072696E74004311
:1025C000616E6E6F7420656E7465722073756264DF
:1025D00069723A2000022E2E004D61696E002100C2
:1025E000486F74656E6420746F6F20636F6C640055
:1025F0004261636B0050726F63656564004F66668D
:10260000004F6E00536F667420456E6473746F7074
:1026100073004D6F74696F6E0044697361626C651D
:10262000205374657070657273004D3834004265D4
:1026300064204C6576656C696E6700486F6D652037
:102640005A004732385A00486F6D652059004732AA
:10265000385900486F6D652058004732385800419E
:1026600075746F20486F6D6500473238004D6169A1
:102670006E0050726568656174202420456E6400A8
:102680005072656865617420242042656400546559
:102690006D706572617475726500436F6F6C646F05
:1026A000776E005072656865617420240046616E23
:1026B000205370656564207E00426564004E6F7A29
:1026C0007A6C65004D61696E004261627973746570
:1026D00070205A00466C6F770046616E205370651B
:1026E0006564207E00426564004E6F7A7A6C6500F6
:1026F000426564205A005370656564004D61696EDF
:1027000000486F6D696E67204661696C6564006F93
:1027100070656E00545249474745524544003A207F
:102720000066696C616D656E74007A5F6D696E003C
:10273000795F6D696E00785F6D696E005265706FCC
:102740007274696E6720656E6473746F7020737441
:10275000617475730A0020746F6F206C6F6E672050
:10276000657874727573696F6E2070726576656EC8
:102770007465640A0020636F6C64206578747275F8
:1027800073696F6E2070726576656E7465640A0099
:102790000000000000000000000000005761726EA1
:1027A000696E673A20486F6D696E672042756D707B
:1027B0002044697669736F72203C20310A0002025E
:1027C0000400809D4300009B430000C843000000BC
:1027D0004100000041000000400000000100000036
:1027E0000100008000555555000000400033333390
:1027F00000AAAA2A004992240000002000C7711CE8
:102800000099991900D1451700555515003BB11392
:10281000002449120011111100000010000F0F0FC9
:1028200000E3380E0043790D00CCCC0C00C3300C13
:1028300000E8A20B0064210B00AAAA0A00703D0A5E
:10284000009DD80900427B090092240900DCD308CE
:1028500000888808001042080000000800F0C10746
:10286000008787070075500700711C07003EEB06C4
:1028700000A1BC06006990060066660600703E0670
:10288000006118060017F4050074D105005BB0055F
:1028900000B29005006272050055550500783905B3
:1028A00000B81E0500050505004EEC040087D404A1
:1028B00000A1BD040090A7040049920400C17D045A
:1028C00000EE690400C7560400444404005C32046E
:1028D000000821040041100400000004003FF00340
:1028E00000F8E0030026D20300C3C30300CCB50305
:1028F000003AA803000A9B0300388E0300C081033E
:10290000009F750300D0690300505E03001D530350
:102910000034480300913D030033330300162903BC
:1029200000381F030097150300300C030003030356
:10293000000BFA020049F10200BAE802005CE00272
:10294000002DD802002DD0020059C80200B0C002EC
:102950000031B90200DAB10200AAAA0200A0A30263
:1029600000BC9C0200FA9502005C8F0200DF880226
:102970000082820200457C02002776020027700256
:1029800000436A02007C640200D05E02003F5902EC
:1029900000C8530200FFFDFCFAF8F6F4F2F0EEEC8A
:1029A000EAE9E7E5E3E1E0DEDCDAD9D7D5D4D2D055
:1029B000CFCDCBCAC8C7C5C3C2C0BFBDBCBAB9B7EB
:1029C000B6B4B3B2B0AFADACAAA9A8A6A5A4A2A153
:1029D000A09E9D9C9A99989795949392908F8E8D96
:1029E0008B8A8988878684838281807F7E7D7B7ABB
:1029F000797877767574737271706F6E6D6C6B6ABF
:102A0000696867666564636261605F5E5D5C5B5AAE
:102A10005958585756555453525150504F4E4D4C8B
:102A20004B4A4A4948474646454443424241403F53
:102A30003E3E3D3C3B3B3A3938383736353534330A
:102A400032323130302F2E2E2D2C2B2B2A292928B3
:102A5000272726252524232322212120201F1E1E4F
:102A60001D1C1C1B1B1A19191818171616151514DE
:102A7000131312121111100F0F0E0E0D0D0C0C0B63
:102A80000A0A0909080807070606050504040303DE
:102A9000020201000000809D4300009B430000C82B
:102AA00043000000000000000000000000536574B7
:102AB00074696E67732053746F7265640045455086
:102AC000524F4D20496E697469616C697A65640A78
:102AD000003B200020204D363033200020440020D1
:102AE000204D34313220530046696C616D656E743F
:102AF0002072756E6F75742073656E736F723A0015
:102B00002055004C0046696C616D656E74206C6FD9
:102B100061642F756E6C6F6164206C656E6774689C
:102B2000733A0020204D343133205300506F7765C5
:102B3000722D4C6F7373205265636F766572793AAC
:102B40000020440020490020204D33303420500024
:102B500020440020490020204D33303120500050C7
:102B600049442073657474696E67733A00204600A7
:102B700020480020204D3134352053004D617465CC
:102B80007269616C20686561747570207061726132
:102B90006D65746572733A002020473239205334D2
:102BA000205A00204A002020473239205333204940
:102BB0000020204D3432302053004D657368204290
:102BC0006564204C6576656C696E673A0020204D1F
:102BD000323036205800486F6D65206F6666736529
:102BE000743A0020580020530020204D3230352008
:102BF0004200416476616E6365643A20423C6D69CF
:102C00006E5F7365676D656E745F74696D655F7522
:102C1000733E20533C6D696E5F66656564726174D6
:102C2000653E20543C6D696E5F74726176656C5FC1
:102C300066656564726174653E20583C6D61785FBD
:102C4000785F6A65726B3E20593C6D61785F795F91
:102C50006A65726B3E205A3C6D61785F7A5F6A6587
:102C6000726B3E20453C6D61785F655F6A65726B93
:102C70003E0020540020520020204D32303420509D
:102C800000416363656C65726174696F6E202875BD
:102C90006E6974732F7332293A20503C7072696EDA
:102CA000745F616363656C3E20523C72657472614F
:102CB00063745F616363656C3E20543C747261763B
:102CC000656C5F616363656C3E0020204D3230317E
:102CD0002058004D6178696D756D20416363656CA6
:102CE00065726174696F6E2028756E6974732F73D5
:102CF00032293A0020204D3230332058004D61787F
:102D0000696D756D206665656472617465732028F0
:102D1000756E6974732F73293A005374657073204C
:102D200070657220756E69743A0020440020204D51
:102D30003230302053002044697361626C65640A4C
:102D40000046696C616D656E742073657474696E9C
:102D500067733A0020204D3134392043203B205501
:102D60006E69747320696E2043656C736975730AAC
:102D70000020286D6D29002020473231202020209E
:102D80003B20556E69747320696E206D6D000000E4
:102D9000FA430000FA430000204100009642000080
:102DA000A0420000A0420000C8430000BA42DC0577
:102DB0000000DC050000640000004B00000024F46B
:102DC000D43050C38E20C2A24017828B7011127A69
:102DD000910D816CD90AA861E108C7586607615155
:102DE00043061E4B5D05C145A7041A411104093D68
:102DF0009803713931034036DB0265339102D430D8
:102E00005402802E1D02632CEE01752AC501B028E4
:102E1000A001102781018F2564012B244B01E022A2
:102E20003401AC211F018D200D01801FFC00841E88
:102E3000ED00971DDF00B81CD200E61BC600201B6A
:102E4000BC00641AB200B219A8000A19A0006A18DE
:102E50009900D117910040178B00B51684003116E8
:102E60007E00B31579003A157300C7146F0058142B
:102E70006A00EE1366008813630025135E00C71214
:102E80005B006C12570015125400C11151007011F3
:102E90004F0021114B00D61049008D1047004610FD
:102EA000440002104200C00F4000800F3E00420F5D
:102EB0003C00060F3B00CB0E3800930E37005C0E33
:102EC0003500270E3400F30D3200C10D3100900D96
:102ED0003000600D2E00320D2D00050D2C00D90C98
:102EE0002B00AE0C2900850C29005C0C2700350C4A
:102EF00027000E0C2600E80B2400C40B2400A00BB6
:102F000023007D0B23005A0B2100390B2100180BE5
:102F10002000F80A1F00D90A1E00BB0A1E009D0AE5
:102F20001D00800A1D00630A1C00470A1B002C0AB2
:102F30001B00110A1A00F7091A00DD091900C4095B
:102F40001900AB091900920917007B0918006309E1
:102F500017004C09160036091600200916000A0948
:102F60001500F5081500E0081400CC081400B80896
:102F70001400A4081400900813007D0812006B08C8
:102F800013005808120046081200340811002308E4
:102F900011001208110001081100F0071000E007ED
:102FA0001000D0071000C0071000B0070F00A107E5
:102FB000100091070E0083070F0074070F006507CC
:102FC0000E0057070E0049070E003B070D002E07A5
:102FD0000E0020070D0013070D0006070D00F9066F
:102FE0000C00ED060D00E0060C00D4060C00C8062F
:102FF0000C00BC060C00B0060C00A4060B009906E1
:103000000C008D060B0082060B0077060B006C0689
:103010000B0061060A0057060B004C060A00420628
:103020000A0038060A002E060A0024060A001A06BC
:103030000A001006090007060A00FD050900F4054C
:103040000900EB050900E2050900D9050900D005D2
:103050000900C7050900BE050900B5050800AD0552
:103060000800A50509009C050800940508008C05CA
:103070000800840508007C050800740508006C053C
:103080000700650508005D050700560508004E05A8
:10309000070047050700400508003805070031050F
:1030A00007002A050700230507001C050600160572
:1030B00007000F0507000805060002050700FB04CE
:1030C0000600F5040700EE040600E8040600E2042A
:1030D0000700DB040600D5040600CF040600C9047F
:1030E0000600C3040600BD040600B7040600B104D0
:1030F0000500AC040600A6040600A00405009B041D
:10310000060095040500900406008A040500850465
:103110000500800406007A040500750405007004AB
:1031200005006B04050066040500610405005C04ED
:10313000050057040500520405004D04050048042D
:103140000500430405003E0404003A04050035046C
:103150000500300404002C040500270404002304A7
:1031600005001E0404001A040400160405001104DE
:1031700004000D0404000904050004040400000414
:103180000400FC030400F8030400F4030400F0034B
:103190000400EC030400E8030400E4030400E0037B
:1031A0000400DC030400D8030400D4030400D003AB
:1031B0000400CC030400C8030300C503030024F487
:1031C00004D9201BC40C5C0E9804C4095F02650777
:1031D0007101F405F900FB04B30048048700C10342
:1031E00069005803550003034500BE023A008402FB
:1031F000310053022A002902250004022000E401C4
:103200001C00C8011900AF011700980114008401C7
:103210001300710110006101100051010E00430103
:103220000D0036010B002B010B0020010B001501D6
:1032300009000C01090003010800FB000800F3006D
:103240000800EB000700E4000600DE000600D800DE
:103250000600D2000600CC000500C7000500C20031
:103260000500BD000400B9000400B5000400B10071
:103270000400AD000400A9000400A5000300A200A2
:1032800003009F0004009B000300980003009500CA
:10329000020093000300900003008D0002008B00E9
:1032A0000300880002008600020084000300810001
:1032B00002007F0002007D0002007B000200790016
:1032C0000200770001007600020074000200720024
:1032D0000100710002006F0002006D0001006C002F
:1032E00002006A0001006900020067000100660038
:1032F000010065000100640002006200010061003D
:103300000100600001005F0002005D0001005C0040
:1033100001005B0001005A00010059000100580043
:103320000100570001005600010055000100540043
:103330000100530000005300010052000100510041
:103340000100500001004F0001004E0000004E003F
:1033500001004D0001004C0001004B0000004B003B
:1033600001004A0001004900010048000000480037
:103370000100470001004600000046000100450032
:10338000000045000100440001004300000043002C
:103390000100420000004200010041000000410025
:1033A0000100400001003F0000003F0001003E001E
:1033B00000003E0001003D0000003D0001003C0017
:1033C00000003C0000003C0001003B0000003B000E
:1033D00001003A0000003A00010039000000390005
:1033E00001003800000038000000380001003700FC
:1033F00000003700010036000000360000003600F3
:1034000001003500000035000000350001003400E7
:1034100000003400000034000100330000003300DD
:1034200000003300010032000000320000003200D2
:1034300001003100000031000000310001003000C7
:10344000000030000000300001002F0000002F00BD
:1034500000002F0000002F0001002E0000002E00B1
:1034600000002E0001002D0000002D0000002D00A6
:1034700000002D0001002C0000002C0000002C009A
:1034800000002C0001002B0000002B0000002B008E
:1034900000002B0001002A0000002A0000002A0082
:1034A00000002A0001002900000029000000290076
:1034B0000000290000002900010028000000280069
:1034C000000028000000280000002800010027005C
:1034D0000000270000002700000027000000270050
:1034E0000100260000002600000026000000260043
:1034F0000000260001002500000025000000250036
:103500000000250000002500000025000100240027
:10351000000024000000240000002400000024001B
:10352000010023000000230000002300000023000E
:1035300000002300000023000000230001002200FF
:1035400000002200000022000000220000002200F3
:1035500000002200010021000000210000002100E5
:1035600000002100000021000000210000002100D7
:1035700001002000000020000000200000002000CA
:1035800000002000000020000000200000002000BB
:1035900001001F0000001F0000001F0000001F00AE
:1035A00000001F0000001F0000001F0001001E009F
:1035B00000001E0000001E0000001E000000393048
:1035C00000003325000087190000B00F0000DB0861
:1035D0000000BD040000740200003F010000204311
:1035E0006F756E7420583A00426564004531006280
:1035F0006564002C2073797374656D2073746F702B
:1036000070656421204865617465725F49443A20A1
:103610000048656174696E67204661696C65640085
:1036200048656174696E67206661696C6564004D08
:103630003131322053687574646F776E001000C9A1
:103640000210012C014001220170011801B0010E8D
:1036500001F00104015002FA00B002F0003003E66C
:1036600000D003DC009004D2007005C800A006BEA4
:10367000000008B400B009AA00D00BA000600E96AC
:103680000060118C000015820020197800C01D6EAA
:1036900000A0226400B0275A00902C500000314650
:1036A00000E0343C0010383200903A2800603C1EA4
:1036B00000A03D1400803E0A00203F000054484511
:1036C000524D414C2052554E415741590054686566
:1036D000726D616C2052756E61776179004572720E
:1036E0003A204D415854454D50004D415854454D98
:1036F0005020747269676765726564004572723A3A
:10370000204D494E54454D50004D494E54454D5065
:103710002074726967676572656400202F0020421B
:10372000403A0020403A0020573A0020573A0049DA
:103730006E76616C69642065787472756465720A6E
:10374000007C3C3E5E2B3D3F2F5B5D3B2C2A225C88
:103750000043616E6E6F74206F70656E20737562CA
:10376000646972200041425300504C410053442090
:10377000496E6974204661696C005344206361722C
:1037800064206F6B0A006F70656E526F6F742066F5
:1037900061696C65640A00766F6C756D652E696E83
:1037A0006974206661696C65640A004E6F20534439
:1037B00020636172640A000A4D3234004D323320B6
:1037C0002573002E0A006F70656E206661696C6556
:1037D000642C2046696C653A200046696C6520734C
:1037E000656C65637465640A002053697A653A20E4
:1037F0000046696C65206F70656E65643A2000450F
:103800004E4420535542524F5554494E450A0022CA
:1038100020706F73002220706172656E743A22000E
:10382000535542524F5554494E452043414C4C202C
:103830007461726765743A220053756263616C6CDF
:10384000204F766572666C6F7700457863656564B6
:103850006564206D617820535542524F5554494E4E
:10386000452064657074683A002E0A0044656C65F2
:1038700074696F6E206661696C65642C2046696CA2
:10388000653A200046696C652064656C6574656402
:103890003A005344207072696E74696E67206279D1
:1038A000746520004E6F74205344207072696E74EA
:1038B000696E670A002F6175746F25632E67005764
:1038C000726974696E6720746F2066696C653A204E
:1038D00000667265736800646F696E6700206669D0
:1038E0006C653A20004E6F77200002FD5555555506
:1038F000555FFFFFFFFFFFFFFFFFFFFE000000001F
:10390000003FFFFFFFFFFFFFFFFFFFFD000007FF7E
:10391000FFFFFFFFFFFFFFFFFFFFFFFE07C0055593
:10392000555555555FFFFFFFFFFFFFFC0A200600BE
:10393000000000003FFFFFFFFFFFFFFE1410050027
:103940000007FFFFFFFFFFFFFFFFFFFC2808060740
:10395000C00555555555555FFFFFFFFE5404040A39
:10396000200600000000003FFFFFFFFC600406147B
:103970001005000007FFFFFFFFFFFFFE50040428B3
:10398000080607C00555555555555FFC600406549B
:1039900004040A200600000000003FFE54041C60DE
:1039A000040614100500000000001FFC28082E501B
:1039B000040428080607C00001F03FFE14105460FC
:1039C00004065404040A200002081FFC0A2066545E
:1039D000041C60040614100005043FFE07C05428B0
:1039E000082E5004042808000A021FFC00002E14B0
:1039F000105460040654040015013FFE00001C0A28
:103A0000206654041C60040018011FFC0000060717
:103A1000C05428082E50040014013FFE000004008A
:103A2000002E14105460040018011FFCFFFFFE005C
:103A3000001C0A206654041C15013FFED555540095
:103A4000000607C05428082A0A021FFC84104600FA
:103A5000000400002E14105105043FFEC41044FF62
:103A6000FFFE00001C0A206102881FFC841046D55E
:103A7000555400000607C05101F03FFE84104484F5
:103A8000104600000400002A00001FFCC41046C4B9
:103A90001044FFFFFE00001C00003FFE8410448421
:103AA0001046D5555400000000001FFCD555568423
:103AB000104484104600000000003FFCFFFFFCC4DF
:103AC0001046C41044FFFFFFFFFF9FFE0000068466
:103AD0001044841046D555555555BFFD555554D500
:103AE000555684104484104104109FFFFFFFFCFFD3
:103AF000FFFCC41046C410410411BFFFFFFFFE00CD
:103B0000000684104484104104109FFFFFFFFD5500
:103B10005554D5555684104104109FFFFFFFFFFFF9
:103B2000FFFCFFFFFCC410410411BFFFFFFFFFFFBC
:103B3000FFFE00000684104104109FFFFFFFFFFFFF
:103B4000FFFD555554D555555555BFFFFFFFFFFF98
:103B5000FFFFFFFFFCFFFFFFFFFF9FFFFFFFFFFFD8
:103B6000FFFFFFFFFE00000000003FFFFFFFFFFF21
:103B7000FFFFFFFFFD55555555555FFFFFFFFFFF49
:103B8000FFFFFFFFFFFFFFFFFFFFFFFFFFFFFFFF45
:103B9000FFFFFFFFFFFFFFFFFFFFFFFFFFFFFFFF35
:103BA000FFFFFFFFFFFFFFFFFFFFFFFFFFFFFFFF25
:103BB000FFFFFFFFFFFFFFFFFFFFFFE02EFB7DFB8F
:103BC000FBCFC1DFBB3EC0E1FE3C1FFDEE7B39F900
:103BD000F3CF9EDFBB3EDFDEFCDDE7FDEE3BBBF956
:103BE000EBD7BF5FBB5EDFDEFDEDF7FDEEBBD3FACB
:103BF000EBB73FDFBB4EDFDFFFCDF3FDEEDBC7FAF8
:103C0000EBBB7FC03B6EC0E3FF1DF3FDEECBEFFAD5
:103C1000DBBB7FDFBB66DFF8FFCDF3FDEEEBEFFB39
:103C20005B033F5FBB76DFFE7FEDF3FDEEF3EFFB63
:103C30005B79BEDFBB7ADFDE7DEDF7FDEEF3EFFBF8
:103C4000BAFD9EDFBB7CDFDEFDCDE7FDEEFBEFFBCB
:103C5000BAFDC1DFBB7EC0E0FE1C1F6D61726C69E6
:103C60006E66772E6F726700322E302E375F4457A4
:103C7000372E33001FFFFFFFFFFFFF600000000033
:103C800001FF400000000000FF8000000000007FF6
:103C900083CF00000C303F87FF80000C301F8679F7
:103CA00080000C000F8C30C7838C30E78C30CFC77E
:103CB000CC31F38C30DCECEC33B98C30D86C6C3319
:103CC000198C30D06C0C33198C30D86C0C33198CA7
:103CD00030DC6C0E3B198C30CF7C079F198C30C7C1
:103CE0007C038F194000000000000260000000000B
:103CF00000061FFFFFFFFFFFF86001F4017001EAFB
:103D0000019001E001B001D601D001CC010002C256
:103D1000013002B8016002AE019002A401D0029A03
:103D2000012003900170038601C0037C01300472FE
:103D300001A004680120055E01B005540160064A37
:103D40000120074001F0073601F0082C01100A227B
:103D500001500B1801C00C0E01500E04013010FA76
:103D6000002012F0005014E600C016DC007019D2DA
:103D700000501CC800501FBE007022B400B025AA1D
:103D800000F028A000202C9600302F8C00103282EA
:103D900000A0347800F0366E00E0386400803A5AB3
:103DA00000403B5500E03B5000F03C4600C03D3C2D
:103DB00000603E3200E03E2800303F1E00503F19B8
:103DC00000703F1400A03F0A00C03F0000D03FF643
:103DD000FFE03FECFF2020506C616E6E6572427513
:103DE0006666657242797465733A20002046726592
:103DF00065204D656D6F72793A2000436F6D706973
:103E00006C65643A20417072203234203230323195
:103E10000A00204C61737420557064617465643AC3
:103E200020323032312D30342D3138207C20417514
:103E300074686F723A2054696E794D616368696E77
:103E4000657333440A00322E302E375F4457372EC5
:103E5000330A004D61726C696E0020536F6674778F
:103E60006172652052657365740A0020576174633E
:103E700068646F672052657365740A002042726F30
:103E8000776E206F75742052657365740A00204543
:103E9000787465726E616C2052657365740A0050A7
:103EA0006F77657255700A0073746172740A004707
:103EB00032385859004D31303031006572726F72AE
:103EC0002077726974696E6720746F2066696C650B
:103ED0000A00446F6E6520736176696E67206669BB
:103EE0006C652E0A004D323900456E6473746F7034
:103EF0007300255320256320256320256320256337
:103F000000205A3A0020593A0020583A00656E6461
:103F100073746F7073206869743A200000000A0B94
:103F200002090C0D0E080703040100000000000048
:103F30000000000000000000000000000000000081
:103F4000000000000000000012111000000000003E
:103F50000000000000000000000000000000000061
:103F60000000004D6F76652025736D6D004D6F76F6
:103F70006520302E316D6D004D6F766520316D6D91
:103F8000004D6F76652031306D6D004D6F76652088
:103F900041786973004578747275646572004D6F7D
:103FA0007665205A004D6F76652059004D6F766515
:103FB000205800693765374368616E676520466938
:103FC0006C616D656E7400556E6C6F61642046693E
:103FD0006C616D656E74004C6F61642046696C6144
:103FE0006D656E7400507265686561742043757309
:103FF000746F6D00507265686561742024004261C1
:10400000636B00FFFFFF486F6D65202573257325E7
:10401000732046697273740073686F7700627574F9
:10402000746F6E00626567696E0044697361626CEB
:104030006552756E6F75740050757267654D6F725D
:10404000650050617573656400436F6E74696E75C9
:1040500065004C6F61642046696C616D656E74200B
:104060005400496E736572742066696C616D656E8B
:104070007420616E642073656E64204D3130380A9F
:1040800000220A00556E6B6E6F776E20636F6D6D48
:10409000616E643A2022002042002050006F6B00C5
:1040A000544D3344204352313056322052656164BE
:1040B000792E005072696E74696E672E2E2E005034
:1040C00072696E742050617573656400204500202C
:1040D0005A00205900204D393220580020453A001E
:1040E000205A3A0020593A00583A0020746F6F2045
:1040F0006C6F6E6720657874727573696F6E20706F
:10410000726576656E7465640A0020636F6C642066
:10411000657874727573696F6E2070726576656EFE
:104120007465640A00526573656E643A20006E6FB0
:1041300074696669636174696F6E20000000220013
:10414000250028002B002E00310034000201000061
:10415000050108010B0100002100240027002A00AE
:104160002D003000330001010000040107010A01A5
:1041700005050505070508080808020202020A0AE3
:104180000808040404040101010101010101030301
:10419000030303030303040707070C0C0C0C0C0CAC
:1041A0000C0C0202020206060606060606060B0BA9
:1041B0000B0B0B0B0B0B01021020200808102040EA
:1041C00010204080020102010804020101020408DB
:1041D0001020408080402010080402018004020169
:1041E00080402010080402010804020101020408B2
:1041F0001020408001020408102040809A01320102
:1042000011241FBECFEFD1E2DEBFCDBF00E00CBF57
:1042100013E0A0E0B2E0EAEFF4EB02E00BBF02C073
:1042200007900D92A836B107D9F728E1A8E6B3E0C8
:1042300001C01D92AF30B207E1F710E2CFEFD0E23C
:1042400000E006C021970109802FFE010F94D3568C
:10425000CE3FD10780E00807A9F70F9485450D945C
:104260006B5A0C940000FC0184910895FC0180813C
:1042700008951198000000009091020187FD90952B
:10428000917090930001119A00000000000000005E
:104290001198000000009091020186FD90959170A8
:1042A00090930001119A0000000000000000119896
:1042B000000000009091020185FD9095917090930F
:1042C0000001119A00000000000000001198000099
:1042D00000009091020184FD9095917090930001EF
:1042E000119A00000000000000001198000000007A
:1042F0009091020183FD9095917090930001119A25
:1043000000000000000000001198000000009091E3
:10431000020182FD9095917090930001119A000026
:1043200000000000000011980000000090910201C0
:1043300081FD9095917090930001119A000000000A
:1043400000000000119800000000809102018170BF
:1043500080930001119A0000000000000000089501
:1043600090E080E00895CF93DF93DB01F9019C9109
:104370009130C1F0943080F094509C938830D1F407
:1043800080819181009771F0019791838083480F1C
:10439000591FEA01188206C08C3539F49C5F9C9342
:1043A000943041F4DF91CF9108958B3339F781E058
:1043B0008C93F8CF20813181B9016F5F7F4F71837A
:1043C0006083420F531FEA018883808191818F357A
:1043D00091056CF7E7CF0F931F9381E00091D815FB
:1043E0001091D9152091DA153091DB154091D41533
:1043F0005091D5156091D6157091D71504171507F2
:104400002607370708F480E01F910F91089590E088
:1044100080E00895282F90916308833021F495FD62
:104420000FC094FD0FC0892F90E0B0E0A0E004C061
:10443000B695A795979587952A95D2F78170089597
:1044400081E0089580E0089510924A088091510219
:1044500090915202A0915302B09154028093390678
:1044600090933A06A0933B06B0933C060895129AA7
:104470000895269A2E9A0895AF92BF92CF92DF9216
:10448000EF92FF920F931F93CF93DF936B01E9019C
:104490004A3009F4C1C0453109F073C0DB011296FE
:1044A000ED91FC91F280C681D781809102018095C7
:1044B00082708093000188E28A950000E9F7BF2CA2
:1044C000B29420EFB22230E1A32EAF0C48E2E42EEA
:1044D00088EF0E9439218E2D8A950000E9F7BFE10F
:1044E000BF1508F485C08F2D807780680E94392120
:1044F0008B2D0E9439218E2D8A950000E9F780E8E6
:104500000E94392180E00E9439218E2D8A95000079
:10451000E9F78AEF0E9439218E2D8A950000E9F78C
:104520008E01005F1F4F8881807F0E943921899111
:104530008295807F0E943921C017D107A1F78E2D67
:104540008A950000E9F7F394E0E1BE0EFA10C0CFBF
:1045500080910201827080930001D6011296CD9164
:10456000DC91CE010F949D38811147C2DF91CF912C
:104570001F910F91FF90EF90DF90CF90BF90AF9081
:104580000895FB0102811381423309F4F1C108F45B
:10459000F5C1463409F4E2C1473409F4E5C14B33AF
:1045A00029F589812B81D80112966C911297139667
:1045B0004C91213009F438C2233009F002C238EF9F
:1045C000380F582F91E0431708F490E041E053175B
:1045D00008F040E031E0561708F430E0592F542B32
:1045E000352309F016C2942309F013C281E0BECF2F
:1045F00080EE8F0D8068807F0E9439218F2D8295FB
:10460000807F0E9439218E2D8A950000E9F780E88D
:104610000E94392180E877CF8091010182608093E8
:10462000010180910201827080930001809101015B
:10463000816080930101809102018170809300016B
:10464000099A119A809102018095827080930001ED
:1046500088E28A950000E9F788E790E0CEE9DFE09C
:10466000FE013197F1F70197D9F788EF0E943921C0
:1046700018E2812F8A950000E9F780E20E94392133
:1046800080E00E943921812F8A950000E9F780E0BF
:104690000E94392180E80E943921812F8A950000EB
:1046A000E9F780E00E94392180E10E943921812FC1
:1046B0008A950000E9F7CE010197F1F7CE01019745
:1046C000F1F7CE010197F1F7CE010197F1F7CE0195
:1046D0000197F1F7CE010197F1F7CE010197F1F7BC
:1046E000CE010197F1F7CE010197F1F7CE010197C5
:1046F000F1F7CE010197F1F7CE010197F1F7CE0165
:104700000197F1F7CE010197F1F72197F1F780E2D8
:104710000E94392180E40E943921812F8A9500006E
:10472000E9F780E20E94392180E60E9439211A953A
:104730000000E9F710E0D0E0C8E28D2F80778068B4
:104740000E943921812F0E9439218C2F8A950000E7
:10475000E9F780E80E94392180E00E9439218C2FFE
:104760008A950000E9F78AEF0E9439218C2F8A95FB
:104770000000E9F790E2119800000000809102012A
:10478000817080930001119A000000000000000079
:104790001198000000008091020181708093000157
:1047A000119A0000000000000000119800000000B5
:1047B00080910201817080930001119A0000000035
:1047C000000000001198000000008091020181703B
:1047D00080930001119A0000000000000000119871
:1047E0000000000080910201817080930001119A05
:1047F00000000000000000001198000000008091FF
:104800000201817080930001119A000000000000F5
:1048100000001198000000008091020181708093D7
:104820000001119A00000000000000001198000033
:10483000000080910201817080930001119A0000B4
:1048400000000000000011980000000080910201AB
:10485000817080930001119A0000000000000000A8
:104860001198000000008091020181708093000186
:10487000119A0000000000000000119800000000E4
:1048800080910201817080930001119A0000000064
:10489000000000001198000000008091020181706A
:1048A00080930001119A00000000000000001198A0
:1048B0000000000080910201817080930001119A34
:1048C000000000000000000011980000000080912E
:1048D0000201817080930001119A00000000000025
:1048E0000000119800000000809102018170809307
:1048F0000001119A00000000000000001198000063
:10490000000080910201817080930001119A0000E3
:104910000000000000008C2F8A950000E9F79150FC
:1049200009F029CF88EF0E9439218C2F8A95000049
:10493000E9F7DF5F105FD03209F0FFCE80E00E9420
:10494000392180EC0E943921CA950000E9F7809155
:10495000020182708093000181E008CED801159693
:104960008C91888381E002CEF80181818883FACF1F
:10497000B901C8010F94BA3881E0F8CD443171F023
:10498000473109F033CE1882F8018281898385810D
:1049900081508A8383818B8381E0E8CDD80115968D
:1049A0004C91159750E0440F551F70E060E016964B
:1049B0008D919C910F940C5AC8010F94B33881E0EB
:1049C000D5CD481708F412CE861708F40FCEFA801A
:1049D000E12CD12C243070F41DC0BE01C8010F940D
:1049E000BA38898198819D0D98838E0D8983FF0C3B
:1049F00009F4FCCDF7FEF6CFF0CF4D8150E0440F27
:104A0000551F70E060E08E819F810F940C5A81E009
:104A1000ADCDFA8030E0F901ED55FD4FD080215643
:104A20003D4FF901E080E6CF58E0580F382FCACD4E
:104A3000EF92FF920F931F93CF93DF93EC018B01C3
:104A40007A018A859B858617970731F0888199813D
:104A50000F94933A1B870A87B701888199810F9435
:104A6000822C2E813F81820F932F911D9F838E83F5
:104A700090E080E0DF91CF911F910F91FF90EF9038
:104A800008959F92AF92BF92CF92DF92EF92FF92E2
:104A90000F931F93CF93DF93EC018B01942EA52EE0
:104AA0008A859B858617970731F0888199810F94B5
:104AB000933A1B870A8788859985019649F5BC80BA
:104AC0000A818E81080FC880D980D6015596ED9154
:104AD000FC91C6011995B80EE92CFA2C10E0F701EB
:104AE00021917F01211127C08E819F81810F911D0E
:104AF0009F838E8390E080E0DF91CF911F910F9193
:104B0000FF90EF90DF90CF90BF90AF909F9008956F
:104B10000E811F81692D7A2D888199810F94822CB5
:104B2000800F912F911D288539852817390738F670
:104B300081E090E0E1CF4B2D602FC6010F94EB3A5E
:104B4000080F180FCCCFDF92EF92FF920F931F93B5
:104B5000CF93DF93EC01D62E1CAD0BAD7C0184E02E
:104B6000E80EF11CE98DFA8DC7011995412F480F08
:104B70002D2D602FC7010F94EB3A9BAD890F8BAFA2
:104B800081E090E0DF91CF911F910F91FF90EF9026
:104B9000DF900895AB01BC014093D8155093D9150F
:104BA0006093DA157093DB158FE397E10C942FCFA8
:104BB000809323028032B8F590910405891724F080
:104BC00091E0980F909304054091000550910105E4
:104BD0006091020570910305082E04C076956795D3
:104BE000579547950A94D2F7417040939B0F87FDE4
:104BF0001DC0282F082E000C330B3F938F9386E89F
:104C000099E09F938F9386E999E09F938F931F92EA
:104C10000E946EB38DB79EB707960FB6F8949EBFED
:104C20000FBE8DBF089510929B0FE1CF0D940B40E6
:104C30000F931F93CF93DF9300D01F92CDB7DEB7B2
:104C40009C0101E318E090E1E6EEFFE0D80101905D
:104C50000D929A95E1F7F9012081318142815381CA
:104C6000F80160857185828593850F94DC56F80183
:104C7000608771878287938780E090E0A0EAB0E444
:104C800089839A83AB83BC83CE0101960E94C8F7C7
:104C90000F900F900F900F90DF91CF911F910F9178
:104CA00008952F923F924F925F926F927F928F92D0
:104CB0009F92AF92BF92CF92DF92EF92FF921F939B
:104CC000CF93DF93CDB7DEB72C970FB6F894DEBF46
:104CD0000FBECDBF7A011901DC012D913D914D919F
:104CE0005C912D833E834F835887FB014080518028
:104CF000628073808090E60F9090E70FA090E80F9D
:104D0000B090E90FA50194016D817E818F81988516
:104D10000F94EA4F81110EC011E0A301920160913E
:104D2000EA0F7091EB0F8091EC0F9091ED0F0F94C3
:104D3000EA4F811110E0D1012D913D914D915C918F
:104D400029873A874B875C87F701C080D180E28052
:104D5000F3802091090230910A0240910B02509198
:104D60000C02C701B6010F94EA4F882309F44EC024
:104D7000C0920902D0920A02E0920B02F0920C0259
:104D80008091F20F9091F30FA091F40FB091F50F75
:104D90004091EA0F5091EB0F6091EC0F7091ED0F85
:104DA0008092310890923208A0923308B092340871
:104DB000409335085093360860933708709338084D
:104DC000C0923908D0923A08E0923B08F0923C0831
:104DD00080933D0890933E08A0933F08B09340080D
:104DE00020E030E040E05FE36091C90F7091CA0FAE
:104DF0008091CB0F9091CC0F0F94505069837A83A0
:104E00008B839C83CE0101960E94C8F72D813E8141
:104E10004F815885209331083093320840933308EE
:104E20005093340840923508509236086092370803
:104E300070923808D1012D913D914D915C91609116
:104E40003D0870913E0880913F08909140080F9472
:104E5000DC5660933D0870933E0880933F08909322
:104E6000400811112FC020E030E0A90169857A8542
:104E70008B859C850F94EA4F811133C060E070E010
:104E800088EC92E469837A838B839C83CE010196BC
:104E90000E94C8F72C960FB6F894DEBF0FBECDBFA8
:104EA000DF91CF911F91FF90EF90DF90CF90BF9057
:104EB000AF909F908F907F906F905F904F903F90BA
:104EC0002F9008952AEF3EE74AE25FE36091CD0F0D
:104ED0007091CE0F8091CF0F9091D00F0F945050C2
:104EE000D1CF60E070E080EA91E4CCCF8091BB0448
:104EF0009091BC04009731F04AE050E070E060E02F
:104F00000D94054E60E070E0CB01089580915C093E
:104F100082FF0BC063E682E79AE00E9489B30F9498
:104F2000A7320E9454BA81E0089580E008958091EC
:104F3000BB049091BC04009731F04AE050E070E06F
:104F400060E00D94D74C60E070E0CB010895AF9223
:104F5000BF92CF92DF92EF92FF920F931F93CF9366
:104F6000DF93EC015B018A01FB01199587FD16C0F7
:104F7000C82ED12CF12CE12C2196F801C082D182CF
:104F8000E282F382CE01DF91CF911F910F91FF90CA
:104F9000EF90DF90CF90BF90AF900895982F907EC4
:104FA000903CA9F48F7190E0B0E0A0E06C017D012D
:104FB00056E0CC0CDD1CEE1CFF1C5A95D1F7CE013F
:104FC0000196F50119958F73C82A2296D6CF982F8E
:104FD000907F903E11F58F7090E0B0E0A0E06C0102
:104FE0007D0136E0CC0CDD1CEE1CFF1C3A95D1F7A0
:104FF000CE010196F50119958F73C82A46E0CC0CB5
:10500000DD1CEE1CFF1C4A95D1F7CE010296F5017E
:1050100019958F73C82A2396B0CF982F987F903F09
:1050200079F5877090E0B0E0A0E06C017D0186E04A
:10503000CC0CDD1CEE1CFF1C8A95D1F7CE0101962D
:10504000F50119958F73C82A96E0CC0CDD1CEE1C77
:10505000FF1C9A95D1F7CE010296F50119958F7331
:10506000C82A26E0CC0CDD1CEE1CFF1C2A95D1F7CB
:10507000CE010396F50119958F73C82A24967DCF2A
:10508000982F907C903841F4807C803869F4219688
:10509000CE01F5011995F8CF8E7F8D3F28F021962E
:1050A000CE01F5011995F8CFC12CD12C760165CF31
:1050B0009CE0899F802D112491E0980F9093050525
:1050C0002CE0280F20932B0830E02E5F3F4F4091BB
:1050D000A2154217130619F014F080E008952091EC
:1050E000A4159217D0F7662341F08E5F0F94AD3967
:1050F00080912B088E5F0F94AD3980912B08909191
:10510000A215891750F32091A41590910505291730
:1051100020F31092A5158093A61581E00895CF93F2
:105120008091F704811154C01092A5151092A61514
:105130001092A71510927315109272151092751592
:10514000109274151092771581E08093761582E2A3
:105150008093781510927D1510927C15E1E9F5E1A8
:105160002FE935E18FEF81932E173F07E1F7C1E07B
:10517000C0938E1520E131E0309384152093831580
:10518000C0938515109286151092871590E4909320
:105190008815109289152AE232E03093A0152093E9
:1051A0009F1526E132E0309371152093701597E139
:1051B0009093951591E19093961590E190939315A6
:1051C00080939215809391150F94D438C093F7046F
:1051D00081E08093F8048FE197E190930F1580931D
:1051E0000E151092111510921015CF91089520915F
:1051F000F604022E000C330B8217130641F0809345
:10520000F6046FE177E18EE695E10D94933A089507
:10521000CF92DF92EF92FF920F931F93CF93DF9382
:10522000CDB7DEB72C970FB6F894DEBF0FBECDBF5B
:105230006F3F71058105910509F0D0F48AE695E18B
:105240000E94A325E0917215F09173153196849117
:1052500090E02C960FB6F894DEBF0FBECDBFDF9165
:10526000CF911F910F91FF90EF90DF90CF90089515
:10527000F090A515E090A6152091F80421110FC01B
:105280004FEF56E16E2D8F2D0F94573B90E080E04D
:10529000F80EF092A515E092A6159927DACFC090E6
:1052A0007215D09073152EE635E13A8329832F2DA0
:1052B00030E03C832B832E2D30E03E832D831886F7
:1052C0001F822FEF3FEF3A8729871C861B8601E458
:1052D00015E29E012F5F3F4FAB01BC01C6010F9449
:1052E0002524B6018EE695E10F94933A8F81988537
:1052F000CFCFCF93DF93FC0125AD211104C021E076
:1053000025AF0F94D438C0917015D0917115E091EC
:105310009F15F091A01582E01995E0919F15F091ED
:10532000A01581E0199530E020E044E1BE018EE651
:1053300095E10F94D03821EA35E147E1BE018EE6D0
:1053400095E10F94D038E0919F15F091A01580E081
:10535000DF91CF911994CF92DF92EF92FF920F934A
:105360001F93CF93DF93CDB7DEB72C970FB6F8948A
:10537000DEBF0FBECDBFF090A515E090A615209121
:10538000F80421111DC04FED56E16E2D8F2D0F94A5
:10539000573B90E080E0F80EF092A515E092A6153C
:1053A00099272C960FB6F894DEBF0FBECDBFDF91C4
:1053B000CF911F910F91FF90EF90DF90CF900895C4
:1053C000C0907215D09073152EE635E13A8329838B
:1053D0002F2D30E03C832B832E2D30E03E832D8318
:1053E00018861F827A8769871C861B8601E415E26E
:1053F0009E012F5F3F4F43E351E2BC01C6010F9472
:10540000E924B6018EE695E10F94933A8F81988551
:10541000C2CF6FEF7FEF0C94AB29CF92DF92EF9268
:10542000FF920F931F93CF93DF93CDB7DEB72C97E7
:105430000FB6F894DEBF0FBECDBFF090A515E0907B
:10544000A6152091F80421111DC04FEB56E16E2DD9
:105450008F2D0F94573B90E080E0F80EF092A51549
:10546000E092A61599272C960FB6F894DEBF0FBED2
:10547000CDBFDF91CF911F910F91FF90EF90DF9003
:10548000CF900895C0907215D09073152EE635E137
:105490003A8329832F2D30E03C832B832E2D30E05F
:1054A0003E832D8318861F827A8769871C861B8618
:1054B00001E415E29E012F5F3F4F46E351E2BC013C
:1054C000C6010F94E924B6018EE695E10F94933A54
:1054D0008F819885C2CFBF92CF92DF92EF92FF92D9
:1054E0000F931F93CF93DF938B01F42EE90141FBC0
:1054F000662760F90E945828882309F45AC0B12C05
:105500000115110521F0C8010E9425BBB82EE12C20
:10551000209721F0CE010E9410BDE82E80E8C82E11
:10552000D12CF0FE1EC085E190E08B199109B7FCEB
:1055300093958E199109E7FC939597FD01969595A2
:105540008795F82E30E8C32ED12CFA94F7FC09C0C9
:1055500060E270E080E090E00E940829C81AD90A51
:10556000F4CFBB2099F0C60166E070E00F94AB5613
:10557000262F40912D0850912E0860912C08C801CB
:105580000E9465BA96E0899F60011124EE2031F0F7
:10559000B601CE010E940D2AC81AD90A87E0C816A2
:1055A000D10438F060E270E080E090E00E940829C9
:1055B000F3CFDF91CF911F910F91FF90EF90DF908C
:1055C000CF90BF9008956FEF7FEF0C940D2AAF92AC
:1055D000BF92CF92DF92EF92FF920F931F93CF93E0
:1055E000DF935C016B010E9425BBE82EC6010E947F
:1055F00010BDF12C03E110E0081B1109C5E20E15E6
:105600001F050CF4CFE18C2F90E09C012E5F3F4FE3
:105610004091A2154217130609F0CCF50997209185
:10562000A415281719069CF140912D0850912E08B9
:1056300060912C081092A515C093A61525E1C5010F
:105640000E9465BAD1E0C114D104B1F06AE370E000
:1056500080E090E00E9408290E151F05D4F4C45F75
:105660008091A215C81740F02091A4154C2F4950E5
:10567000550B241715067CF4DF91CF911F910F91E4
:10568000FF90EF90DF90CF90BF90AF900895D0E063
:10569000DACFDD2389F3802F880F080F000F0093E6
:1056A000A515C093A61560E270E080E090E00E942E
:1056B0000829C601DF91CF911F910F91FF90EF90C4
:1056C000DF90CF90BF90AF900C94E32A8F929F927F
:1056D000AF92BF92CF92DF92EF92FF920F931F9300
:1056E000CF93DF93CDB7DEB72C970FB6F894DEBF1C
:1056F0000FBECDBF982F862F5A017901D02E692F6A
:105700000E945828882309F489C0C701002391F119
:105710000E9425BBC82E80907215909073158091C1
:10572000F804811145C01FEF23E12C1940912D0889
:1057300050912E0860912C08C5010E9465BACC20BA
:1057400009F46CC0B6E08B9F500111246AE370E04D
:1057500080E090E00E94082957E0A516B10408F403
:1057600044C060E270E080E090E00E940829A81A3E
:10577000B90AF2CF0E9410BDC82E80907215909089
:1057800073158091F804882371F2FE0133968AE044
:10579000DF011D928A95E9F78EE695E19A83898368
:1057A00008E115E29E012F5F3F4F46E351E212C030
:1057B000FE0133968AE0DF011D928A95E9F78EE6B5
:1057C00095E19A83898308E115E29E012F5F3F4F9F
:1057D00043E351E2B701C4010F94E924B4018EE61A
:1057E00095E10F94933A1F819FCF40912B08212F71
:1057F00030E0A6E0CA9EC00111242E5F3F4F28175B
:1058000039070CF49C0180E8821B8093A515409316
:10581000A615C701DD20A9F00E94092A2C960FB613
:10582000F894DEBF0FBECDBFDF91CF911F910F91D6
:10583000FF90EF90DF90CF90BF90AF909F908F90B0
:1058400008950E94E32AEACFEAE6F5E183AF64AF68
:10585000CA010C94E32A2F923F924F925F926F926B
:105860007F928F929F92AF92BF92CF92DF92EF92F0
:10587000FF920F931F93CF93DF93D62FC72FFC0177
:1058800080809180A280B380C501B40120E831E519
:1058900041E050E00F942E56C9016DE671E00F947F
:1058A000AB566B017C01C501B40120E13EE040E054
:1058B00050E00F942E56CA01B90128E130E040E0D3
:1058C00050E00F942E56362E272E062F172F8CE3DE
:1058D000482E512C612C712CC501B401A3019201F9
:1058E0000F942E56B62EA72ECA01B901A30192011C
:1058F0000F942E56CB01C114D10479F1AF92BF920F
:105900007F936F932F923F92FF92EF92DF92CF920D
:105910008DE195E19F938F93CF93DF930F94814F08
:105920008DB79EB70E960FB6F8949EBF0FBE8DBF73
:105930008D2F9C2FDF91CF911F910F91FF90EF90B2
:10594000DF90CF90BF90AF909F908F907F906F909F
:105950005F904F903F902F900895E114F104C9F0AB
:10596000AF92BF927F936F932F923F92FF92EF92ED
:105970008DE095E19F938F93CF93DF930F94814FA9
:10598000EDB7FEB73C960FB6F894FEBF0FBEEDBF65
:10599000CFCF012BB9F0AF92BF927F936F932F922D
:1059A0003F9281E095E19F938F93CF93DF930F9484
:1059B000814F8DB79EB70A960FB6F8949EBF0FBE63
:1059C0008DBFB6CF892BA9F0AF92BF927F936F9313
:1059D00089EF94E19F938F93CF93DF930F94814F3F
:1059E000EDB7FEB738960FB6F894FEBF0FBEEDBF09
:1059F0009FCFAF92BF9285EF94E19F938F93CF9308
:105A0000DF930F94814F0F900F900F900F900F9096
:105A10000F908ECF8F929F92AF92BF92CF92DF92D4
:105A2000EF92FF920F931F93CF93DF931092F504A1
:105A30001092F4042FE32093F3041092F2041092D6
:105A4000F1041092F0041092EC041092ED04109204
:105A5000EE041092EF049C01F90190812F5F3F4FFB
:105A60009032D1F39E34C9F4818190ED980F9A3031
:105A700020F08D3211F08B3281F432969F012F5F2E
:105A80003F4F808180538A3008F47BC09F012F5F95
:105A90003F4F8081803209F476C0F0935008E09344
:105AA0004F088F010F5F1F4FC0816AE270E0C8018D
:105AB0000F94315A009731F0FC0131978081803288
:105AC000E1F31182CD3429F0C43519F0C73409F05F
:105AD0004BC0F80180810F5F1F4F8032D1F380539C
:105AE0008A3008F041C0C093F30430E020E04AE07F
:105AF000DF011196429FC001439F900D11249C012C
:105B0000205331098081280F311D87FD3A9581810D
:105B100090ED980F9A30C8F13093F2042093F1047D
:105B20008E3261F4329690E04AE0DF0131968C913A
:105B300050ED580F5A3058F19093F004CD01DC012C
:105B400001964C914032D9F3CD3489F52E3131058F
:105B500039F018F52731310519F02C31310539F5B7
:105B6000B093F504A093F404DF91CF911F910F91AE
:105B7000FF90EF90DF90CF90BF90AF909F908F906D
:105B80000895F9017BCFF90181CFFD01B1CF949F39
:105B9000800D112490ED980FC8CF2537310538F0CE
:105BA00027373105E8F2203A83E03807C9F2D0916F
:105BB0004F0840E050E0BA0110E000E0C12CD12CC9
:105BC0007601C394FD0131968C91882309F47FC03E
:105BD0008132E1F4CD34D1F420323105B9F440936F
:105BE000EC045093ED046093EE047093EF04F09393
:105BF000F504E093F40463E270E0CF010F94315AAE
:105C0000009709F4B1CFFC011082AECF81548A31E4
:105C100008F058C0DF019D91903291F0A0EDA90FDE
:105C2000AA30E8F09E3271F4918190539A30B8F026
:105C30000115110519F48F010150110990E013C0ED
:105C4000FD01E8CF9D3211F09B3291F79181A0EDDB
:105C5000A90FAA3020F09E3259F79281E6CF9E2FED
:105C60009D1B309759F3A82FB0E04601570104C09F
:105C7000880C991CAA1CBB1C8A95D2F74829592963
:105C80006A297B29AE52BB4F9C9380818154DF01EE
:105C90008A3108F497CFDF018191882309F492CFEC
:105CA00090ED980F9A30B8F393ED980F923098F3E7
:105CB0008B3289F3CD010196EC91E03209F082CF6D
:105CC000DC01F8CF0115110501F78D01DECF10932E
:105CD000F5040093F4044093EC045093ED046093B6
:105CE000EE047093EF0440CF9B01AC01485F5F4F1F
:105CF000BC016C5F7F4F0C9451260F931F93CF9381
:105D0000DF9300D000D01F921F92CDB7DEB7FC0109
:105D10008B0183A5811112C081E083A784819581C5
:105D2000A681B781B05889839A83AB83BC83BE01B7
:105D30006F5F7F4F81E398E00E94742E1D821E8268
:105D40001F82188620E030E040E05FE36091EE0FB4
:105D50007091EF0F8091F00F9091F10F0F94DC563E
:105D600069837A838B839C839E012B5F3F4FAE01B7
:105D70004F5F5F4F6AEE7FE086EE9FE00E94512604
:105D80001D821E821F82188620E030E040E05FE323
:105D9000F80160857185828593850F94DC5669834F
:105DA0007A838B839C83B8016C5F7F4F9E012B5F4E
:105DB0003F4FAE014F5F5F4FC8010E9451262896AA
:105DC0000FB6F894DEBF0FBECDBFDF91CF911F910C
:105DD0000F9108952F923F924F925F926F927F9210
:105DE0008F929F92AF92BF92CF92DF92EF92FF92EB
:105DF0000F931F93CF93DF93CDB7DEB7A2970FB664
:105E0000F894DEBF0FBECDBF8C011B015E834D83B6
:105E10004090E60F5090E70F6090E80F7090E90F08
:105E20008090EA0F9090EB0FA090EC0FB090ED0FE8
:105E3000DB018D919D910D90BC91A02D8F87988B4A
:105E4000A98BBA8B9C01AD01C301B2010F94DB5643
:105E50006B017C01D10114968D919D910D90BC91A7
:105E6000A02D8B8B9C8BAD8BBE8B9C01AD01C50196
:105E7000B4010F94DB566F8B788F898F9A8FAD8129
:105E8000BE818D919D910D90BC91A02D8F8398879F
:105E9000A987BA879C01AD01C301B2010F94DB56FB
:105EA0006B8F7C8F8D8F9E8FAD81BE8114968D916F
:105EB0009D910D90BC91A02D8B879C87AD87BE874F
:105EC0009C01AD01C501B4010F94DB566F8F78A31F
:105ED00089A39AA3A7019601C701B6010F94505058
:105EE0006B017C012F89388D498D5A8DCA01B9010A
:105EF0000F9450509B01AC01C701B6010F94DC56C2
:105F00004B015C012F85388949895A896F817885D1
:105F100089859A850F94DB562B013C012B893C899E
:105F20004D895E896B857C858D859E850F94DB56BA
:105F30006B017C01A3019201C301B2010F94505087
:105F40002B013C01A7019601C701B6010F945050E7
:105F50009B01AC01C301B2010F94DC560F948A5926
:105F60006B017C012B8D3C8D4D8D5E8DCA01B9017D
:105F70000F9450502B013C012F8D38A149A15AA1FB
:105F8000CA01B9010F9450509B01AC01C301B20189
:105F90000F94DC569B01AC01C501B4010F943C5930
:105FA0001816B4F520E030E0A901C701B6010F943E
:105FB0003C5987FF2AC0C701B601905820E030E065
:105FC00040EA50E40F943C59181614F5A1016D8174
:105FD0007E81C8010E94EA2EA2960FB6F894DEBF19
:105FE0000FBECDBFDF91CF911F910F91FF90EF902A
:105FF000DF90CF90BF90AF909F908F907F906F90E9
:106000005F904F903F902F900895C701B601D6CF73
:1060100020E030E040E050E4C501B4010F943C5969
:10602000181624F4B101C8010E947D2E19821A822B
:106030001B821C82BE016F5F7F4FC1010E94742EC4
:106040002DEC3CEC4CEC5CE3C701B6010F945050D6
:106050009B01AC01F80160817181828193810F9471
:10606000505069837A838B839C83C8010F94B42B2F
:10607000BE016F5F7F4F8D819E810E94742EACCFD9
:106080004F925F926F927F929F92AF92BF92CF9208
:10609000DF92EF92FF920F931F93CF93DF93CDB7D1
:1060A000DEB768970FB6F894DEBF0FBECDBFFB0119
:1060B0009080342F390D353008F026C1E180022F51
:1060C0000E0D053008F020C1EE2DF0E0EE54FB4F30
:1060D0004080512C712C612C092C04C0769467945B
:1060E000579447940A94D2F740FE0EC110E0F8018D
:1060F000EE54FB4F4080512C712C612CC32ED12CBF
:1061000004C076946794579447943A95D2F740FE2A
:10611000FBC0F22E642F5C01660F770B072E000C7C
:10612000880B990B0F94F14F2B013C01892D94E0C2
:106130008902F0011124E354FA4EA3019201608117
:106140007181828193810F94DC566D877E878F8762
:10615000988BF601EE0FFF1FEE0FFF1FE354FA4E70
:10616000A301920160817181828193810F94DB563A
:1061700069837A838B839C836F2D660F770B072E41
:10618000000C880B990B0F94F14F2B013C018E2DC5
:1061900094E08902F0011124E755FA4EA30192011F
:1061A00060817181828193810F94DC56698B7A8B37
:1061B0008B8B9C8B000F111F000F111FF801E755EF
:1061C000FA4EA301920160817181828193810F94C3
:1061D000DB566D837E838F839887F501808591855B
:1061E000A285B38589879A87AB87BC878D8B9E8B69
:1061F000AF8BB88F45E351E061E070E0CE0141968E
:106200000E9406D645E351E061E070E0CE010596BC
:106210000E9406D64AE351E061E070E0CE010D969F
:106220000E9406D64AE351E061E070E0CE0101969B
:106230000E9406D6C988DA88EB88FC8827E137EB0C
:1062400041ED58EBC701B6010F943C5987FD5CC086
:1062500023E030E04BE953E4C701B6010F94EA4F65
:1062600018160CF451C0CD84DE84EF84F88827E141
:1062700037EB41ED58EBC701B6010F943C5987FD50
:1062800043C023E030E84DE953E4C701B6010F9461
:10629000EA4F1816CCF1CD80DE80EF80F88427E13C
:1062A00037EB41ED58EBC701B6010F943C5987FD20
:1062B0002BC023E030E04BE953E4C701B6010F9453
:1062C000EA4F18160CF1C980DA80EB80FC8027E1D8
:1062D00037EB41ED58EBC701B6010F943C5987FDF0
:1062E00013C023E030E84DE953E4C701B6010F9431
:1062F000EA4F18164CF0AE014F5F5F4FBE01635F6F
:106300007F4FC5010E94EA2E68960FB6F894DEBF53
:106310000FBECDBFDF91CF911F910F91FF90EF90F6
:10632000DF90CF90BF90AF909F907F906F905F90E5
:106330004F9008958C38910514F08CE890E090937C
:106340006F0880936E080C944BC70E94972797FDA7
:106350000CC00E9497276F3F71058105910509F0D8
:1063600034F40E949727862F089580E008958FEFD8
:1063700008958091BB049091BC04892B41F00E9448
:10638000A53191E0811101C090E0892F089591E03D
:10639000FCCF0E949727CB0108950F931F93CF93B3
:1063A0008091BB049091BC040097E9F0FC018F013F
:1063B000C1912C2F2F7D81F0C53411F0C536B9F76E
:1063C000F801108270E060E00F94794BF801C0830F
:1063D000CF911F910F91089570E060E0CF911F91D0
:1063E0000F910D94794B60E070E0CB01F1CF2FEB72
:1063F000280F2A3108F047C0E22FF0E08091EC042A
:106400009091ED04A091EE04B091EF0404C0B69514
:10641000A795979587952A95D2F780FD02C0817040
:106420000895EE52FB4FE081EE2341F180914F0839
:1064300090915008E80FF92FF11D808190ED980F91
:106440009A3030F08E3251F4818180538A3098F442
:10645000F093BC04E093BB0481E008958D3211F009
:106460008B3249F4818190ED980F9A3088F38E3207
:1064700011F48281EACFF0E0E0E0EACF1092BC04B0
:106480001092BB04E9CF80E008950E94F731882381
:1064900041F081E02091BB043091BC04232B09F42E
:1064A00080E00895CF93DF93EB010E94453288236B
:1064B00019F00E949727EB01CE01DF91CF9108954B
:1064C000CF92DF92EF92FF926A017B010E944532E8
:1064D000882331F0FF90EF90DF90CF900C94CD3176
:1064E000C701B601FF90EF90DF90CF9008954F92D3
:1064F0005F926F927F928F929F92AF92BF92CF9254
:10650000DF92EF92FF921F93CF93DF9300D01F9201
:10651000CDB7DEB719821A821B821C82CE0101968A
:106520004C0186EEC82E8FE0D82E91E3E92E98E03C
:10653000F92E2CE4A22E29E0B22E10E088E5810F7E
:106540000E944532F40181934F01882341F00E945B
:10655000CD312B013C0180919B0F882359F0F6012E
:1065600080819181A281B381F70180839183A2838D
:10657000B38314C0812F0E940A22882309F4D0C05B
:10658000F6012081318142815381C301B2010F9410
:10659000DC56F70160837183828393831F5FF4E08D
:1065A000CF0ED11C84E0E80EF11C94E0A90EB11CC2
:1065B000133021F685E40E9445328C83882309F448
:1065C000B9C00E94CD316B017C0183E00E940A2298
:1065D000882371F02091F20F3091F30F4091F40F66
:1065E0005091F50FC701B6010F94DC566B017C0189
:1065F000C0923D08D0923E08E0923F08F0924008D9
:106600008091CB05882359F18091DC1582FF27C04A
:106610008C81882321F18981811103C08A8188239B
:10662000F1F02DEC3CEC4CE45DE36091A30870913B
:10663000A4088091A5089091A6080F94DC569B01B0
:10664000AC016091EE0F7091EF0F8091F00F90917F
:10665000F10F0F943C59181614F40F946C3C40E061
:1066600050E0BA0186E40E94603220E030E0A901E7
:106670000F943C59181684F40E94CD3120E030E08C
:1066800040E752E40F94D6576093740270937502FA
:10669000809376029093770280919C0F83FD2CC0AB
:1066A00080919B0F811128C08091AB07882321F135
:1066B0002091F20F3091F30F4091F40F5091F50FAC
:1066C00060913D0870913E0880913F08909140088C
:1066D0000F94DB562091B8073091B9074091BA0763
:1066E0005091BB070F94DC566093B8077093B907BD
:1066F0008093BA079093BB070F900F900F900F9065
:10670000DF91CF911F91FF90EF90DF90CF90BF90DE
:10671000AF909F908F907F906F905F904F90089573
:10672000F5012081318142815381C301B2010F946F
:10673000DB562FCF8091F20F9091F30FA091F40FC1
:10674000B091F50F80933D0890933E08A0933F08C9
:10675000B093400855CFCF93DF93EB010E944532B1
:10676000882321F0DF91CF910C94C931CE01DF91C4
:10677000CF910895CF93DF93C82FD62F0E94453233
:10678000882321F0DF91CF910C94B9318C2F0E9496
:10679000F731811101C08D2FDF91CF910895EAE982
:1067A000F8E082EBDF011D928A95E9F70895809168
:1067B000CB05811104C00E94CF330D94103F80910E
:1067C000DC1582FD0D946C3C089580919A08882315
:1067D00061F090914B09891308C08091DC1583FF0B
:1067E00004C088ED98E00D941B3F80E00895FC0103
:1067F000238121110C94DBD20895CF92DF92EF9286
:10680000FF920F931F93CF9390912402913009F43C
:1068100061C0662351F010929E0410929A04109267
:106820009B0410929C0410929D04C82F0F946E320A
:10683000C0909A04D0909B04E0909C04F0909D043A
:106840009B01AC012C193D094E095F0969017A01D0
:10685000F7FC40C020919E04C7FD15C04C2F0C2EA4
:10686000000C550B4C5F5F4FE22F022E000CFF0B0C
:106870004E175F077CF144EFC42EDD24D394E12C46
:10688000F12C2C1734F438EEC32E33E0D32EE12C48
:10689000F12CC60ED71EE81EF91EC0929A04D092A3
:1068A0009B04E0929C04F0929D04022F017010E082
:1068B00084E2809FB001819F700D701B112460598C
:1068C0007C4F82E390E00E94747E80919E048F5FF3
:1068D00080939E04CF911F910F91FF90EF90DF90D6
:1068E000CF9008950F931F9301E010E020E030E077
:1068F000082E04C0000F111F221F331F0A94D2F765
:1069000040910005509101056091020570910305C9
:10691000402B512B622B732B4093000550930105A4
:10692000609302057093030590912302891303C0BD
:1069300081E080939B0F1F910F9108951092300674
:10694000109231061092320610923306ECECF5E00C
:1069500084E6DF011D928A95E9F708959091E50F8D
:106960009817B1F00E94EADC8091E50F882341F08E
:1069700086EE9FE00E940DDD1092E50F0C94D8F09A
:1069800081E08093E50F86EE9FE00E943FDCF6CF2A
:1069900008954F925F926F927F928F929F92AF92E3
:1069A000BF92CF92DF92EF92FF921F93CF93DF932C
:1069B000EC01162F2091640830916508409166081B
:1069C00050916708688179818A819B810F94EA4F91
:1069D000882309F4AEC0B090E50F80E00E94AE3489
:1069E000C880D980EA80FB8020E030E0A901C7019F
:1069F000B6010F943C5918161CF0C12CD12C76010D
:106A0000C0926408D0926508E0926608F092670828
:106A10002DEB37E346E855EBC701B6010F943C591F
:106A200087FD0BC02DEB37E346E855E3C701B60100
:106A30000F94EA4F18160CF078C0A701960160E099
:106A400070E080E89FE30F94D6576093AF05709392
:106A5000B0058093B1059093B20580EF9FEFA9E751
:106A6000B4EC8093B3059093B405A093B505B093AF
:106A7000B605BB2009F45DC04090E60F5090E70FCB
:106A80006090E80F7090E90F8090EA0F9090EB0F04
:106A9000A090EC0FB090ED0FC090EE0FD090EF0FE4
:106AA000E090F00FF090F10F81E00E94AE341123DE
:106AB00009F43FC02091E60F3091E70F4091E80FB5
:106AC0005091E90FC301B2010F94EA4F81111CC02C
:106AD0002091EA0F3091EB0F4091EC0F5091ED0FA8
:106AE000C501B4010F94EA4F81110EC02091EE0F41
:106AF0003091EF0F4091F00F5091F10FC701B601A7
:106B00000F94EA4F8823A9F0DF91CF911F91FF9056
:106B1000EF90DF90CF90BF90AF909F908F907F903D
:106B20006F905F904F900C9480F960E070E0CB0123
:106B30008CCFDF91CF911F91FF90EF90DF90CF909E
:106B4000BF90AF909F908F907F906F905F904F908D
:106B50000895EF92FF920F931F93CF93DF930CEC66
:106B600015E0C5E07801D5E0F7016191719181915F
:106B700091917F0120E030E0A9010F94EA4F81114B
:106B80000EC0D15089F7C1500C5E1F4FC111EACF22
:106B9000DF91CF911F910F91FF90EF90089581E0C9
:106BA000F7CFEFE6F0E080818260808308958091E6
:106BB000450890914608892B79F480914508909179
:106BC0004608892B49F4209145083091460881E018
:106BD000232B19F480E0089581E00895CF92DF928D
:106BE000EF92FF926B017C0183E3C816D104E104AC
:106BF000F10470F082E3C81AD108E108F10862E3F9
:106C000070E080E090E00F943B320E94DAF0ECCF2D
:106C1000C701B6010F943B32FF90EF90DF90CF9009
:106C20000C94DAF080912B0781110AC080916208E0
:106C3000813041F08091DC1582FB882780F908952E
:106C400080E0089581E008955F9A8091BF078E7F6C
:106C50008093BF078A9A8091BF078D7F8093BF077B
:106C60008091080180958170809306018091BF0713
:106C70008B7F8093BF070C9437229091DC1593FB98
:106C8000882780F993FF06C081E090914217911107
:106C900001C080E0089580912B07811110C0809180
:106CA0006208823061F00E943D36882349F080916D
:106CB000DC1582FB882780F991E08927089581E01F
:106CC00008950E944B3681110DC01092000510925C
:106CD00001051092020510920305109204058FEF32
:106CE0000E94D8250C94CFFCE6E8F9E010821182CE
:106CF000089581E008958F929F92AF92BF92CF92B4
:106D0000DF92EF92FF920F93CF93DF931F92CDB755
:106D1000DEB75C017B0149016B01C40ED51EF50194
:106D2000808191810F9408568983002311F0F70127
:106D30008083BE016F5F7F4FC4010F940F24F50164
:106D400080819181019691838083FFEFEF1AFF0A82
:106D5000EC14FD0421F780E00F90DF91CF910F91AB
:106D6000FF90EF90DF90CF90BF90AF909F908F906B
:106D700008959091C00095FFFCCF8093C6000895C0
:106D8000CF93DF93EC018991882319F00E94B936E3
:106D9000FACF8DE00E94B9368AE0DF91CF910C9452
:106DA000B936CF92DF92EF92FF92CF936B017C01C5
:106DB000C42F4A3069F4F7FE0BC0F094E094D094ED
:106DC000C094C11CD11CE11CF11C8DE20E94B9369B
:106DD0004C2FC701B601CF91FF90EF90DF90CF907D
:106DE0000D94CE3BCF93DF93EC01FE01849121966D
:106DF000882319F00E94B936F8CFDF91CF9108951A
:106E00000F931F93CF938C01C62F8DE592E10E94C3
:106E1000F236C8010E94F2368AE30E94B93680E356
:106E20008C0F0E94B9368AE0CF911F910F910C947C
:106E3000B93680EE93E10E94F23660E080ED93E196
:106E40000E94003760E08BEB93E10E94003761E025
:106E500084EB93E10E94003761E089EA93E10E94AC
:106E6000003761E089E993E10E94003760E080E942
:106E700093E10E94003761E086E893E10E940037C9
:106E800060E08CE793E10E94003761E085E793E1E1
:106E90000E94003760E08DE693E10E94003761E0D8
:106EA0008FE593E10E94003761E081E593E10E9464
:106EB000003760E082E493E10E94003760E084E301
:106EC00093E10E94003760E08EE193E10E94003779
:106ED00061E08DE093E10E94003761E08EEF92E186
:106EE0000E94003761E087EF92E10E94003760E086
:106EF00080EF92E10E94003761E087EE92E10E940C
:106F0000003761E082ED92E10E94003761E084EC9D
:106F100092E10E94003761E081EB92E10E9400372C
:106F200060E084EA92E10E94003761E08FE992E13B
:106F30000E94003761E082E992E10E94003760E040
:106F40008EE792E10E94003760E08BE692E10E94BA
:106F5000003760E08EED95E10E940722682F617096
:106F600082E692E10C9400370E94B93685E29DE0FA
:106F70000C94F2360F931F93CF938C01C62F8CE99C
:106F800099E00E94F236C8010E94F236CC2331F01B
:106F90008AE0CF911F910F910C94B936CF911F9138
:106FA0000F9108950F931F93CF938C01C62F60E02C
:106FB0008CEA99E00E94BA37C8010E94F236CC23CD
:106FC00031F08AE0CF911F910F910C94B936CF9197
:106FD0001F910F91089561E084EB99E00C94D237F2
:106FE000EF92FF920F931F93CF937C018B01C42FDD
:106FF00060E08CEA99E00E94BA37C7010E94F2363D
:1070000080E20E94B936C8010E94F236CC2319F002
:107010008C2F0E94B9368AE0CF911F910F91FF907B
:10702000EF900C94B936DF92EF92FF920F931F937B
:10703000CF93DF93D82E7B018A01E9010E94EB37C1
:10704000D092490840E0B70184E290E40E94F03712
:107050000115110531F040E0B8018DE190E40E9486
:10706000F037209731F040E0BE018DE190E40E94BE
:10707000F03761E088E190E4DF91CF911F910F91AB
:10708000FF90EF90DF900C94D23761E086EA99E0B0
:107090000C94BA37AF92BF92CF92DF92EF92FF92E9
:1070A0000F931F93CF93DF9381E799E00E94F2360D
:1070B00060913006709131068091320690913306CE
:1070C00045E00F944F078EE599E00E94F236C0E04C
:1070D000D9E0D15021F080E20E94B936FACF8C2F4E
:1070E0000F94353CCF5FC53099F78AE00E94B936DE
:1070F0000CEC15E0C0E080E20E94B9368C2F0F94B2
:10710000353C5801D5E080E20E94B936F501C080D7
:10711000D180E280F380A7019601C701B6010F94E8
:10712000CE5981112CC020E030E0A901C701B60181
:107130000F943C5987FD03C08BE20E94B93645E0AD
:10714000C701B6010F944F07D15084E1A80EB11CBE
:10715000D111D9CF8AE00E94B936CF5F0C5F1F4FA3
:10716000C53049F68AE0DF91CF911F910F91FF90D2
:10717000EF90DF90CF90BF90AF900C94B936F12C88
:1071800080E20E94B936F3948DE3F8E0FF12F9CF64
:10719000DBCF811107C083E69EE00E94F2368AE0D1
:1071A0000C94B93687E69EE0F8CFCF93DF93EB01DE
:1071B0000E94F236CE01DF91CF910D943C3CCF93EB
:1071C000C62F0E94F2368C2FCF910D94353CCF9272
:1071D000DF92EF92FF926A017B010E94F23642E059
:1071E000C701B601FF90EF90DF90CF900D944F074D
:1071F000CF92DF92EF92FF926A017B010E94F236FA
:107200004AE0C701B601FF90EF90DF90CF900C9459
:10721000D1362F923F924F925F926F927F928F92D0
:107220009F92AF92BF92CF92DF92EF92FF920F9315
:107230001F93CF93DF93CDB7DEB7C654D1090FB6F6
:10724000F894DEBF0FBECDBF70E060E085E40E9421
:10725000AB33182F8F3F09F483C08823E9F08BE903
:1072600096E1CA5BDF4F0FB6F894DEBF0FBECDBF0D
:10727000DF91CF911F910F91FF90EF90DF90CF9012
:10728000BF90AF909F908F907F906F905F904F9046
:107290003F902F900C94F23624EB30E03A83298310
:1072A00083E50E944532882321F00E94C9319A83E8
:1072B000898365E070E083E40E94AB338AA760E0D5
:1072C00085E50E94BA3325968FAF259760E08EE85A
:1072D00096E10E9489B3A981BA81BD01BB0F880BD9
:1072E000990B0F94F14F6D837E838F8327969FAF09
:1072F00027970F946E32688B798B8A8B9B8B1F3FFD
:1073000009F045C420E030E04CE053E46D817E811B
:107310008F8127969FAD27970F943C5918160CF034
:10732000AAC183E696E10E94F236CA5BDF4F0FB630
:10733000F894DEBF0FBECDBFDF91CF911F910F91AB
:10734000FF90EF90DF90CF90BF90AF909F908F9085
:107350007F906F905F904F903F902F900D940B40D7
:1073600046E450E05A8349839BCF1FAEAFC12496B9
:10737000EEADFFAD2497808383C2FBEE4F2E512CE0
:10738000612C712C04C384E190E0A0E0B0E08C8B10
:107390009D8BAE8BBF8BE4E14E2E512C612C712C5A
:1073A00004C34C8A5D8A6E8A7F8AFFC22496EEAD42
:1073B000FFAD24978083D4C389819A81AB81BC813E
:1073C00029A93AA94BA95CA9821B930BA40BB50B65
:1073D000B7FD59C08FAD0F94F3078AE00E94B9360C
:1073E00089819A81AB81BC818053984FAF4FBF4F49
:1073F00089AB9AABABABBCAB9DA9911177C02EA961
:107400003FA948AD59ADB101802F26969FAD269773
:107410000F943C5918160CF053C020E030E040E0C7
:1074200050E4B101802F26969FAD26970F94DC562D
:107430006EAB7FAB88AF99AF2CA53DA54EA55FA5E0
:1074400089819A81AB81BC81280F391F4A1F5B1F3C
:107450002AAF3BAF4CAF5DAF20E030E040EC50E4F2
:107460006D817E818F8127969FAD27970F94DB5684
:107470009101402F26965FAD26970F94EA4F881F03
:107480008827881F8DAB88899989AA89BB89C816E6
:10749000D906EA06FB0610F4D701C60129813A8114
:1074A0004B815C81281B390B4A0B5B0BDA01C9014C
:1074B00081389F44A241B105A8F18FEA95E10EC23F
:1074C00089819A81AB81BC812AAD3BAD4CAD5DAD6C
:1074D000821B930BA40BB50B41E156E360E276E30C
:1074E000B7FDD1CF812F0E9448D6CDCF20E030E02C
:1074F00040EF51E46D817E818F8127969FAD279764
:107500000F94DB569B01AC01B101802F26969FADF5
:1075100026970F94EA4F87FFB6CF4DEB56E36DECFD
:1075200076E3E0CF4AA55BA5888D998D481759076A
:107530000CF09EC003970CF49BC082E595E10E947D
:10754000F2361F3F09F076C0A2E4B5E1BA83A98301
:1075500081E395E10E94F23689819A810E94F23698
:10756000488559856A857B858EE495E10E94E738D8
:107570008AE00E94B93681E395E10E94F236898162
:107580009A810E94F23649A15AA16BA17CA18AE49A
:1075900095E10E94E7388AE00E94B93681E395E1DF
:1075A0000E94F23689819A810E94F236B501A401C7
:1075B00086E495E10E94E7388AE00E94B936259674
:1075C000FFAD2597FF2391F12CEA35EC47E25EE30E
:1075D00069A17AA18BA19CA10F9450506B017C01F1
:1075E0002CEA35EC47E25EE3C501B4010F94D657AF
:1075F000288539854A855B851F3F09F520937108E9
:10760000309372084093730850937408C0927508C1
:10761000D0927608E0927708F09278086093790823
:1076200070937A0880937B0890937C0881E0809324
:107630005D027BCEE2E6FFE3FA83E98389CF209304
:107640002115309322154093231550932415C09291
:107650002515D0922615E0922715F09228156093F3
:10766000291570932A1580932B1590932C15DECF36
:107670000E9495B780C08FE496E10E94F2360E9486
:107680003BD58FE78093700824EB30E0A8EEB3E0A1
:107690000F9482566CA77DA78EA79FA7288939894A
:1076A0004A895B89260F371F481F591F2AAF3BAFF6
:1076B0004CAF5DAF10925D0281E080936C0232E0CE
:1076C000310F3EAF323008F450CE1FAFC888D98892
:1076D000EA88FB88C9AADAAAEBAAFCAA812C912C19
:1076E000540189A29AA2ABA2BCA288869986AA86D6
:1076F000BB868FE790E0A0E0B0E08C8B9D8BAE8BDB
:10770000BF8B1C8690E49A8FACE1AB8FB6E4BC8F44
:107710001D8E1E8E1F8E18A23FE7432E512C612C0A
:10772000712C1DAA8EAA9FAAA8AEB9AE1EA21FA236
:1077300018A619A6E1E0EDA3198E188E212C312C84
:1077400000E026961FAE2697F5E11F02C001112426
:107750009C01285E3A4E22963FAF2EAF2297285FBB
:107760003F4F24963FAF2EAF24974AA5042E000C1E
:10777000550B5BA74AA780916C02882309F4B0C01F
:107780000F946E3269837A838B839C8350914D066C
:1077900058AB552309F48BC00E94EED560916C085C
:1077A00070916D081F3F39F02296AEADBFAD2297A4
:1077B00014966D917C91072E000C880B990B0F94F9
:1077C000F14F1B01082F26969FAF26972D8D3E8DDA
:1077D0004F8D58A126969FAD26970F943C591816A9
:1077E0003CF42D8E3E8E0F8F2696BFAD2697B8A304
:1077F0002C853A8D4B8D5C8DB101802F26969FADE7
:1078000026970F94EA4F87FF07C02C863A8E0B8F7E
:107810002696EFAD2697EC8FFDA19101402F26967D
:107820005FAD26976D817E818F8127969FAD2797CB
:10783000FF2309F45AC00F94EA4F87FF38C04981EB
:107840005A816B817C814C195D096E097F09DB01CE
:10785000CA0188589341A109B109B7FD28C08C8994
:107860009D89AE89BF8984199509A609B709B5957F
:10787000A795979587951F3F09F079CD809370085C
:107880004EA35FA368A779A7FD81FD8F2E812E8F60
:107890003F813F8F27964FAD279748A389819A81D3
:1078A000AB81BC81888B998BAA8BBB8B1DA220E0FE
:1078B00030E040EF51E46D817E818F8127969FAD4E
:1078C00027970F94DC569101402F26965FAD26979F
:1078D0000F94EA4F87FF70CD8DEC95E10E94F23650
:1078E00010926C020E943BD5A1CE0F943C59181601
:1078F000F4F689819A81AB81BC81288939894A89CA
:107900005B89821B930BA40BB50BAC01BD014858DE
:1079100053416109710977FDCACF488D598D452BB7
:1079200009F40DC1CEA0DFA0E8A4F9A4C80ED91EA9
:10793000EA1EFB1E2EA13FA148A559A5281B390B05
:107940004A0B5B0BC301B2010F941E56A7019601AF
:107950000F9450564C885D886E887F88420E531E67
:10796000641E751E54E145165104610471040CF443
:107970000ACD8CEE48165104610471040CF0FDCC64
:1079800090E849165104610471040CF40ACD4C8A44
:107990005D8A6E8A7F8A2EEF30E040E050E0241945
:1079A00035094609570929013A014C895D896E89D3
:1079B0007F8987E496E10E94F838B301A20182E44E
:1079C00096E10E94F8384C855A8D6B8D7C8D8BE347
:1079D00096E10E94E7384D8D5E8D6F8D78A184E32E
:1079E00096E10E94E738A88DB98D13970CF4A7C0D3
:1079F000C301B2010F94F14F20E030E040E850E4C1
:107A00000F9450504B015C012C853A8D4B8D5C8D51
:107A10006D8D7E8D8F8D98A10F94DB562BED3FE001
:107A200049E450E40F94505020E030E040E05FE340
:107A30000F9450509B01AC01C501B4010F94D6576F
:107A40006C877D878E879F87C701B6010F94F14FA2
:107A50002FE632E143E85AE30F9450506B017C016A
:107A60001E3F59F02AE939E949E15FE3812C912C65
:107A7000A12C6EE3B62E1F3F59F42DEC3CEC4CE4E8
:107A80005EE37BEA872E7AEA972EA92C7EE3B72E57
:107A90006C857D858E859F850F945050688779878A
:107AA0008A879B879B01AC010F94DC56A701960146
:107AB0000F94D65769A37AA38BA39CA328853985F5
:107AC0004A855B85C701B6010F945050A50194010A
:107AD0000F9450504B015C014C855D856E857F8510
:107AE0008EE296E10E94E738B701A60188E296E1AE
:107AF0000E94E7388AE00E94B936BEAD89E196E17E
:107B0000B23010F08AE096E10E94F236488559853D
:107B10006A857B8584E096E10E94E73849A15AA1F5
:107B20006BA17CA18EEF95E10E94E738B501A4011D
:107B300088EF95E10E94E7388AE00E94B9368C8987
:107B40009D89AE89BF89840D951DA61DB71DB5956C
:107B5000A795979587951F3F09F028CC80937008CB
:107B6000288D398D2F5F3F4F398F288F3D813C877E
:107B70004E814A8F5F815B8F27968FAD27978C8FC1
:107B8000C980DA80EB80FC8098A99DA390CEE12E7D
:107B9000012E000CFF08F70183E0EE0FFF1F8A950E
:107BA000E1F7EC59FD4F668177816F507109072E1F
:107BB000000C880B990B0F94F14F9B01AC016D8168
:107BC0007E818F8127969FAD27970F943C59181679
:107BD0000CF4A7CB8FE496E10E94F2360E943BD5CD
:107BE00085E18E9DF0018F9DF00D1124E85EFA4E27
:107BF0008FE7808722E330E049CDCF93DF93EB011D
:107C00000E94F236CE01DF91CF910D94C6252F92BE
:107C10003F924F925F926F927F928F929F92AF921C
:107C2000BF92CF92DF92EF92FF920F931F93CF9369
:107C3000DF93CDB7DEB7C058D1090FB6F894DEBFD9
:107C40000FBECDBF80EB9CE00E94F2360F942D401A
:107C500081118FC084E50E944532882329F00E945B
:107C6000C93181110E94F1D480E090E0A0E8BFE327
:107C700089839A83AB83BC838D839E83AF83B887CC
:107C80008DEC9CECACE4BEE389879A87AB87BC871C
:107C900080E090E0A0E2B1E48D879E87AF87B88B4B
:107CA0008CE390E09A8B898B8DEC90E09C8B8B8B96
:107CB0008DEC9CECACECBEE38D8B9E8BAF8BB88FC8
:107CC00080E090E0A0EEBFE3898F9A8FAB8FBC8FEE
:107CD0001BA61CA64AE959E969E97EE38FE40E94E4
:107CE00060326D8F7E8F8F8F98A360E083E40E9457
:107CF000BA3389A360E08BE40E94BA338AA389E493
:107D00000E94453210E0F12CE12C8823C1F00E9442
:107D1000A53190E01816190614F481E090E011E006
:107D2000180F212F2150330BC90126E0289FF001A5
:107D3000299FF00D1124EB5FF74FE280F38082E47E
:107D40000E944532882319F00E94C9317C01E11458
:107D5000F10459F1C70188978536910520F16CE847
:107D600070E082E89CE00E94FD3D8DE79CE00E946F
:107D7000F236C058DF4F0FB6F894DEBF0FBECDBF4E
:107D8000DF91CF911F910F91FF90EF90DF90CF90F7
:107D9000BF90AF909F908F907F906F905F904F902B
:107DA0003F902F900895FA8AE98A8CE40E94453228
:107DB0008823E1F00E94CD316B017C01C986DA860F
:107DC000EB86FC8620E030E0A9010F943C5987FD4A
:107DD0000AC020E030E040E050E4C701B6010F9453
:107DE000EA4F18161CF485E59CE0C1CF81E50E949E
:107DF000F731882331F18091BB049091BC04892B29
:107E0000E9F00E94CD316B017C01CD82DE82EF82F0
:107E1000F8862DEC3CEC4CE45DE30F943C5987FD77
:107E20000AC020E030E040E751E4C701B6010F94FA
:107E3000EA4F181634F484E29CE099CF89EF9BE076
:107E400096CF83E50E9445328823E9F00E94CD3128
:107E50006B017C01CD8ADE8AEF8AF88E2DEC3CEC3A
:107E60004CEC5DE30F943C5987FD0AC020E030E004
:107E700040E050E4C701B6010F94EA4F18161CF415
:107E800082ED9BE074CF80E50E94F731882341F0BA
:107E90008091BB049091BC04892B29F58FEF8BA7AF
:107EA00086E40E944532882309F43DC00E94CD310A
:107EB0006B017C01C98EDA8EEB8EFC8E20E030E007
:107EC00040E85FE30F943C5987FD0AC020E030E0B2
:107ED00040E850E4C701B6010F94EA4F18161CF5AC
:107EE00081E89BE044CF8BA58F5F8BA70E94CD31AB
:107EF0006B017C01CD86DE86EF86F88A20E030E0DB
:107F0000A9010F943C5987FD0BC020E030E048ECFC
:107F100051E4C701B6010F94EA4F18160CF0C0CF18
:107F20008AEA9BE024CFC98CDA8CEB8CFC8C8D88A0
:107F30009E88AF88B88CA7019601C701B6010F943F
:107F400050509B01AC0160E070E084E490E40F9439
:107F5000D65729813A814B815C810F9450502B0177
:107F60003C01A5019401C501B4010F945050A70133
:107F700096010F9450502CEE31E548EB5DE30F94E1
:107F8000D6579B01AC01C301B2010F9450506983D5
:107F90007A838B839C83112309F1412F4150550B28
:107FA00026E0249FF001259FF00D1124EB5FF74F91
:107FB0000081118188E40E944532882319F00E94D3
:107FC000C9318C010115110571F0C801855A91095B
:107FD0008F30914030F083E59BE0C9CE10E000E0A7
:107FE000E9CF1C8B0B8B85E50E94F7318823C9F004
:107FF0000F946E32611571058105910511F00F9492
:10800000704B8091BB049091BC04892BC9F00E94F5
:10801000CD316093B7047093B8048093B904909302
:10802000BA046AE170E082E50E94AB33E5969FAF47
:108030008EAFE5971816190644F08FE19BE097CEB6
:1080400060E070E088E492E4E4CF89E50E94453284
:10805000882309F40AC10E94CD3120915009309142
:10806000510940915209509153090F94DB564B012D
:108070005C0188E50E944532882309F4FFC00E9414
:10808000CD3120914C0930914D0940914E095091CC
:108090004F090F94DB566B017C01CBA2DCA2EDA251
:1080A000FEA28FA298A6A9A6BAA627E137EB41EDBA
:1080B00058EBC501B4010F943C5987FDE8C023E09B
:1080C00030E04BE953E4C501B4010F94EA4F1816B0
:1080D0000CF4DDC027E137EB41ED58EBC701B601E9
:1080E0000F943C5987FDD3C023E030E84DE953E4B9
:1080F000C701B6010F94EA4F18160CF4C8C084E407
:108100000E94F73111E081270E94AE3480E090E0B8
:10811000A0EAB0E48DA79EA7AFA7B8ABCE018D961D
:108120000F94592B80918108EC968FAFEC971092A9
:1081300081080E94FCC482EA9AE00E94F236898992
:108140009A894A970CF0A6C063E68FE79AE00E94EE
:1081500089B30F94A7328B899C890E946CDC41E023
:1081600061E080E00F94EB09882309F4A6C00F9426
:108170000B400F94A7321092F20F1092F30F10924F
:10818000F40F1092F50F82EF9FE00E9420ED1BA5E7
:10819000112309F4F5C020E030E040E751E460919C
:1081A000CD0F7091CE0F8091CF0F9091D00F0F9483
:1081B000D65721966CAF7DAF8EAF9FAF21971F3FF3
:1081C00009F0F9C481E08093FD0463E687ED9AE04D
:1081D0000E9489B368E873E182E090E00E94747EB7
:1081E00080E1E6EEFFE0A1E3B8E001900D928A9510
:1081F000E1F7CE0101960F94B42BC12CD12C76015E
:1082000080915C0982FDB1C068E873E182E090E092
:108210000E94747E20E030E040E85EE360913D081B
:1082200070913E0880913F08909140080F94DC5671
:1082300060933D0870933E0880933F0890934008F8
:1082400020E030E040E85EE3C701B6010F94DC5661
:108250006B017C0120E030E84BE354E40F943C597F
:1082600087FD73C01092FD0428C08090EA0F9090A3
:10827000EB0FA090EC0FB090ED0FFBCEC090E60F8F
:10828000D090E70FE090E80FF090E90F06CF85EF70
:108290009AE06DCD63E682E99AE00E9489B30F947B
:1082A000A7321093FD0489899A890E949A3161E06E
:1082B00081E00F946608811147CF6FEF89EE9AE055
:1082C0000E9489B38CA5811112C081E08CA78D8199
:1082D0009E81AF81B885B0588DA79EA7AFA7B8ABD8
:1082E000BE01635D7F4F81E398E00E94742E80E0C1
:1082F00090E0A0EAB0E48093390890933A08A09304
:108300003B08B0933C081DA61EA61FA618AABE01D6
:10831000635D7F4F81E398E00E94742EEC965FAD21
:10832000EC97509381080E94FCC41092FD048AA12E
:1083300081111FCD10926F0810926E080E944BC7DA
:1083400090E080E00E946CDC14CDCE01CD960E94BE
:10835000C8F780E1E6EEFFE0A1E3B8E001900D92FE
:108360008A95E1F70E94EADC4BCF0E9454BA63E69B
:108370008AEC9AE00E9489B30F94A7321092FD0410
:10838000E2EBF4E085E0DF011D928A95E9F780E1F8
:10839000E6EEFFE0A1E3B8E001900D928A95E1F7E7
:1083A00089859A85AB85BC858093390890933A0876
:1083B000A0933B08B0933C081DA61EA61FA618AAB2
:1083C000BE01635D7F4F81E398E00E94742EBE0181
:1083D000635E7F4F81E398E00E94742E81E080937A
:1083E000FD0489A1882309F43CC42091E60F309153
:1083F000E70F4091E80F5091E90FAC962CAF3DAFDD
:108400004EAF5FAFAC978091EA0F9091EB0FA091C8
:10841000EC0FB091ED0FE0968CAF9DAFAEAFBFAF5C
:10842000E097ADEBB5E1A196BFAFAEAFA197312C10
:10843000212CBFEF6C96BFAF6C97EFEFA496EFAF18
:10844000A497FFEFE396FFAFE3972FE4EA962FAFF1
:10845000EA9733ECEB963FAFEB9707E481E090E0CF
:10846000A0E0B0E0022C04C0880F991FAA1FBB1F18
:108470000A94D2F7C458DF4F88839983AA83BB83B9
:10848000CC57D040A2EBB4E0E296BFAFAEAFE297DC
:10849000E9EAF5E1A396FFAFEEAFA39710E0C0586D
:1084A000DF4F2882C058D040E296AEADBFADE29714
:1084B0008D91E296BFAFAEAFE29790E0B0E0A0E062
:1084C000C458DF4F288139814A815B81CC57D04025
:1084D00082239323A423B523892B8A2B8B2B09F08A
:1084E000E5C0A196AEADBFADA197CD90DD90ED906A
:1084F000FC90A396AEADBFADA3972D913D914D914C
:108500005C91A8962CAF3DAF4EAF5FAFA897A70187
:108510009601AC966CAD7DAD8EAD9FADAC970F94D2
:10852000DB562B013C01A8962CAD3DAD4EAD5FADA9
:10853000A897E0966CAD7DAD8EAD9FADE0970F94A2
:10854000DB564B015C01A3019201C301B2010F9400
:1085500050502B013C01A5019401C501B4010F94B9
:1085600050509B01AC01C301B2010F94DC560F9433
:108570008A594B015C01A70196016BA17CA18DA1D9
:108580009EA10F94DB566B017C01A8962CAD3DADEE
:108590004EAD5FADA8976FA178A589A59AA50F9458
:1085A000DB562B013C01A7019601C701B6010F94D0
:1085B00050506B017C01A3019201C301B2010F94E1
:1085C00050509B01AC01C701B6010F94DC560F94CB
:1085D0008A5920E030E040E751E40F94D657A501D6
:1085E00094010F94DC566B017C018090B70490904D
:1085F000B804A090B904B090BA0420E030E040E89C
:108600005FE3C501B4010F943C591816F4F4C50199
:10861000B4010F9448584B015C0160E070E0CB015D
:10862000181419041A041B0434F40F94214BA501E7
:1086300094010F9450560F94F14F9B01AC01B60179
:10864000C7010F94DC566B017C01E3962FADE397D5
:10865000EA963FADEA97EB964FADEB97502FB601F8
:10866000C7010F94EA4F87FF21C06C961FAF6C972C
:10867000C058DF4FB881C058D040A496BFAFA49770
:10868000E696CFAEE697E796DFAEE797E896EFAED1
:10869000E897E996FFAEE997E396CFAEE397EA96BF
:1086A000DFAEEA97EB96EFAEEB970F2D1F5FA39629
:1086B000EEADFFADA3973496A396FFAFEEAFA397B1
:1086C000153009F0F1CEFFEF2F1A3F0AA1962EAD1B
:1086D0003FADA1972C5F3F4FA1963FAF2EAFA19723
:1086E00035E02316310409F0B9CE6C964FAD6C9786
:1086F000E42FF0E0EE54FB4F208181E090E0A0E019
:10870000B0E0A4960FACA49704C0880F991FAA1FCD
:10871000BB1F0A94D2F7822B8083A4965FADA497E7
:1087200062965FAF629763964FAF6397E6968FADA1
:10873000E697E7969FADE797E896AFADE897E9969D
:10874000BFADE99767968CAF9DAFAEAFBFAF6797F0
:108750005F3F09F414C24F3F09F411C284E048029C
:10876000F0011124E755FA4E1081018132802380F7
:1087700027E137EB41ED58EB612F702F832D922DC0
:108780000F943C5987FDFFC123E030E04BE953E4EF
:10879000612F702F832D922D0F94EA4F18160CF431
:1087A000F2C1A4969FADA497A4E09A02F00111240F
:1087B000E354FA4EC080D180E280F38027E137EBAA
:1087C00041ED58EBB601C7010F943C5987FDDBC161
:1087D00023E030E84DE953E4B601C7010F94EA4FB6
:1087E00018160CF4D0C120E030E040EA50E4B601A5
:1087F000C7010F94DC56A0966FAFA097A2967FAFEB
:10880000A297A5968FAFA597A9969FAFA997CB01E1
:10881000A596AFADA597A996BFADA99721968CAFA8
:108820009DAFAEAFBFAF2197812F902FA32DB22D5B
:1088300025968CAF9DAFAEAFBFAF2597A496BFADC9
:10884000A497B11150C26C96EFAD6C97E11118C2AC
:1088500020E030E040EA50E4612F702F832D922D0C
:108860000F94DC56A4966FAFA497AD967FAFAD97EB
:10887000E1968FAFE197E3969FAFE3976C96FFADDC
:108880006C97FF2309F4F1C26C963FAD6C97A096EC
:10889000CFAEA097A296DFAEA297A596EFAEA59712
:1088A000A996FFAEA99734300CF014C222ED822EA7
:1088B00023E5922E2BE7A22E21E4B22E21964CAC7A
:1088C0005DAC6EAC7FAC219725962CAD3DAD4EAD29
:1088D0005FAD25976F962CAF3DAF4EAF5FAF6F97F3
:1088E000A3019201B601C7010F94DB562D966CAF20
:1088F0007DAF8EAF9FAF2D976F962CAD3DAD4EAD3A
:108900005FAD6F97612F702F832D922D0F94DB56E3
:1089100061966CAF7DAF8EAF9FAF6197A30192015F
:108920006091E60F7091E70F8091E80F9091E90F49
:108930000F94DB562B013C016F962CAD3DAD4EAD37
:108940005FAD6F976091EA0F7091EB0F8091EC0F24
:108950009091ED0F0F94DB566F966CAF7DAF8EAF9D
:108960009FAF6F97A0968FADA097A2969FADA2974D
:10897000A596AFADA597A996BFADA9978DA79EA7C0
:10898000AFA7B8ABA4968FADA497AD969FADAD97AA
:10899000E196AFADE197E396BFADE39789AB9AABB4
:1089A000ABABBCABC984DA84EB84FC84CDAADEAA71
:1089B000EFAAF8AE2DEC3CEC4CEC5CE3C501B40145
:1089C0000F94505029813A814B815C810F94505013
:1089D0002091F20F3091F30F4091F40F5091F50F69
:1089E0000F94DC5669AF7AAF8BAF9CAFA3019201B5
:1089F000C301B2010F9450502B013C016F962CAD76
:108A00003DAD4EAD5FAD6F97CA01B9010F945050A7
:108A10009B01AC01C301B2010F94DC5620E030E0B1
:108A200040E050E40F943C591816ACF420E030E0DC
:108A300040E05FE3C701B6010F94DC5629966CAFA6
:108A40007DAF8EAF9FAF2997BE01635C7F4FCE0194
:108A500001960E947D2E89859A85AB85BC852996D5
:108A60008CAF9DAFAEAFBFAF29976B961CAE1DAE5E
:108A70001EAE1FAE6B97BE01695A7F4FCE01CD96D9
:108A80000E94742ECE0101960F94B42BA090C50FB6
:108A9000B090C60FC090C70FD090C80FE090C10F24
:108AA000F090C20F0091C30F1091C40F9701A8015D
:108AB000B501C6010F943C59181614F075018601D2
:108AC0008090740290907502A0907602B090770228
:108AD0002DEC3CEC4CEC5DE3B701C8010F94505019
:108AE000609374027093750280937602909377027C
:108AF00040E0BE01675B7F4FCE018D960F946833D7
:108B000080E1E6EEFFE0A1E3B8E001900D928A95E6
:108B1000E1F78092740290927502A0927602B09270
:108B200077020E9486278111C8CB20E04FEFBE015B
:108B30006F5A7F4FCE0101960E94403020E041E005
:108B4000BE016F5A7F4FCE0101960E9440302FEF39
:108B500040E0BE016F5A7F4FCE0101960E94403027
:108B600021E040E0BE016F5A7F4FCE0101960E9486
:108B700040300E94EADC0E94862781119ECB8091C2
:108B8000F60F8093F70FE5964EAD5FADE597415038
:108B90005109E5965FAF4EAFE597452B09F48DCBB4
:108BA00062968FAD629787FD88CB63968FAD639792
:108BB00087FF17CC82CB63E687EB9AE00E9489B3EC
:108BC0000F94A73280E1E6EEFFE0A1E3B8E0019068
:108BD0000D928A95E1F72D853E854F8558896091E4
:108BE0003D0870913E0880913F08909140080F9495
:108BF000DC5660933D0870933E0880933F08909345
:108C00004008CE01CD960E94C8F72D853E854F8540
:108C1000588960913D0870913E0880913F0890917D
:108C200040080F94DB5660933D0870933E08809394
:108C30003F08909340088CA58111A2CB81E08CA7BE
:108C40008D819E81AF81B885B0588DA79EA7AFA7B3
:108C5000B8ABBE01635D7F4F81E398E00E94742E44
:108C60008FCB2BA13CA14DA15EA1AC962CAF3DAF0B
:108C70004EAF5FAFAC978FA198A5A9A5BAA5CBCBF6
:108C8000C601D70121968CAF9DAFAEAFBFAF219784
:108C900020E030E040EA50E4612F702F832D922DC8
:108CA0000F94DB5625966CAF7DAF8EAF9FAF2597A7
:108CB0006C962FAD6C9724300CF4CACDA4961FAFE0
:108CC000A497AD960FAFAD97E1963FAEE197E396CF
:108CD0002FAEE39792ED892E93E5992E9BEFA92E67
:108CE00090E4B92EEBCDA4964FADA49744300CF48C
:108CF0006EC06C965FAD6C975430BCF120E030E0F4
:108D000040EA50E4B601C7010F94DB5621966CAFE0
:108D10007DAF8EAF9FAF219720E030E040EA50E476
:108D2000612F702F832D922D0F94DB56A4966FAF79
:108D3000A497AD967FAFAD97E1968FAFE197E3969D
:108D40009FAFE3976C969FAD6C97A096CFAEA09720
:108D5000A296DFAEA297A596EFAEA597A996FFAE15
:108D6000A99794300CF0B6CFA1CDC601D7012196BA
:108D70008CAF9DAFAEAFBFAF219720E030E040EAAF
:108D800050E4612F702F832D922D0F94DC56259681
:108D90006CAF7DAF8EAF9FAF25976C968FAD6C9704
:108DA0008111BACF20E030E040EA50E4B601C701BB
:108DB0000F94DB56A0966FAFA097A2967FAFA297B5
:108DC000A5968FAFA597A9969FAFA99777CF6C96D9
:108DD000AFAD6C97A1112BC020E030E040E251E430
:108DE000A0966FADA097A2967FADA297A5968FADE6
:108DF000A597A9969FADA9970F94DB56A0966FAF44
:108E0000A097A2967FAFA297A5968FAFA597A99698
:108E10009FAFA997A4961FAFA497AD960FAFAD973C
:108E2000E1963FAEE197E3962FAEE3973FCD6C9688
:108E3000BFAD6C97B43034F120E030E040E251E453
:108E4000A0966FADA097A2967FADA297A5968FAD85
:108E5000A597A9969FADA9970F94DB5621966CAF65
:108E60007DAF8EAF9FAF2197D5CFA096CFAEA09705
:108E7000A296DFAEA297A596EFAEA597A996FFAEF4
:108E8000A99728CFA4961FAFA497AD960FAFAD9723
:108E9000E1963FAEE197E3962FAEE39782ED882E01
:108EA00083E5982E8BEFA82E81E4B82E07CD87E5B9
:108EB00099E00C94F236CF92DF92EF92FF920F93EB
:108EC0001F93CF93DF9388E50E94F731D82E89E472
:108ED0000E94F731C82E8823D1F10E94C931D82FC2
:108EE00089E50E94F731182F8AE40E94F731082F94
:108EF000882309F455C00E94C931C82F8AE50E9411
:108F0000F731E82EF12C811104C081E50E94F73180
:108F1000F82EC11001C000E0802F90E0D11001C0F8
:108F200010E0810F911D019721F4E11062C0F11052
:108F300060C00E94574783E49EE0DF91CF911F916C
:108F40000F91FF90EF90DF90CF900C94F236D110FC
:108F500002C0DFEFC5CF0E94CD3120914C09309186
:108F60004D0940914E0950914F090F94DB5620E076
:108F700030E040EF51E40F94DB5620E030E040EF6A
:108F800051E40F94DC5629E838E848E85CE30F9494
:108F900050500F944858D62F653008F4A1CFD9CF40
:108FA000111102C0CFEFAACF0E94CD3120915009FC
:108FB0003091510940915209509153090F94DB5659
:108FC00020E030E040EF51E40F94DB5620E030E049
:108FD00040EF51E40F94DC5629E838E848E85CE3B8
:108FE0000F9450500F944858C62F653008F486CF20
:108FF000D9CFD7FD02C0C7FF05C00E9457478AE2FC
:109000009EE09BCF0E94CD319B01AC010D2FDD0F67
:10901000110BAC2FCC0FBB0B60E070E0CB01FF203D
:1090200091F065E0609FF001619FF00D1124EA0F5F
:10903000FB1FEE0FFF1FEE0FFF1FE453FA4F60817F
:10904000718182819381E5E0E09FE001E19FD00D95
:109050001124CA0FDB1FCC0FDD1FCC0FDD1FC45343
:10906000DA4F0F94DC56688379838A839B83DF9180
:10907000CF911F910F91FF90EF90DF90CF900895C7
:1090800081E599E00C94F236CF9384E50E94453255
:10909000C0E08823D9F00E94A531C82F1816B4F477
:1090A0000E9440488DE40E94B9368091F10490916D
:1090B000F2040F943C3C6C2FCC0F770B8BE29FE0BB
:1090C0000E94FD3D8AE00E94B936CFEF8C2FCF91F0
:1090D00008954F925F926F927F928F929F92AF927C
:1090E000BF92CF92DF92EF92FF92CF93DF93CDB7F3
:1090F000DEB72C970FB6F894DEBF0FBECDBF409001
:109100004C0950904D0960904E0970904F09209184
:10911000390230913A0240913B0250913C02C30126
:10912000B2010F94DC5669837A838B839C83809091
:10913000500990905109A0905209B0905309209184
:109140003D0230913E0240913F0250914002C501E4
:10915000B4010F94DC566D837E838F839887C09013
:109160005409D0905509E0905609F0905709209184
:109170004102309142024091430250914402C701A2
:10918000B6010F94DC5669877A878B879C8720917C
:109190004502309146024091470250914802C30176
:1091A000B2010F94DC562B013C0120914902309111
:1091B0004A0240914B0250914C02C501B4010F94F8
:1091C000DC564B015C0120914D0230914E024091E2
:1091D0004F0250915002C701B6010F94DC566B014B
:1091E0007C010E9440488CE79EE00E94F23683E5B5
:1091F0000E94F731882321F00E94B9318093370211
:1092000080913702811151C083E69EE00E94F236C0
:1092100084E79EE00E94F23649815A816B817C810D
:1092200083EE9BE20E94E7384D815E816F817885F5
:1092300082ED90E40E94E73849855A856B857C85EC
:109240008FEC90E40E94E73882E79EE00E94F236BD
:109250008AE69EE00E94F236B301A20183EE9BE211
:109260000E94E738B501A40182ED90E40E94E7383E
:10927000B701A6018FEC90E40E94E7388AE02C96B3
:109280000FB6F894DEBF0FBECDBFDF91CF91FF9038
:10929000EF90DF90CF90BF90AF909F908F907F9096
:1092A0006F905F904F900C94B93687E69EE0AECFFA
:1092B0002F923F924F925F926F927F928F929F92E6
:1092C000AF92BF92CF92DF92EF92FF920F931F93D4
:1092D000CF93DF93CDB7DEB76A970FB6F894DEBFB2
:1092E0000FBECDBF83E50E94F731182F3090E50FF8
:1092F000882319F00E94B931382E4090E60F509023
:10930000E70F6090E80F7090E90F8091EA0F90915D
:10931000EB0FA091EC0FB091ED0F8B8B9C8BAD8B75
:10932000BE8B8091EE0F9091EF0FA091F00FB09156
:10933000F10F8F8B988FA98FBA8F112329F03110DD
:1093400003C080E00E94AE3486E50E94F731888B2E
:109350000E94A935882309F4BFC083E40E94F73135
:10936000882309F498C00E94CD316B017C01ACECDC
:10937000B5E0BF83AE83B987A887F5E0FD831D867E
:109380001E8628EC2F8702EC1A86212C88EC8B870E
:1093900092E49C87A885B985BA8BA98B15E0E989E9
:1093A000FA8981909190A190B190FA8BE98B2A85EE
:1093B000322D4B855C85C501B4010F94EA4F87FFC0
:1093C00004C08A86292CAB86BC862D853E854F85B8
:1093D000502FC501B4010F943C59181624F48D8602
:1093E0009E86AF860B2D1150D1F6FD81F150FD8385
:1093F00088859985449699878887F111CBCF2D85EB
:109400003E854F85502F6A85722D8B859C850F94E4
:10941000DC5620E030E040E05FE30F945050A701BD
:1094200096010F94DC566B017C012DEB37E346E887
:1094300055EB0F943C5987FD0AC02DEB37E346E806
:1094400055E3C701B6010F94EA4F181624F580E0E2
:109450000E94AE3415E0AE80BF8005E0D5016D916D
:109460007D918D919D915D014D01B4E08B1A910824
:10947000A70196010F94DB56F40160837183828308
:109480009383015059F711508E819F8144969F8399
:109490008E831111E0CFA889AA2351F00E94A9352B
:1094A000882331F080E09DE00E94F2360E944A3825
:1094B0008AE50E94F731882359F00E94CD316983F3
:1094C0007A838B839C8360E0CE0101960E94C9342D
:1094D000832D0E94AE340BC0311003C098899923AC
:1094E00039F30E94404886E19DE00E94F236332025
:1094F00051F08091E50F811106C00E94574781EE1F
:109500009CE00E94F2360E94404883ED9CE00E945D
:10951000F2368091E50F0E94C9380E94404886ECDF
:109520009CE00E94F236C0906408D0906508E090FC
:109530006608F090670820E030E0A901C701B60195
:109540000F943C5918160CF053C042E0C701B60105
:109550000F944F078DE00E94B9368AE00E94B93619
:10956000A30192016091E60F7091E70F8091E80FDF
:109570009091E90F0F94EA4F81111FC02B893C890C
:109580004D895E896091EA0F7091EB0F8091EC0F2D
:109590009091ED0F0F94EA4F81110FC02F89388DF4
:1095A000498D5A8D6091EE0F7091EF0F8091F00F01
:1095B0009091F10F0F94EA4F81110E9480F96A9601
:1095C0000FB6F894DEBF0FBECDBFDF91CF911F91D4
:1095D0000F91FF90EF90DF90CF90BF90AF909F9052
:1095E0008F907F906F905F904F903F902F90089555
:1095F00081EC9CE00E94F236B3CFCF93C82F82E07B
:10960000C11184E040E060E00E94C9850E944048AA
:1096100089EC99E0CC2311F08EED99E0CF910C9478
:10962000F236FF920F931F93CF93DF93EC018B01E0
:10963000F42E0E943BD50E94574781E399E00E9497
:10964000F2360115110511F402E61FE3209711F41B
:10965000C8E2D9E00E9445BA1F930F93DF93CF93DE
:1096600088E199E09F938F9381E08F930E946EB37E
:109670000E94E084C0916F15C695C6958AE695E173
:109680000E947929DC2FDD0F1D2F1C0FEDB7FEB7CF
:1096900037960FB6F894FEBF0FBEEDBF83E00E9471
:1096A000F7284DEA52E16C2F80E00E94242C1092A2
:1096B000A515D093A61589E099E00E94092A109279
:1096C000A5151093A6158CEF98E00E94092A8EE646
:1096D00095E10F94613A8111E1CF61E08FE199E06A
:1096E0000E94BA3789EE93E030E6019729F0232FE4
:1096F0002A950000E9F7F9CFF89489EE93E038EE67
:10970000019729F0232F2A950000E9F7F9CF0E944D
:109710003BD5FF2041F00E9424360E9439229099C7
:1097200005C0A895FCCF0E943722F7CF909B02C0BE
:10973000A895FCCFF0E0E0E0DF91CF911F910F9171
:10974000FF9019945F926F927F928F929F92AF9247
:10975000BF92CF92DF92EF92FF920F931F93CF931E
:10976000DF931F92CDB7DEB77C0139018B015B011E
:10977000A40EB51ED12CC12CA016B10609F450C000
:10978000F70180809180F80151908F015982C401C6
:109790000F9408565816B9F1652DC4010F94105650
:1097A000FFEFCF1ADF0AC6018F779927892B21F1A6
:1097B00062E070E080E090E00F943B32C4010F94CF
:1097C000085699818917F9F00E9440488BE596E088
:1097D0000E94F23681E00F90DF91CF911F910F919F
:1097E000FF90EF90DF90CF90BF90AF909F908F90C1
:1097F0007F906F905F90089562E070E080E090E06D
:109800000E94EE35DBCFBE016F5F7F4FC3010F9427
:109810000F24F70180819181019691838083ACCFE1
:1098200080E0D9CF8091F60F9091F70F2FEF3FEFA7
:10983000981751F0E92FF0E0EA50F04F228130E024
:109840009F5F9F779093F70FC90108951F920F9222
:109850000FB60F9211240F900FBE0F901F90189506
:109860001F920F920FB60F9211240BB60F920F9307
:109870001F932F933F934F935F936F937F938F9398
:109880009F93AF93BF93CF93DF93EF93FF93C091D9
:10989000C6000091F70FD091F60F11E01D0F1F7752
:1098A00090917904913108F09FC0E92FF0E088276A
:1098B000E35AF34B8F4F0D94D3566E4C9D4CAC4CEA
:1098C000BB4CC24CF44CC64CF44CCA4CCE4CF44C81
:1098D000D24CD64CDA4CE14CF44CEC4CC03229F072
:1098E00028F5CA3011F0CD3031F5011731F0ED2FE8
:1098F000F0E0EA50F04FC283D12FD093F60FFF91E2
:10990000EF91DF91CF91BF91AF919F918F917F9117
:109910006F915F914F913F912F911F910F910F90F8
:109920000BBE0F900FBE0F901F901895CD3481F095
:1099300081E0CE3471F080E10CC0CA3338F4C0331A
:10994000A0F6C03291F2CD32B1F7CFCFCD3499F736
:1099500082E080937904C9CFC13359F018F4C03242
:1099600021F2E9CF88E0C433A1F38BE0C83389F357
:10997000E2CF83E0EECF84E0C03359F386E0C13319
:1099800041F3D9CF85E0C833B1F6E3CF87E0C233E6
:1099900091F6DFCF89E0C13371F6DBCF8AE0C033C7
:1099A00051F6D7CF8CE0C73331F6D3CF8DE0C63335
:1099B00011F6CFCFC03209F498CF8EE0C33549F20B
:1099C000BACF80ED8C0F8A3008F08FCF9FE0909354
:1099D00079048093780489CFCA3019F0CD3009F02A
:1099E00084CF1092790481CFCA3019F0CD3009F0BC
:1099F0007CCF8091A8158823A1F3973041F138F4EA
:109A0000953079F710926C0210924C08EACF9A3098
:109A100011F19F3031F790917804809149081092AC
:109A20004908823089F38430E9F08130D1F69923F6
:109A3000B1F09130B1F682E080934B0880914A08F2
:109A4000882379F2109255020E942422CACF81E025
:109A500080934206C6CF81E080934106C2CF8093B7
:109A60004B08BFCF8BE09EE19093C2078093C10764
:109A7000B8CF8EBD0DB407FEFDCF08958FEF8EBD1C
:109A80000DB407FEFDCF8EB50895909164009B7FC5
:109A900090936400982F906A96959CBD80FD03C0BA
:109AA00091E0863009F490E09DBD0895CF93DF9357
:109AB000EB010E94F236CE01DF91CF910C9423CFBF
:109AC000AF92BF92CF92DF92EF92FF920F931F93CC
:109AD000CF93DF93CDB7DEB7E6970FB6F894DEBF2E
:109AE0000FBECDBF0091F4041091F504F801019070
:109AF0000020E9F731976F01C01AD10AF801CF01B0
:109B0000801B910B8C159D053CF481918F32B9F728
:109B1000DF0111971C92F3CF8BE1EBEFF5E1DE0152
:109B20005C9601900D928A95E1F7F12CE12CEC14F2
:109B3000FD040CF05DC0F801EE0DFF1D8081811168
:109B400003C08FEFE81AF80A5801AE0CBF1CF501EC
:109B50008081882309F44CC0FFEFEF1AFF0AF80157
:109B6000EE0DFF1D7F01E01AF10A81918111FACFFC
:109B7000CE014C960E941ED38BE1FE017C96DE0145
:109B8000119601900D928A95E1F7B501CE010196EB
:109B90000E94E5CBCE0101960E94F7338FE20E942E
:109BA000B93680916A1281113BC087E593E00E942B
:109BB00023CF8091DC1584FF1BC019821C8221E019
:109BC000A501BE01645E7F4FCE0101960F94700522
:109BD000811129C08AE00E94B9360E944048B5012F
:109BE00081EE94E10E94564DCE0101960E94F7331A
:109BF0008AE00E94B936CE014C960E94F733E69671
:109C00000FB6F894DEBF0FBECDBFDF91CF911F918D
:109C10000F91FF90EF90DF90CF90BF90AF9008959D
:109C20008AE692E1C4CFCE014C960E94DBD28BE152
:109C3000FE013196DE015C9601900D928A95E1F766
:109C4000CE0101960E94F73372CF2F923F924F922E
:109C50005F926F927F928F929F92AF92BF92CF92BC
:109C6000DF92EF92FF920F931F93CF93DF9300D079
:109C700000D000D01F921F92CDB7DEB7B82E8091D2
:109C8000E310843008F0D1C10F946E326B017C0177
:109C90008091E310811108C08091F60F9091F70F29
:109CA000891B8F7709F4D9C681E6A82E13C08A30A4
:109CB00019F08D3009F0F6C01092DE1080917C1002
:109CC00090917D10FC01E858FF4E1682892BF1F42B
:109CD0000E94DAF08091E310843008F0ECC08091AB
:109CE000F60F9091F70F891B8F7709F4E4C00E945B
:109CF000124C97FFDCCF0E94574781EA97E00E9401
:109D0000F2368091F60F8093F70FE4CF10927D101A
:109D100010927C100EE710E1F8018191803209F475
:109D200046C08E3409F0A9C06CE977E0C8010F94F1
:109D3000674F4C01892B41F06EE470E0C801049636
:109D40000F94315A009709F4C8014AE050E070E0DE
:109D500060E001960F94D74C2B013C018091781064
:109D600090917910A0917A10B0917B100196A11D6D
:109D7000B11D481659066A067B0629F060E089E69F
:109D800097E0892851F16AE270E0C8010F94605AA7
:109D90009C01009729F1982F901B912C992349F051
:109DA0009150F801E90FF11D80819826F7CF8F01BE
:109DB000B3CF4AE050E070E060E0C90101960F9433
:109DC000D74C292D30E050E040E06217730784073C
:109DD000950751F060E08AE497E00F9476277ACFF8
:109DE00060E080E297E0F9CF4092781050927910CD
:109DF00060927A1070927B10809104088130E1F0BB
:109E000067E470E0C8010F94315A0097A9F04AE066
:109E100050E070E060E001960F94D74C643071051B
:109E20008105910548F48FE796E00E94F23660E0E4
:109E300085E796E00E9489B3C0925108D0925208FB
:109E4000E0925308F092540880917E108B3309F40D
:109E500041CF8091E310843008F03CCF8091E51031
:109E60008A9DC00111246EE770E18A519F4E0F94C4
:109E70003C5A80E00F9430272DCF8091DC1580FF75
:109E8000BBCF65EE7EE3C8010F94674F009731F0BA
:109E9000FC01838180538A3008F0AECF60E086EF0A
:109EA00096E09BCF2CE730E14EE750E16EED70E19C
:109EB0000E94B3210FCF8091DC1582FFB6C01A82B9
:109EC000198271E6F72EE0E1EE2EF9E6DF2E8091A1
:109ED000E310843008F0A9C00E94EB218111A5C0D5
:109EE00041E050E0BE016B5F7F4F8FE397E10E943E
:109EF000C3CF0D8110E0019711F00FEF1FEF80919C
:109F0000471790914817A0914917B0914A1780932D
:109F1000D8159093D915A093DA15B093DB150E944C
:109F2000EB210F3F100749F4811107C00E945747EA
:109F30008FEB97E00E94F236CACF4091E510242FB4
:109F400030E00A3061F00D3051F0882309F45FC031
:109F500089819A81009719F001969A8389831092DA
:109F60007A0489819A81F29EF001F39EF00D11240A
:109F7000ED51FF4EE80FF91F1382892B69F50E94FE
:109F8000DAF00E94EB21882309F4A1CF0E94EADCD9
:109F90008FE397E10E94DBD28091D315882391F162
:109FA00081508093D3158D9DC001112462E0805DA6
:109FB000984F0F94CB40E091D31524E0E29FF0013D
:109FC0001124E45DF84F60817181828193810E9448
:109FD000CA250F94CB3D7BCF1A82198281E00F9462
:109FE00030278091D8159091D915A091DA15B091AC
:109FF000DB158093DF109093E010A093E110B093F5
:10A00000E210BFCF0F94BA3DE092040860CF4F9D9D
:10A01000A00111244A515F4E9E012F5F3F4F6AE716
:10A0200074E0802F0E94B32152CF0F946E326B01E7
:10A030007C01B11004C080912B07882351F0C0929D
:10A040004108D0924208E0924308F0924408BB24B1
:10A05000B3948091CD049091CE04A091CF04B0919F
:10A06000D0040097A105B10551F1409141085091EC
:10A0700042086091430870914408840F951FA61F01
:10A08000B71FA7019601281B390B4A0B5B0BDA019E
:10A09000C901B7FD14C00E94574760914F087091E5
:10A0A00050088AE198E00E94564D8AE00E94B93635
:10A0B00040E070E060E090E080E00E94114B809111
:10A0C000100290911102A0911202B0911302892BFB
:10A0D0008A2B8B2B79F0909142158091431598171C
:10A0E00009F4ACC1C0924108D0924208E092430802
:10A0F000F092440880918B0490918C049099E0C177
:10A10000019690938C0480938B0480918B049091A2
:10A110008C048E3E92406CF00E94574787EF97E088
:10A120000E94F23640E070E060E090E080E00E9443
:10A13000114B0F946E324B015C0180914C088111E0
:10A1400008C0209142159091431581E0291301C068
:10A1500080E020911C1530911D1591E089272A3A45
:10A1600031050CF480E091E040917F04509180042F
:10A170006091810470918204452B462B472B09F492
:10A1800090E0981789F0882309F4A0C1D501C40193
:10A1900080569444A24FBF4F80937F0490938004D5
:10A1A000A0938104B09382044090F20F5090F30F7B
:10A1B0006090F40F7090F50F20917B0430917C0437
:10A1C00040917D0450917E04C301B2010F94EA4F87
:10A1D000882319F180917F0490918004A0918104DB
:10A1E000B091820440927B0450927C0460927D0482
:10A1F00070927E04892B8A2B8B2B09F449C0D501E0
:10A20000C40180569444A24FBF4F80937F04909323
:10A210008004A0938104B093820480917F04909184
:10A220008004A0918104B09182040097A105B1053A
:10A2300079F1881A990AAA0ABB0AB7FC29C01092B8
:10A240007F0410928004109281041092820482EEA6
:10A2500097E00E94F23660E08EEC97E00E9489B3AE
:10A2600080911E1590911F151816190624F490E080
:10A2700080E00E946CDC80916E0890916F08181647
:10A28000190634F410926F0810926E080E944BC7A2
:10A290008091870490918804A0918904B0918A04E8
:10A2A00046015701881A990AAA0ABB0AD501C401B6
:10A2B000B7FD9CC1209142159091431540915C02DD
:10A2C00080915B02291306C190918609899FC00184
:10A2D0001124880F892F881F990B91958D83809168
:10A2E0008709489FC0011124880F892F881F990B67
:10A2F00091958E830F946E3269837A838B839C83CE
:10A3000040E0BE016F5F7F4FCE0105960E943EDDAB
:10A310006D8170E089E00F94653141E0BE016F5FAF
:10A320007F4FCE0105960E943EDD6E8170E087E092
:10A330000F94653180914E06882309F44AC100913B
:10A34000330210913402C801029720911E153091FA
:10A350001F15281739070CF43CC1809043158F82D4
:10A36000188619861A861B86809142159F8089154A
:10A3700009F4CAC0892D90E030E6A32EA89EF00112
:10A38000A99EF00D1124E556F64F45895689678937
:10A39000708D452B462B472B81F4418D528D638D5B
:10A3A000748D452B462B472B41F4458D568D678D7B
:10A3B00070A1452B462B472BE1F120E6B22EB89E2B
:10A3C0009001B99E300D1124A9014556564F1A012E
:10A3D000FA0161817281838194810F948A594B01C2
:10A3E0005C01F10161A172A183A194A10F94EF4FCF
:10A3F0002B013C01F10165A176A187A190A50F94E5
:10A40000EF4F9B01AC01C301B2010F94D657A501D8
:10A4100094010F9450504B015C01288539854A8581
:10A420005B850F943C59181624F488869986AA8671
:10A43000BB868F818F5F8F708F8396CFBB2019F083
:10A4400010928D0457CE0F946E32009141081091F6
:10A450004208209143083091440880901002909067
:10A460001102A0901202B0901302080D191D2A1DAE
:10A470003B1D601B710B820B930B97FDE1CF80910D
:10A480008D04811137CE81E080938D045F9A809195
:10A49000BF078E7F8093BF078A9A8091BF078D7F09
:10A4A0008093BF0780910801809581708093060199
:10A4B0008091BF078B7F8093BF070E9437221ACEFF
:10A4C000181619060CF021CE01971BCE80E090E003
:10A4D000DC0162CE2091431550E6259F90011124A6
:10A4E0002556364FF901EA5AFF4F9081899FC001E6
:10A4F0001124880F892F881F990B91958D83295AD4
:10A500003F4FF9018081EDCE20912D0230912E0236
:10A5100040912F0250913002688579858A859B850C
:10A520000F9450504B015C01B801012E000C880BB8
:10A53000990B0F94F14F9B01AC01C501B4010F942D
:10A54000DC5669837A838B839C83409131025091DE
:10A550003202B801CE0101960E9406D689809A8007
:10A56000AB80BC804090830450908404609085044C
:10A5700070908604A3019201C501B4010F94EA4FC3
:10A5800087FF16C028E431EE4AE75FE3C301B2015A
:10A590000F94505020E037ED43EA5CE30F94DC5613
:10A5A000A50194010F94505069837A838B839C8317
:10A5B00069817A818B819C81609383047093840488
:10A5C00080938504909386040F944858CB010E9491
:10A5D0006CDCF4E6CF0ED11CE11CF11CC0928704A8
:10A5E000D0928804E0928904F0928A040E94DAF002
:10A5F00080910408882309F4F0C1809155028823D2
:10A6000009F471C080914A0881116DC00E94123610
:10A61000811105C080912B07882309F464C0F89448
:10A62000649B10C08091510290915202A0915302FC
:10A63000B09154028093390690933A06A0933B065A
:10A64000B0933C066091390670913A0680913B06C2
:10A6500090913C06789420E030E0A9010F94EA4FF5
:10A6600087FF41C001E000934A0880912B078111C8
:10A6700038C00E94EB370093490840E366E878E071
:10A6800084E290E40E94F03761E088E190E40E9467
:10A69000D2371091D10460E0102784E59AE069F484
:10A6A00084E798E00E94BA3780E30E94B9368AE0D6
:10A6B0000E94B93660E087E598E00E94BA3782E6EA
:10A6C00098E00E94F23680E30E94B9368AE00E9448
:10A6D000B936112331F08DE598E09093C20780934D
:10A6E000C1070E94EADC90910901892F8095817051
:10A6F00010910802181709F45AC02091DC15206245
:10A700002093DC158093080290FD10C064EF71E087
:10A7100080E090E00E94EE350F94423E8091DC157F
:10A7200083FDBEC1112309F442C002C00F94313E23
:10A73000123008F46BC100E00E948F2883E0809300
:10A7400078020F946E326C597F4F8F4F9F4F6093FA
:10A75000F9047093FA048093FB049093FC040023A3
:10A7600031F1123021F58091DC1583FF20C00F9468
:10A77000263D882379F081E00F94423C42EB50E083
:10A780006AE978E080EE95E10E94C3CF80EE95E122
:10A790000E94DBD20E94E533811144C10E94CF3375
:10A7A0000F94103F81E08093D2150F94523F0F9485
:10A7B0006E326B017C0110910F021123F1F0809138
:10A7C0004D088823D1F040918E0450918F04609100
:10A7D00090047091910446015701841A950AA60AC3
:10A7E000B70AB501A40177FD1AC0833009F430C15E
:10A7F0000CF01FC181300CF024C1212F30E0A8EEF5
:10A80000B3E00F948256C60ED71EE81EF91EC09202
:10A810008E04D0928F04E0929004F0929104809183
:10A820006208813009F073C00F946E326B017C01B5
:10A830008091960490919704A0919804B091990406
:10A84000A7019601281B390B4A0B5B0BDA01C901E2
:10A85000B7FD3AC0D701C601805F984DAF4FBF4FDB
:10A860008093960490939704A0939804B0939904CE
:10A870008090BF059090C005A090C105B090C20522
:10A880000E940DFCAB01BC014093BF055093C00575
:10A890006093C1057093C2058091B0079091B10794
:10A8A000A091B207B091B30788199909AA09BB0909
:10A8B000840F951FA61FB71F8093B0079093B10711
:10A8C000A093B207B093B307809192049091930440
:10A8D000A0919404B091950446015701881A990AF1
:10A8E000AA0ABB0AD501C401B7FD11C020E8C20EF7
:10A8F0002EEED21E26E3E21EF11CC0929204D092EC
:10A900009304E0929404F09295040E94EEDB0F947D
:10A91000D8010E9495B78091CC04882379F10F94D7
:10A920006E326B017C018091C8049091C904A091A2
:10A93000CA04B091CB0446015701881A990AAA0AA1
:10A94000BB0AD501C401B7FD19C02091CC0430E089
:10A95000A8EEB3E00F948256C60ED71EE81EF91E6D
:10A96000C092C804D092C904E092CA04F092CB0409
:10A9700080E00F94F3078AE00E94B9368091C70403
:10A98000882359F10F946E326B017C018091C304CE
:10A990009091C404A091C504B091C604A70196018A
:10A9A000281B390B4A0B5B0BDA01C901B7FD15C037
:10A9B0002091C70430E0A8EEB3E00F948256C60E93
:10A9C000D71EE81EF91EC092C304D092C404E092C0
:10A9D000C504F092C6040F943A3D2B960FB6F89436
:10A9E000DEBF0FBECDBFDF91CF911F910F91FF90C2
:10A9F000EF90DF90CF90BF90AF909F908F907F901F
:10AA00006F905F904F903F902F90089560E087E99E
:10AA100098E00E9489B38091070581118CCE0E9435
:10AA2000E08489CE84EB98E09093C2078093C107BD
:10AA3000BECE843009F0E1CE0E9440488BEB98E016
:10AA400004C00E9440488AEE98E00E94F236D5CEBB
:10AA50000E94404883ED98E0F8CF80915108909192
:10AA60005208A0915308B0915408A7019601281BE1
:10AA7000390B4A0B5B0BDA01C901885E9340A109CF
:10AA8000B109B7FD11C989EB97E00E94F236C09277
:10AA90005108D0925208E0925308F092540804C929
:10AAA000123028F460E085EA98E00E9489B301E062
:10AAB00043CECF93DF93C82FD62F80919C0F83FD79
:10AAC00014C080919809811110C080917D029091ED
:10AAD0007E02AC014150510920911E1530911F1585
:10AAE0002417350714F40E946CDC40E06D2F8BE0D6
:10AAF0000E94C985CC2339F040E061E080E0DF911D
:10AB0000CF910D94EB098091980991E0892780936A
:10AB10006C0280916C02882389F080911C159091C1
:10AB20001D1520911E1530911F15821B930B97FF49
:10AB300003C0919581959109029744F410926C029B
:10AB400080919C0F83FF06C0C1E01AC080E00E9484
:10AB5000254EDFCFC0919809C11112C080917D02AE
:10AB600090917E02019720911E1530911F15281794
:10AB7000390754F70E94404888EB99E00E94F2366A
:10AB80008C2FDF91CF910895AF92BF92CF92DF9239
:10AB9000EF92FF920F931F93CF93DF93CDB7DEB762
:10ABA00064970FB6F894DEBF0FBECDBF0E94444835
:10ABB000D82E87FDB5C08AE50E944532882309F466
:10ABC000C0C040E050E0BA018AE50E9460327B01DB
:10ABD0008C014D2D63E085E00E94C9852091EE0F28
:10ABE0003091EF0F4091F00F5091F10F60E070E065
:10ABF00088EC93E40F94DB565B016C019701A8018C
:10AC00000F943C59181614F07501860120E030E0CD
:10AC1000A901B701C8010F943C59181624F4E12C7E
:10AC2000F12C00E010E0B701C8010F944858072E3E
:10AC3000000C880B990B0F94F14F6D837E838F83EB
:10AC4000988720E030E0A9010F94EA4F882321F093
:10AC5000CE0105960E94182680E090E0A0EAB1E4BB
:10AC600089879A87AB87BC871D861E861F86188AB0
:10AC70008CE40E94F731882309F468C00E94CD312A
:10AC80006B017C0120E030E0A901C701B6010F94FF
:10AC90003C5987FF04C0F7FAF094F7F8F094C98A9A
:10ACA000DA8AEB8AFC8A20911E1530911F15243018
:10ACB000310574F080911C1590911D15821B930B2A
:10ACC00097FF03C091958195910901E004970CF4D9
:10ACD00000E063E080E00E945955811140C083E0AC
:10ACE00080932402109206050E94E0846D817E818B
:10ACF0008F8198858B019C01305809831A832B839F
:10AD00003C8320E030E0A9010F94EA4F882321F032
:10AD1000CE0101960E941826109206050E94E0843A
:10AD200064960FB6F894DEBF0FBECDBFDF91CF9112
:10AD30001F910F91FF90EF90DF90CF90BF90AF9059
:10AD40000895E12CF12C00E211E443CFC090C70537
:10AD5000D090C805E090C905F090CA0593CF83E074
:10AD6000E82E22E0AE01475F5F4FBE016F5E7F4F6E
:10AD7000CE010D960F947A29B9CF6F927F928F9260
:10AD80009F92AF92BF92CF92DF92EF92FF920F937A
:10AD90001F93CF93DF9300D000D01F921F92CDB7A7
:10ADA000DEB75C014B013A01F22E680100914706C3
:10ADB00010924306109244061092450610924606E1
:10ADC000109247060F947A3280911E1590911F15AC
:10ADD0008C159D051CF4C6010E946CDC60E080E0CF
:10ADE0000E94595581112FC1109206050E94E084DE
:10ADF0001C141D0444F4C6010E946CDC40E060E0B9
:10AE000080E00F94EB0940E060E088E00E94C98593
:10AE100060E081E00E94595580E090E0A0E7B2E454
:10AE200089839A83AB83BC8380E090E0A0E8B0EC98
:10AE30008D839E83AF83B887BE016F5F7F4FCE0146
:10AE400005960E94A8F087E00E94E8EE811158C0A4
:10AE50008091EE0F9091EF0FA091F00FB091F10F54
:10AE60004091A6045091A7046091A8047091A90490
:10AE7000C090A204D090A304E090A404F090A50494
:10AE8000C0923108D0923208E0923308F092340830
:10AE9000409335085093360860933708709338080C
:10AEA0008093390890933A08A0933B08B0933C08EC
:10AEB00080E090E0A8E4B2E489839A83AB83BC830A
:10AEC000CE0101960E94C8F78091AA049091AB042C
:10AED000A091AC04B091AD048093390890933A08E6
:10AEE000A0933B08B0933C0880E090E0A0EAB0E477
:10AEF00089839A83AB83BC83CE0101960E94C8F7F5
:10AF0000C12CD12C80E7E82E82E4F82EC982DA82A7
:10AF1000EB82FC8280E090E0A0E8B0E48D839E8329
:10AF2000AF83B887BE016F5F7F4FCE0105960E9449
:10AF3000A8F020E030E0A9016091AE047091AF0468
:10AF40008091B0049091B1040F94EA4F87FF0BC039
:10AF5000C982DA82EB82FC82BE016F5F7F4F8EEA8C
:10AF600094E00E94A8F08091AE049091AF04A0916B
:10AF7000B004B091B1048093F20F9093F30FA093BB
:10AF8000F40FB093F50F80933D0890933E08A09383
:10AF90003F08B09340088DE398E00E9420ED809137
:10AFA000CB0581110F946C3C109206050E94E08441
:10AFB00061E081E69AE00E94BA3780912B078150C8
:10AFC00080932B074CEC5DE169E67AE085E00F9415
:10AFD000842A80912B07882339F00F94CB3D8091F0
:10AFE0002B07815080932B078091A104882351F077
:10AFF0001092A10480919F04809386098091A004FF
:10B00000809387090E94242280916208823011F483
:10B010000E94CFFC0F940B400E94E08428960FB64C
:10B02000F894DEBF0FBECDBFDF91CF911F910F917E
:10B03000FF90EF90DF90CF90BF90AF909F908F9058
:10B040007F906F900895E12C2F2DA301B401C501CD
:10B050000F947A29CDCE4F925F926F927F92AF92EA
:10B06000BF92CF92DF92EF92FF921F93CF93DF9325
:10B0700000D000D01F921F92CDB7DEB75C01E62E44
:10B08000F42E642F80E00E945955182F81111BC0A7
:10B09000EE2021F0109206050E94E084812F289670
:10B0A0000FB6F894DEBF0FBECDBFDF91CF911F91D9
:10B0B000FF90EF90DF90CF90BF90AF907F906F9018
:10B0C0005F904F900895EE2029F040E06F2D83E0CF
:10B0D0000E94C98580E090E0A0E7B2E48D839E8362
:10B0E000AF83B88780E090E0A0E8B0EC89839A83D2
:10B0F000AB83BC83BE016B5F7F4FCE0101960E9484
:10B10000A8F068E873E180E090E00E94EE35C12C81
:10B11000D12C88ECE82E81E4F82ECD82DE82EF82FD
:10B12000F88680E090E0A0E8B0E489839A83AB835E
:10B13000BC83BE016B5F7F4FCE0101960E94A8F0D9
:10B140004090D50F5090D60F6090D70F7090D80FC9
:10B15000C092D50FD092D60FE092D70FF092D80FB1
:10B1600080E090E0A0E2B2E48D839E83AF83B88755
:10B17000F50180819181A281B38189839A83AB8318
:10B18000BC83BE016B5F7F4FCE0101960E94A8F089
:10B190004092D50F5092D60F6092D70F7092D80F71
:10B1A000129A64E670E080E090E00E94EE3576CF7F
:10B1B000BF92CF92DF92EF92FF920F931F93CF93A4
:10B1C000DF9300D01F92CDB7DEB77C016B018A01FF
:10B1D000B22E61E084E59AE00E94BA374CEC5DE162
:10B1E0006BE57AE085E00F94842A90912B0781E04B
:10B1F000890F80932B078091DC1582FF06C08B7F1F
:10B200008093DC159E5F90932B070E9407FD80E1E1
:10B21000E6EEFFE0A2EAB4E001900D928A95E1F734
:10B220000E94EADC8091A10481110FC081E080932B
:10B23000A1048091860980939F04109286098091D1
:10B2400087098093A0041092870920E030E0A901CB
:10B25000F70160817181828193810F94EA4F882385
:10B26000F1F08091980981110CC080917D0290913C
:10B270007E02019720911C1530911D152817390762
:10B2800074F080E090E0A0E7B2E489839A83AB8316
:10B29000BC83BE016F5F7F4FC7010E94A8F087E0AB
:10B2A0000E94E8EE811103C0B6010F941D0120E059
:10B2B00030E0A901F80160817181828193810F944E
:10B2C000EA4F882329F042E06B2DC8010E942B58D9
:10B2D000129A64E670E080E090E00E94EE3581E032
:10B2E0000F900F900F900F90DF91CF911F910F91C2
:10B2F000FF90EF90DF90CF90BF900895CF92DF92B4
:10B30000EF92FF92CF93DF936B017C01D42FC0911A
:10B310004D0883E080934D0881E080934C08C11470
:10B32000D104E104F10431F00F946E32C60ED71E41
:10B33000E81EF91E80914C08882389F0C114D104BD
:10B34000E104F10421F48D2F0E94254EF3CF0F94D8
:10B350006E326C197D098E099F0997FDF4CF10920A
:10B360004C08C0934D08DF91CF91FF90EF90DF9094
:10B37000CF9008951F93CF93DF93D82FC62F0E94AD
:10B38000FD4A61E08C2F0E94FD330F946E326853AA
:10B3900070458F4F9F4F6093430670934406809390
:10B3A0004506909346061092470610914D0883E09B
:10B3B00080934D0830E020E049E450E466E47AE010
:10B3C00082E00E94133881E080934C0880914C0801
:10B3D000882309F463C060E08C2F0E94FD338091C4
:10B3E0004706882309F456C040E060E08AE00E94E6
:10B3F000C9850E9440488CE29AE00E94F23630E013
:10B4000020E046E15AE06DE17AE082E00E941338E4
:10B4100041E060E070E0CB010E947E5930E020E026
:10B4200050E040E069E07AE085E00E941338109235
:10B43000430610924406109245061092460610925A
:10B4400047060F947A3260E080E00E9459558D2FB4
:10B450000E94FD4A0F946E32685370458F4F9F4F84
:10B460006093430670934406809345069093460686
:10B470001092470630E020E049E450E46DEF79E0B7
:10B4800082E00E94133881E080934C0861E08C2FA9
:10B490000E94FD3381E00E94254E98CF10934D0805
:10B4A000DF91CF911F910895CF92DF92EF92FF929B
:10B4B0000F931F93CF93DF93CDB7DEB7A0970FB64F
:10B4C000F894DEBF0FBECDBF0E94444887FDD1C0B7
:10B4D000482F61E081E00E94C98585E40E94F73130
:10B4E000882309F4D5C00E94CD316B017C0120E096
:10B4F00030E0A9010F943C5987FF04C0F7FAF0949B
:10B50000F7F8F094F7FAF094F7F8F094C98ADA8A29
:10B51000EB8AFC8A8CE0E3E8F2E0DE011196019010
:10B520000D928A95E1F78AE50E944532882351F011
:10B5300040E050E0BA018AE50E94603269877A876C
:10B540008B879C8788E50E944532882351F040E034
:10B5500050E0BA0188E50E94603269837A838B8368
:10B560009C8389E50E944532882351F040E050E0F9
:10B57000BA0189E50E9460326D837E838F8398874C
:10B5800085E50E94F731882309F489C00E94CD31F6
:10B590006B017C0120E030E0A901C701B6010F94E6
:10B5A0003C5987FF04C0F7FAF094F7F8F094F7FAE3
:10B5B000F094F7F8F094CD8ADE8AEF8AF88E198E2F
:10B5C0001A8E1B8E1C8E8CE40E94F731882309F49E
:10B5D0006FC00E94CD316B017C0120E030E0A901F9
:10B5E000C701B6010F943C5987FF04C0F7FAF094E5
:10B5F000F7F8F094CD8EDE8EEF8EF8A262E070E068
:10B6000082E40E94AB33F82E80912B07811131C068
:10B6100021E0AE014B5E5F4FBE016F5F7F4FCE01F9
:10B6200041960E94D858882321F16F2D81E00E9415
:10B63000BA5982E50E944532882309F442C00E942B
:10B64000C93140E050E060EA71E44D875E876F8762
:10B65000788B20912B07222361F08C012F2DAE01D6
:10B66000435F5F4FBE01635E7F4FCE0149960E94EC
:10B67000BD56A0960FB6F894DEBF0FBECDBFDF91CA
:10B68000CF911F910F91FF90EF90DF90CF90089591
:10B69000C12CD12C80E8E82E80E4F82E33CFC09066
:10B6A000C305D090C405E090C505F090C60572CFE3
:10B6B000C090C705D090C805E090C905F090CA05B4
:10B6C0008CCF90E080E0BDCFCF92DF92EF92FF92DF
:10B6D0000F931F93CF93DF93CDB7DEB76C970FB661
:10B6E000F894DEBF0FBECDBF8CE40E94F7318823F3
:10B6F00009F4C3C00E94CD316B017C0120E030E031
:10B70000A9010F943C5987FF04C0F7FAF094F7F8A9
:10B71000F094F7FAF094F7F8F094C98EDA8EEB8E85
:10B72000FC8E8CE0E3E8F2E0DE01119601900D92D0
:10B730008A95E1F788E50E9445328823A1F040E030
:10B7400050E0BA0188E50E94603220914C093091A6
:10B750004D0940914E0950914F090F94DB56698372
:10B760007A838B839C8389E50E9445328823A1F0EC
:10B7700040E050E0BA0189E50E94603220914C0916
:10B7800030914D0940914E0950914F090F94DB566D
:10B790006D837E838F8398878AE50E944532882354
:10B7A00051F040E050E0BA018AE50E9460326987BA
:10B7B0007A878B879C87F090DC15F2FAFF24F0F8EB
:10B7C00040E061E080E00E94C98560E080E50E9481
:10B7D000BA33E82E1D861E861F86188A80912B0795
:10B7E00081113CC02E2DAE01435F5F4FBE016F5FE4
:10B7F0007F4FCE0149960E94D858882379F18091D5
:10B80000CB0581110F946C3CFF2011F0EE2031F13B
:10B8100060E080E00E94BA59898D9A8DAB8DBC8D15
:10B82000B0588D8B9E8BAF8BB88F198A1A8A1B8A62
:10B830001C8A1D861E861F86188A80912B078823E6
:10B8400069F010E000E020E0AE014B5E5F4FBE010A
:10B850006F5E7F4FCE010D960E94BD566C960FB65F
:10B86000F894DEBF0FBECDBFDF91CF911F910F9136
:10B87000FF90EF90DF90CF900895C12CD12C80E8FD
:10B88000E82E80E4F82E45CF2F923F924F925F92A0
:10B890006F927F928F929F92AF92BF92CF92DF92E0
:10B8A000EF92FF920F931F93CF93DF93CDB7DEB745
:10B8B000E1970FB6F894DEBF0FBECDBF89AB2091E4
:10B8C0004D0828AB11E010934D088091F3048D349E
:10B8D00009F463C4843511F40C940271873409F0BF
:10B8E00044C18091F1049091F2048A31910509F4E8
:10B8F000D7C108F03DC18430910508F030C12091D6
:10B9000004088230910508F451C1213009F054C176
:10B9100011E0029709F010E00E94773219821A8232
:10B920001B821C821D821E821F82188682E50E9455
:10B930004532882309F453C10E94CD316B017C014B
:10B9400020E030E0A9010F94EA4F882309F4EAC00F
:10B950004090E60F5090E70F6090E80F7090E90F6D
:10B960008091EA0F9091EB0FA091EC0FB091ED0F49
:10B9700088A799A7AAA7BBA7809031089090320802
:10B98000A0903308B0903408809135089091360823
:10B99000A0913708B09138088CA79DA7AEA7BFA784
:10B9A000A5019401C301B2010F94EA4F81110DC0AA
:10B9B0002CA53DA54EA55FA568A579A58AA59BA543
:10B9C0000F94EA4F882309F4ADC0A3019201C50189
:10B9D000B4010F94DB5620E030E040E05FE30F94C9
:10B9E00050506CA37DA38EA39FA328A539A54AA57B
:10B9F0005BA56CA57DA58EA59FA50F94DB5620E0C9
:10BA000030E040E05FE30F9450502B013C0120E018
:10BA100030E0A901C701B6010F94EA4F881F8827BB
:10BA2000881F181709F4D2C080E090E0A0E8BFEBAF
:10BA300088A799A7AAA7BBA72CA13DA14EA15FA14A
:10BA4000CA01B9010F9450504B015C01A30192014E
:10BA5000C301B2010F9450509B01AC01C501B40168
:10BA60000F94DC560F948A594B015C01AC019B0189
:10BA7000C701B6010F94DB566CA77DA78EA79FA7C1
:10BA8000A5019401C701B6010F94DC569B01AC01DE
:10BA90006CA57DA58EA59FA50F9450506B017C01D0
:10BAA00020E030E0A9010F943C5987FD94C0C70104
:10BAB000B6010F948A596B017C01C301B201905801
:10BAC000A50194010F94D65728A539A54AA55BA5D1
:10BAD0000F945050A70196010F9450502CA13DA1F6
:10BAE0004EA15FA10F94DC5669837A838B839C837C
:10BAF000A50194016CA17DA18EA19FA10F94D657A1
:10BB000028A539A54AA55BA50F945050A701960119
:10BB10000F945050A30192010F94DC566D837E83E5
:10BB20008F83988720E030E0A90169817A818B8139
:10BB30009C810F94EA4F811166C020E030E0A9019A
:10BB40006D817E818F8198850F94EA4F81115BC052
:10BB50000E9457478EE39FE00E94F2362DC084304A
:10BB6000910509F463C0459739F10F946C2924C0FD
:10BB70008A32910509F4ECC158F48C31910509F42D
:10BB8000AAC008F490C04D9781F70E94137414C0A6
:10BB90008B35910509F459C28C35910509F459C2C8
:10BBA0008A35910511F71092630806C0213021F4FF
:10BBB0000E9477320E9415F539A9311102C00F9405
:10BBC000CF3288A980934D080C94946980E090E06E
:10BBD000A0E8BFE32DCFC12CD12C76016ECF89E434
:10BBE0000E944532882331F00E94CD3169837A83E7
:10BBF0008B839C838AE40E944532882309F492CF88
:10BC00000E94CD318BCF412FBE016F5F7F4F81E30B
:10BC100098E00F9468330F946E32609341087093EC
:10BC200042088093430890934408C6CF80E50E9461
:10BC30004532C12CD12C7601882321F00E94762731
:10BC40006B017C0183E50E944532882361F00E94EC
:10BC5000CD3120E030E04AE754E40F9450500F9487
:10BC60004F586B017C010E94EADC8091AD1281117A
:10BC700005C060E084E59FE00E9489B30F946E32B6
:10BC8000C60ED71EE81EF91E0F946E326C197D0980
:10BC90008E099F0997FF90CF80E00E94254EF4CF38
:10BCA0000E94073E89CF0F942D40811185CF8CE0F3
:10BCB000EFE8F2E0DE01119601900D928A95E1F72E
:10BCC00070E060E080E50E945232BE016F5F7F4FFE
:10BCD0000F941D0171CF87E00E94E8EE811106C02C
:10BCE00060E08FE40E94BA33811166CF0E94EADCE3
:10BCF000109238026091E50F8CE40E94BA33982EBE
:10BD000080E00E94AE340F946E32609341087093CD
:10BD10004208809343089093440880917402909164
:10BD20007502A0917602B09177028093BF04909340
:10BD3000C004A093C104B093C20480916E0290919C
:10BD40006F029093BE048093BD0484E690E09093CC
:10BD50006F0280936E0281E08093BD070E9489FA92
:10BD60008AE50E94F731A82E88E50E94F731182F46
:10BD700089E50E94F731B82E181308C0B12EA11220
:10BD800005C011E0BB24B394AA24A39482E50E94C9
:10BD90004532882309F4D2C00E94CD316C8F7D8F4B
:10BDA0008E8F9F8F20E030E0A9010F94EA4F882307
:10BDB00049F0111103C0BB2009F494C0CE014C9688
:10BDC0000F94592B112309F488C0BB2009F482C0B9
:10BDD0001092E60F1092E70F1092E80F1092E90F01
:10BDE0001092EA0F1092EB0F1092EC0F1092ED0FE1
:10BDF0000E94D8F0E1ECF7E2C590D590E590F49080
:10BE0000E5ECF7E24590559065907490A701960196
:10BE1000C301B2010F94EA4F87FF95C0A7019601B5
:10BE2000C301B2010F94D6579B01AC010F9450503F
:10BE300020E030E040E85FE30F94DC560F948A592D
:10BE400020E030E048E452E40F94505069837A8354
:10BE50008B839C838091EE0F9091EF0FA091F00F58
:10BE6000B091F10F8CA39DA3AEA3BFA320E030E05F
:10BE700040EC5FE3C301B2010F9450502B013C0131
:10BE800077FA709477F8709420E030E040EC5FE34C
:10BE9000C701B6010F9450509058DE0111966D0104
:10BEA000ECA0FDA00EA11FA1A30192010E94D1EF61
:10BEB0000E94FFFB1092E60F1092E70F1092E80F1E
:10BEC0001092E90F1092EA0F1092EB0F1092EC0F04
:10BED0001092ED0F80E00E942FF8BB2019F081E056
:10BEE0000E942FF8AA2019F082E00E942FF80E94E9
:10BEF000D8F08091BC078093BD07892D0E94AE3495
:10BF00008091BF049091C004A091C104B091C2047B
:10BF10008093740290937502A0937602B093770297
:10BF20008091BD049091BE0490936F0280936E0245
:10BF300083E0809378020E9480F93ECE60E070E05A
:10BF400080E890E42BCFA3019201C701B6016ACF2C
:10BF500080910408813009F02FCE89E40E94453297
:10BF6000082F10E0882319F00E94C931182F8AE4A5
:10BF70000E944532F82E882339F00E94C931011100
:10BF800006C0853068F005C080E0002349F0153018
:10BF900028F08DE59FE00E94F2360ECEF110F1CF31
:10BFA00090E1E6EEFFE0A1E3B8E001900D929A95F2
:10BFB000E1F7002391F0B4E01B02F0011124E354F7
:10BFC000FA4E4081518162817381409331085093D0
:10BFD00032086093330870933408FF2091F024E016
:10BFE0008202F0011124E755FA4E80819181A281ED
:10BFF000B3818093350890933608A0933708B093A7
:10C00000380840E050E0BA0186E40E9460326B01DB
:10C010007C0120E030E0A9010F943C5918168CF403
:10C0200020E030E040E752E4C701B6010F94D65754
:10C0300069837A838B839C83CE0101960E94C8F723
:10C04000BBCD60E070E0CB01F3CF8FE0809363085D
:10C05000B3CD8091F004882381F1893009F0ACCD13
:10C060006BE9A62E62E0B62E76EEC72E7FE0D72EC5
:10C07000E12C00E010E0D5018D915D010E94453278
:10C08000F82E882361F0133011F4082FFE2C0E9443
:10C09000CD31F6016083718382839383EF2C1F5F20
:10C0A000F4E0CF0ED11C143031F7EE2009F457C064
:10C0B0000E94D8F00E9480F97FCD5BE9C52E52E046
:10C0C000D52EF12CE12C00E010E0D6018D916D0110
:10C0D0000E944532382E8823D9F10E94CD314B0180
:10C0E0005C01133059F0F701E45BF64F2081318198
:10C0F000428153810F94DB564B015C01F701EA51F9
:10C10000F04F2081318142815381C501B4010F94E8
:10C11000DB562B013C012DEB37E346E855EB0F9442
:10C120003C5987FD0AC02DEB37E346E855E3C301D0
:10C13000B2010F94EA4F18165CF41330C1F48092E8
:10C14000F20F9092F30FA092F40FB092F50F032D1F
:10C150001F5FB4E0EB0EF11C143009F0B6CF0023E2
:10C1600009F4A8CF82EF9FE00E9420EDA3CFF70152
:10C17000EE57F74F5F01A3019201608171818281C7
:10C1800093810F94DC56D5016D937D938D939C9391
:10C190001397812F0E94C8EEDBCF8091F10490911C
:10C1A000F2048837910511F40C94A26B08F07BC25D
:10C1B0008D34910509F4E6C708F0D3C08A319105A2
:10C1C00009F408C708F094C08431910509F44EC6FB
:10C1D00008F071C08131910509F40FC608F044C020
:10C1E000029708F0C2CC80E50E944532C12CD12CC8
:10C1F0007601882321F00E9476276B017C0183E57C
:10C200000E944532882361F00E94CD3120E030E069
:10C210004AE754E40F9450500F944F586B017C013F
:10C220000E94EADC8091F4049091F504009709F4EF
:10C23000DEC50F94D93F8091F1049091F2046EE72E
:10C240007FE0892B11F466E77FE030E020E049E4ED
:10C2500050E482E00E94133840E0C701B6010E941A
:10C260007E590F940B40A8CC429709F07ECC83E511
:10C270000E944532882311F40C94D96A0F946E32CF
:10C280006093410870934208809343089093440858
:10C290000E94CD3120E030E04AE754E40F94505042
:10C2A0000F944F5860931002709311028093120202
:10C2B0009093130281CC8731910509F40CC670F478
:10C2C0008531910509F403C6469709F04ECC80915B
:10C2D000DC1582FD71CC0F94313E6ECC8831910516
:10C2E00009F40EC6499709F040CC0E94645B64CC07
:10C2F0008F31910509F413C7D0F48C31910509F4FD
:10C30000D6C608F47AC68D31910509F4D8C64E9781
:10C3100009F02BCC8091DC1583FF4ECC0F94522971
:10C320008091F4049091F5040F94A83E45CC893493
:10C33000910509F413C750F48032910509F4C6C67B
:10C34000819709F012CC0E94604D36CC8B34910558
:10C3500009F414C78C34910509F007CC0E9407FD3D
:10C360002BCC8B36910511F40C94AD6908F00FC1FC
:10C370008435910509F47BCF40F58135910511F4A1
:10C380000C94B96A90F48E34910509F0EECB70E00C
:10C3900060E083E50E94AB338E34910509F0F7C667
:10C3A0000E9410DC0F940B4007CC8235910511F4EC
:10C3B0000C94D16A8335910509F0D7CB809163083D
:10C3C0008F7E806280936308F7CB8836910509F4ED
:10C3D00062C708F09CC08535910511F40C941C6B64
:10C3E0008C35910509F0C1CB0E94444887FDE4CB10
:10C3F0008091EC0484FD0AC08091EE0487FD06C0A4
:10C400008091EF04837011F40C944A6B2BE9C22ED7
:10C4100022E0D22E3DE9E32E3FE0F32E10E0D601DC
:10C420008D916D010E944532882309F466C0133056
:10C4300011F00C94416B0E94CD314B015C0120E066
:10C4400030E040EA51E40F94EA4F87FF4EC0A50167
:10C4500094016091BD0F7091BE0F8091BF0F9091BC
:10C46000C00F0F94D6572B013C01AC019B0160918A
:10C470006A0970916B0980916C0990916D090F9414
:10C48000505060936A0970936B0980936C09909384
:10C490006D09A30192016091CD0F7091CE0F809133
:10C4A000CF0F9091D00F0F9450506093CD0F709399
:10C4B000CE0F8093CF0F9093D00F60917A09709137
:10C4C0007B0980917C0990917D090F94EF4FA30126
:10C4D00092010F9450500F944F5860937A097093C3
:10C4E0007B0980937C0990937D098092BD0F909287
:10C4F000BE0FA092BF0FB092C00F1F5FF4E0EF0E0F
:10C50000F11C143009F08BCF0E94C6DC55CB893664
:10C51000910509F4F7C68A36910509F026CB80E526
:10C520000F948D2AF82E81E08F1508F445CB81E415
:10C530000E94F73160918609062F10E0811102C038
:10C540000FEF10E089E40E944532882311F40C9427
:10C5500031710E94A53190E01816190614F481E09B
:10C5600090E026E0289FF001299FF00D1124EB5F59
:10C57000F74F04811581EF2DF0E0EA57F64F0F3F9A
:10C58000110519F010F00FEF10E0008315CB813783
:10C59000910509F444C708F068C08E36910509F486
:10C5A000EAC608F059C08C36910509F405CB8D36E2
:10C5B000910509F0DACA80919C0F83FDFDCA0E94A3
:10C5C0004448F82E87FDF8CA89E40E944532882342
:10C5D00011F40C9420710E94A53190E018161906F0
:10C5E00014F481E090E026E0289FF001299FF00DEF
:10C5F0001124EB5FF74F8081918110E00E946CDC89
:10C6000061E081E00F941A4420911E1530911F15AE
:10C6100080911C1590911D15821793070CF069C627
:10C620008FE690E19F938F938AE790E19F938F939A
:10C630001F920E946EB30F900F900F900F900F906B
:10C6400001E00F94E343002309F4B6CA40E0612FF0
:10C650008F2D0F94EB09B0CA8F36910509F49EC651
:10C660008037910509F4A8CA80CA8537910511F46D
:10C670000C94576B60F48237910511F40C944F6B56
:10C680008337910509F071CA0E94193795CA863718
:10C69000910511F40C94696B8737910509F065CA0F
:10C6A0000E9466FA89CA8039E1E09E0711F40C9471
:10C6B000586E08F059C28D3C910511F40C94AC6C85
:10C6C00008F0A6C08B39910509F42CC740F58D37C9
:10C6D000910509F40ACE58F48937910509F045CA45
:10C6E0001092BD071092BC070E9489FA65CA8C3867
:10C6F000910509F4B3C68139910509F036CA70E095
:10C7000060E083E50E94AB33823010F40C94AA6B96
:10C710000E94574780ED90E10E94F2364DCA893C55
:10C72000910511F40C94176CB0F58E3B910509F44A
:10C73000BBC6883C910509F018CA0E944448182FCE
:10C7400087FD3ACA0091810884E40E944532F82EA0
:10C750008823C1F00E94CD314B015C0120E030E024
:10C76000A9010F94EA4F882311F40C94146C24E06F
:10C770001202F0011124E358F74F80829182A282C5
:10C78000B3820F2D602F83E50E94BA338093810816
:10C790000E94FCC411CA8B3C910511F40C94416CAD
:10C7A0008C3C910509F0E1C98091ED0487FF02C03E
:10C7B0000C94646C8091EE048E7011F00C94646C97
:10C7C0004091D10F5091D20F6091D30F7091D40F3F
:10C7D00085EF90E10E94E7384091D50F5091D60F38
:10C7E0006091D70F7091D80F82EF90E10E94E738E7
:10C7F0004091D90F5091DA0F6091DB0F7091DC0FEF
:10C8000082E79CE20E94E7388AE00E94B936D4C9E8
:10C81000823221E0920711F40C94946D08F09CC0D0
:10C82000833D910511F40C94336D08F050C0AEE8CF
:10C83000EA2EA8E0FA2E10E08E3C910509F095C989
:10C8400088E5810F0E94F731882351F00E94CD3195
:10C85000F7016083718382839383812F0E94C8EEE6
:10C860001F5FF4E0EF0EF11C133051F78091EE04DE
:10C8700087FD20CC8091EF04837009F01BCC4091A0
:10C880008E0850918F08609190087091910887E30D
:10C8900091E10E94E738409192085091930860918D
:10C8A00094087091950882ED90E40E94E7384091D9
:10C8B00096085091970860919808709199088FECAC
:10C8C00090E40E94E7388AE00E94B93675C98C3D31
:10C8D000910511F40C94376D8D3D910509F045C912
:10C8E0000E944448082F87FD67C983E50E944532AE
:10C8F000002E000C110B7801EE0CFF1C882311F4A4
:10C900000C947A6D0E94C931F701EB5CFD4F918365
:10C910008083000F111F000F111F980127583D4FF2
:10C920007901BC01990F880B990B0F94F14F2AE004
:10C9300037ED43E25CE30F94505009541A4FD8018D
:10C940002D913D914D915C910F945050F701608372
:10C9500071838283938330C98E32A1E09A0711F4E8
:10C960000C940E6E08F083C08C32E1E09E0711F447
:10C970000C94F06D8D32914009F0F7C885E40F9466
:10C980008D2A81110C94066E80E50E94F731882370
:10C9900051F00E94CD316093211570932215809340
:10C9A00023159093241589E40E94F731882381F0A0
:10C9B0000E94CD312CEA35EC47E25EE30F945050F3
:10C9C000609325157093261580932715909328154D
:10C9D00084E40E94F731882381F00E94CD312CEA53
:10C9E00035EC47E25EE30F94D657609329157093B8
:10C9F0002A1580932B1590932C150E944048409146
:10CA000021155091221560912315709124158FE501
:10CA100091E10E94E7382CEA35EC47E25EE3609151
:10CA200025157091261580912715909128150F9442
:10CA3000D657AB01BC018BE591E10E94E7382CEAA7
:10CA400035EC47E25EE36091291570912A158091DB
:10CA50002B1590912C150F945050AB01BC0187E51C
:10CA600091E10E94E7388AE00E94B936A5C88F326A
:10CA700021E0920711F40C94546E8033914009F038
:10CA800074C880E50E94F731882351F00E94CD31AF
:10CA90006093710870937208809373089093740880
:10CAA00089E40E94F731882381F00E94CD312CEA7D
:10CAB00035EC47E25EE30F94505060937508709335
:10CAC0007608809377089093780884E40E94F73181
:10CAD000882381F00E94CD312CEA35EC47E25EE3F9
:10CAE0000F94D6576093790870937A0880937B08E7
:10CAF00090937C080E9440484091710850917208C0
:10CB000060917308709174088DE791E10E94E73895
:10CB10002CEA35EC47E25EE3609175087091760887
:10CB200080917708909178080F94D657AB01BC019B
:10CB300089E791E10E94E7382CEA35EC47E25EE3B1
:10CB40006091790870917A0880917B0890917C08B7
:10CB50000F945050AB01BC0185E791E10E94E7388A
:10CB60008AE00E94B93628C8873FA1E09A0711F4ED
:10CB70000C946C6F08F0B8C0853AE1E09E0711F4A0
:10CB80000C94AF6EE8F48C3921E0920711F40C9408
:10CB90005C6E38F48A39914011F40C94DC5D0C948D
:10CBA000B55D8D39B1E09B0711F40C94E570843AC2
:10CBB000914011F00C94B55D0E9458490C94DC5DD5
:10CBC000843FF1E09F0711F40C94646F08F07DC07E
:10CBD0008C3A31E0930711F40C94B36E863E914089
:10CBE00011F00C94B55D84E50E94F7318823A1F023
:10CBF0001092000510920105109202051092030593
:10CC0000109204058FEF0E94D82561E070E084E562
:10CC10000E94AB338093040583E50E94F73188239B
:10CC200021F00E94C9310E94D82583E40E94F73187
:10CC3000882331F080912302803210F40E947234F4
:10CC400080E50E94F731882331F00E94C93180329B
:10CC500010F40E94723485E50E94F731882311F4A4
:10CC60000C94DC5D0E94C931803210F00C94DC5DC4
:10CC700041E050E060E070E0082E04C0440F551F12
:10CC8000661F771F0A94D2F740955095609570956E
:10CC900000910005109101052091020530910305D6
:10CCA00040235123622373234093000550930105D1
:10CCB00060930205709303059091230289130C94ED
:10CCC000DC5D10929B0F0C94DC5D853FB1E09B070F
:10CCD00011F40C94686F863F914011F00C94B55D8F
:10CCE0000E9494FA0C94DC5D8E3BF2E09F0711F4F5
:10CCF0000C94147060F5883532E0930711F40C94AD
:10CD0000906FB0F4883FB1E09B0711F40C94756FFD
:10CD10008C30924011F00C94B55D8091DC1582FD51
:10CD200002C00C94886F80648093DC150C94DC5DE9
:10CD30008B35F2E09F0711F40C94946F8D3B924079
:10CD400011F00C94B55D0E94C4550C94DC5D873ED7
:10CD500033E0930711F40C94D570C8F48C36B3E02B
:10CD60009B0711F40C94DC5D803A934011F00C9415
:10CD7000B55D2091F4043091F5049091DC1592603A
:10CD80009093DC15C9010F9482400C94DC5D883EC1
:10CD9000F3E09F0711F40C94FE70893E934011F06C
:10CDA0000C94B55D0F94523F81110C94DC5D0E9490
:10CDB000CF330F94103F0E940DFC6D337105810538
:10CDC000910520F089E592E10E94857185E592E167
:10CDD0000E94857184EE8093FE0481E492E10E94BA
:10CDE000F2368DE392E10E9485710C94DC5D60E087
:10CDF00086E89FE00E9489B31ECA8091EC0484FDFE
:10CE000017C08091EE0487FD13C08091EF048370FA
:10CE100079F460E089E99FE00E9489B35F988A987D
:10CE20008091080181708093060112980C94DC5D5A
:10CE300088E50E94F73181115F9889E50E94F731FA
:10CE400081118A988AE50E94F731882329F0809120
:10CE5000080181708093060185E40E94F7318823E0
:10CE600011F40C94DC5D12980C94DC5D8091DC155F
:10CE700083FF25C081EB9FE00E94F2368091DC1594
:10CE800083FF17C08BEF95E10E941ED38BE1EBEF80
:10CE9000F5E1DE01119601900D928A95E1F770E0BF
:10CEA00060E0CE0101960F946806CE0101960E94C3
:10CEB000F73382EA9FE00E94F2360C94DC5D0E9418
:10CEC000404882EC9FE00E94F2360C94DC5D0F94A7
:10CED000423E0C94DC5D8091F4049091F504FC01D9
:10CEE0002191222331F02032D9F7DF0111971C92D2
:10CEF000F7CF60E00F94CB401092FE040C94DC5D01
:10CF000083E50E944532882321F00E9497270E94E2
:10CF1000CA2584E50E9445328823A9F00E949727FC
:10CF20006B017C010E94B4FCC092BB05D092BC0591
:10CF3000E092BD05F092BE05CD28CE28CF2819F08D
:10CF400081E08093620880912B078823F9F080E0CC
:10CF500090E0A0EAB1E489839A83AB83BC831C8E02
:10CF60001D8E1E8E1F8E18A219A21AA21BA210E0DF
:10CF700000E020E0AE014F5F5F4FBE01645E7F4F77
:10CF8000CE0180960E94BD560C94DC5D0E943D3619
:10CF9000882381F00F94CB3D0E94613688ED98E0A4
:10CFA0000F94733D1092DF101092E0101092E11078
:10CFB0001092E21061E084E09EE10E94BA374CECEE
:10CFC0005DE16CEC7FE085E00F94842A0F940B40C8
:10CFD0000C94DC5D8091DC1583FD02C00C94DC5D5B
:10CFE00083E50E944532882311F40C94DC5D0E9495
:10CFF00097270E94CA250C94DC5D83E40E94F731D8
:10D00000882361F182EE9FE00E94F2368091421700
:10D010008823F9F0BE016F5F7F4F8FE397E10E9495
:10D02000E4D2CE0101960E9423CFCE0101960F9447
:10D03000AB3F80916A12882339F080E20E94B936B2
:10D040008AE692E10E9423CF8AE00E94B9360C94CE
:10D05000DC5D88ED9FE00E94F236F6CF83E50E940A
:10D060004532882301F10E94A531182F8C3308F036
:10D070008CE38093C7040F946E326B017C01212FE7
:10D0800030E0A8EEB3E00F948256C60ED71EE81E1D
:10D09000F91EC092C304D092C404E092C504F09279
:10D0A000C6040C94DC5D0F943A3D0C94DC5D8091D9
:10D0B000F4049091F5040F9482400C94DC5D80910F
:10D0C000DC158E7F8093DC150C94DC5D8091DC1583
:10D0D00082FD0E94EADC8091DC1583FD02C00C9485
:10D0E000DC5D60E080E50E94BA33182F682F8091E4
:10D0F000F4049091F5040F94CB4083E50E944532EF
:10D10000882321F00E9497270E94CA250F94CB3DC7
:10D1100011110C94DC5D0E9461360C94DC5D0E9460
:10D120000DFC6C8F7D8F8E8F9F8FBE016F5F7F4F49
:10D13000CE014C960E942B2CCE0101960F94D93F24
:10D140000E944048BE016F5F7F4F81EF9FE00E94C9
:10D15000564D8AE00E94B9360C94DC5D80E50E9451
:10D16000F731882311F40C94DC5D0E94A5318536DB
:10D1700008F084E68093FE040C94DC5D0E94613626
:10D180000C94DC5D81E00E943FFC0C94DC5D8CE53E
:10D1900090E10E94F2366091AC077091AD0783E593
:10D1A00090E10E94D5386091AE077091AF0786E498
:10D1B00090E10E94D5386091AC077091AD078091E5
:10D1C000AE079091AF07681B790B80916208815080
:10D1D00021E030E0823010F030E020E0621B730B81
:10D1E0008BE390E10E94D5388AE00E94B93683E350
:10D1F00090E10E94F2368091B0079091B107A09122
:10D20000B207B091B3078C8F9D8FAE8FBF8FBE01D9
:10D210006F5F7F4FCE014C960E942B2CBE016F5F3B
:10D220007F4F86E290E10E94564D8091B407909125
:10D23000B507A091B607B091B7078C8F9D8FAE8FC1
:10D24000BF8FBE016F5F7F4FCE014C960E942B2C8B
:10D25000BE016F5F7F4F86E190E10E94564D20E056
:10D2600030E04AE754E46091B8077091B9078091C3
:10D27000BA079091BB070F94D657AB01BC018EEF54
:10D280009FE00E94E7388DE60E94B9368AE00E944E
:10D29000B9360C94DC5D80919C0F83FF02C00C9426
:10D2A000DC5D0E94444887FF02C00C94DC5D89E489
:10D2B0000E944532882309F4BAC70E94A53190E044
:10D2C0001816190614F481E090E026E0289FF0017A
:10D2D000299FF00D1124EB5FF74F808191810E940F
:10D2E0006CDC61E080E00F941A440F94E3430C94EB
:10D2F000DC5D84E690E1112309F494C9012FA1C9F2
:10D30000182F9FC90E944448182F87FD0AC08FE735
:10D3100090E10E94F236812F0F94F3078AE00E9479
:10D32000B93638A930934D08E1960FB6F894DEBFB0
:10D330000FBECDBFDF91CF911F910F91FF90EF9066
:10D34000DF90CF90BF90AF909F908F907F906F9025
:10D350005F904F903F902F90089580E50F948D2A15
:10D36000823010F00C94DC5DE82FF0E0EA57F64FC5
:10D3700010820C94DC5D8EE40E944532882311F407
:10D380000C94DC5D0E94972760937810709379105D
:10D3900080937A1090937B100C94DC5D83E50E945F
:10D3A000F731882329F083E50F948D2A80939C0F11
:10D3B0000E94404880E990E10E94F23680919C0FE3
:10D3C000882351F110E000E020E080919C0F90E074
:10D3D000B0E0A0E0002E04C0B695A795979587957C
:10D3E0000A94D2F780FF12C0FF24F394F20E222396
:10D3F00019F08CE20E94B936F801EE0FFF1FEA57D0
:10D40000FF4E859194910E94F2362F2D0F5F1F4F92
:10D4100005301105D1F618CE82E890E11CCE83E5E7
:10D420000E944532882369F00E94A5318D3320F493
:10D4300080930F020C94DC5D8CE380930F020C94BC
:10D44000DC5D0E94404860910F0287E990E10E94F4
:10D45000DF388AE00E94B9360C94DC5D80919C0F25
:10D4600083FF02C00C94DC5D89E40E94453288236E
:10D4700009F403C70E94A53190E01816190614F4A8
:10D4800081E090E026E0289FF001299FF00D112413
:10D49000EB5FF74F828193810E949A3161E080E0D7
:10D4A0000F941A440C94DC5D80919C0F83FF02C0A2
:10D4B0000C94DC5D89E40E944532882309F4E7C6B8
:10D4C0000E94A53190E01816190614F481E090E04E
:10D4D00026E0289FF001299FF00D1124EB5FF74F04
:10D4E0008281938110E00E949A3160E081E00F9484
:10D4F0001A4420916E0830916F0880916C089091C9
:10D500006D08821793071CF48DEA90E102C08EE942
:10D5100090E160E00E9489B360E0812F0F9466087B
:10D520000C94DC5D83E50E944532882311F40C9451
:10D53000DC5D0E94A531182F8C3308F08CE38093BA
:10D54000CC040F946E326B017C01212F30E0A8EEE9
:10D55000B3E00F948256C60ED71EE81EF91EC09285
:10D56000C804D092C904E092CA04F092CB040C948F
:10D57000DC5D0E943BD50E94FBDC81E00E943FFC09
:10D580000E94743668EE73E080E090E00E94EE3511
:10D590000E94392260E08CEB90E10E9489B30C94E8
:10D5A000DC5D809163088F7D8061809363080C94BB
:10D5B000DC5D8091EC0484FD0CC08091EE0487FD5D
:10D5C00008C08091EF04837021F40E94FBDC0C946E
:10D5D000DC5D0E94EADC88E50E94F731882331F0A7
:10D5E0005F9A8091BF078E7F8093BF0789E50E9475
:10D5F000F731882331F08A9A8091BF078D7F80931D
:10D60000BF078AE50E94F731882359F0809108010D
:10D6100080958170809306018091BF078B7F8093F6
:10D62000BF0785E40E94F731882311F40C94DC5D78
:10D630000E9437220C94DC5D83E50E94F731882339
:10D6400011F40C94DC5D0F946E326093410870937A
:10D65000420880934308909344080E94CD3120E013
:10D6600030E04AE754E40F9450500F944F586093C1
:10D67000CD047093CE048093CF049093D0040C9487
:10D68000DC5D0E94CD31F701648B758B868B978BA7
:10D690000C947D6281E00F9417290C94DC5D0F944B
:10D6A000B22884E495E10E9408D80C94DC5D809156
:10D6B000F4049091F504009741F0DC012C912223B1
:10D6C00021F00F94D93F0C94DC5D0F940B400C9427
:10D6D000DC5D0091F4041091F50494E0F12C40E03D
:10D6E0009150F9F0F8018081282F2B7F213499F493
:10D6F00021812133B1F4813411F1853409F441E001
:10D7000098012E5F3F4F89012F5F3F4FF8018081C5
:10D710008032C9F3E5CF803521F4818180538A308E
:10D7200078F341110E944048FF2021F08DEC90E1F8
:10D730000E94F236C8010E94C0360C94DC5DFF24C2
:10D74000F394DECF1093BD071093BC070E9489FAB3
:10D750000C94DC5D8C01112788E40E9445328823FB
:10D76000C1F00E94C9318A3A91050CF44BC00E9465
:10D77000C931843B91400CF048C00E94C93126E079
:10D78000209FF001219FF00D1124EB5FF74F918353
:10D79000808382E40E9445328823A9F00E94C93127
:10D7A0000597B4F10E94C9318D389105A4F50E9406
:10D7B000C93126E0209FF001219FF00D1124EB5F7D
:10D7C000F74F9383828386E40E944532882311F4C5
:10D7D0000C94DC5D0E94C93197FD20C00E94C931C4
:10D7E0008F3F910509F0ECF40E94C93126E0209F9B
:10D7F000F001219FF00D1124EB5FF74F9583848397
:10D800000C94DC5D8AEA90E0BACF83EB91E0B7CF6D
:10D8100085E090E0CECF8CE890E0CBCF90E080E048
:10D82000E5CF8FEF90E0E2CF80E00C94C6630E94DA
:10D83000444887FF02C00C94DC5D0BE912E08DE9DF
:10D84000E82E8FE0F82E9FE9C92E92E0D92ED8015C
:10D850008D918D010E94F731882359F00E94CD31BE
:10D860000F944F58F70160837183828393830E94E2
:10D8700078DCF4E0EF0EF11CC016D10641F70C94F1
:10D88000DC5D0E94444887FF02C00C94DC5DBBE96C
:10D89000EB2EB2E0FB2E10E000E0D7018D917D0170
:10D8A0000E94F731882349F00E94CD31F801E356F8
:10D8B000F04F64A375A386A397A30C5F1F4F00319D
:10D8C000110559F70C94DC5D83E50E9445328823ED
:10D8D00091F00E94CD316093D10F7093D20F80935D
:10D8E000D30F9093D40F6093D90F7093DA0F809376
:10D8F000DB0F9093DC0F80E50E944532882351F0C6
:10D900000E94CD316093D10F7093D20F8093D30FCB
:10D910009093D40F82E50E944532882351F00E94F3
:10D92000CD316093D50F7093D60F8093D70F90931E
:10D93000D80F84E50E944532882311F40C94DC5DF5
:10D940000E94CD316093D90F7093DA0F8093DB0F73
:10D950009093DC0F0C94DC5D8091EC04827151F4A7
:10D960008091EE048C7831F48091EF04837011F48F
:10D970000C94DC5D82E40E94F731882351F00E9410
:10D9800076276093AD0F7093AE0F8093AF0F909397
:10D99000B00F83E50E94F731882351F00E94CD310A
:10D9A0006093DD0F7093DE0F8093DF0F9093E00F95
:10D9B00084E50E94F731882351F00E94CD316093B5
:10D9C000E10F7093E20F8093E30F9093E40F88E5EB
:10D9D0000E94F731882351F00E94CD3160935E0997
:10D9E00070935F09809360099093610989E50E94B3
:10D9F000F731882351F00E94CD3160936209709312
:10DA0000630980936409909365098AE50E94F73160
:10DA10008823B1F00E94CD31609366097093670945
:10DA200080936809909369092DEC3CEC4CEC5DE324
:10DA30000F94EA4F181624F085E091E10E94F23627
:10DA400085E40E94F731882311F40C94DC5D0E9478
:10DA5000CD3160936A0970936B0980936C09909340
:10DA60006D090C94DC5D0E9469480C94DC5D82E4D5
:10DA70000E94F731882341F080916E0290916F02ED
:10DA8000909315028093140282E50E94F731882357
:10DA900041F0809114029091150290936F0280934F
:10DAA0006E0283E50E944532882331F00E94C9311D
:10DAB00090936F0280936E028091EC049091ED043C
:10DAC000A091EE04B091EF04892B8A2B8B2B11F0DF
:10DAD0000C94DC5D60916E0270916F028EE391E1B7
:10DAE0000E94FD3D85E20E94B9368AE00E94B93667
:10DAF0000C94DC5D0E94404885E40E94B93680E3C6
:10DB0000800F0E94B936F701EB5CFD4F6081718197
:10DB100082E491E10E94FD3D85E20E94B9368AE0EF
:10DB20000E94B9360C94DC5D8AE50E944532882358
:10DB300031F10E94CD3120E030E040E050EC0F9414
:10DB4000EA4F87FD3CC00E94CD3120E030E040E04C
:10DB500050E40F943C591816BCF10E94CD3120912D
:10DB6000B90F3091BA0F4091BB0F5091BC0F0F9479
:10DB700050500F944858CB010F94223305C083E5D1
:10DB80000E9445328111D5CF8091EE0487FD21C0DE
:10DB90008091EF048370E9F40E9440484091300680
:10DBA0005091310660913206709133068AE491E11A
:10DBB0000E94E7388AE00E94B9360C94DC5D60E090
:10DBC00070E080E090ECCBCF60E070E080E090E42B
:10DBD000C6CF82E50E94F7318111DECF0C94DC5D67
:10DBE00064E071E083E50E9452328C0168EE73E0DC
:10DBF00080E50E9452328938F3E19F0710F088E8EF
:10DC000093E1B8010E94747E0C94DC5D0E9457473A
:10DC100083E691E10E94F2360C94DC5D83E50E947C
:10DC2000F731182F882369F00E94C9319C01909325
:10DC30007E0280937D0291E0232B09F090E0909387
:10DC4000980980E50E94F731882361F020917D02D8
:10DC500030917E02232B11F00E94B93180939809F4
:10DC60000C94DC5D11110C94DC5D0E9440488DE940
:10DC700091E10E94F23680919809882391F085E81D
:10DC800091E10E94F23660917D0270917E028CE8F3
:10DC900091E10E94FD3D88E891E10E94F2360C94EA
:10DCA000DC5D81E891E1EDCF0E9409390C94DC5DE7
:10DCB0000E94EADC0C94DC5D8091EC048878F9F435
:10DCC0008091EE048670D9F40E94404880ED91E185
:10DCD0000E94F236809155020E94C938409151024B
:10DCE00050915202609153027091540280EB91E185
:10DCF0000E94E7388AE00E94B9360C94DC5D88E423
:10DD00000E94F731882321F00E94B9318093D10419
:10DD100082E50E94F731082F83E50E94F731182F22
:10DD2000011102C0882341F00E942422112321F016
:10DD30000E94B9318093550284E40E94F731882310
:10DD400011F40C94DC5D0E94CD316093510270930C
:10DD5000520280935302909354020C94DC5D0E9413
:10DD60005B470C94DC5D0F942D4081110C94DC5DBD
:10DD700070E9C72E77E2D72E26EE3FE03DA32CA315
:10DD8000CE0101961C017C0110E000E0F6016591D6
:10DD9000759185919491ACA1BDA18D909D90AD9010
:10DDA000BD90BDA3ACA3A50194010F94DB562B013C
:10DDB0003C01F701408251826282738220E030E0B0
:10DDC00040EA51EC0F943C5987FD0AC020E030E056
:10DDD00040EA51E4C301B2010F94EA4F181684F4EB
:10DDE000F801ED5FFF4BE4911E1654F4B7FAB094BE
:10DDF000B7F8B094D7018D929D92AD92BC921397D3
:10DE0000F70181909190A190B1907F0120E030E0E6
:10DE100040EA51ECC501B4010F943C5987FD3FC065
:10DE200020E030E040EA51E4C501B4010F94EA4F2C
:10DE30001816ACF10F5F1F4FF4E0CF0ED11C03306A
:10DE4000110509F0A3CF6EE8E62E68E0F62E10E08B
:10DE5000F10181919191A191B1911F01F7018193FC
:10DE60009193A193B1937F01812F0E94C8EE1F5F10
:10DE7000133071F70E9480F960E081EE91E10E9419
:10DE800089B363E972E084E690E00E94747E6AEBF5
:10DE900072E084E690E00E94747E0C94DC5D0E9447
:10DEA00057478FEF91E10E94F23661E081EF91E1F7
:10DEB0000E9489B30E94E08468E270E088EC90E000
:10DEC0000E94747E0C94DC5D0E94BAD80C94DC5DD8
:10DED0000F9495120C94DC5D61E083E50E94BA33E7
:10DEE00081270F94790B0C94DC5D81E080933406DC
:10DEF0000F94891210923406882311F40C94DC5D7F
:10DF00000E9440488DE192E10E94F2360C94DC5D63
:10DF100083FD02C00C94DC5D0F9452290C94DC5DEF
:10DF20000E94545A0C94DC5D0E944448082F87FFDD
:10DF300002C00C94DC5D85E50E94F731882359F11D
:10DF40000E94CD314B015C01E02E002E000CFF0839
:10DF500020E030E0A9010F943C5987FF04C0B7FAD4
:10DF6000B094B7F8B09420E030E84BE354E4C50136
:10DF7000B4010F943C59970153E0220F331F5A9577
:10DF8000E1F72D533A4F1816D4F1D9018D929D9295
:10DF9000AD92BC9213978CE40E94F731882311F460
:10DFA0000C94DC5D0E94CD316B017C01002E000CD5
:10DFB000110B20E030E0A9010F943C5987FF04C009
:10DFC000F7FAF094F7F8F09420E030E84BE354E4EB
:10DFD000C701B6010F943C59980143E0220F331F4B
:10DFE0004A95E1F72D533A4F18169CF0D901149633
:10DFF000CD92DD92ED92FC9217970C94DC5D80E05F
:10E0000090E8ABE3B4E4F90180839183A283B38306
:10E01000C2CF80E090E8ABE3B4E4F9018483958358
:10E02000A683B7830C94DC5D0E944448182F87FFB9
:10E0300002C00C94DC5D8AE50E944532812C912C53
:10E0400090E2A92E91E4B92E882341F040E050E0FF
:10E05000BA018AE50E9460324B015C01412F64E005
:10E0600083E00E94C98520E030E0A901C501B40128
:10E070000F943C5918167CF580E090E0A0EAB0E4DB
:10E0800089839A83AB83BC832091EE0F3091EF0F8D
:10E090004091F00F5091F10FC501B4010F94DC567F
:10E0A0006B017C0120E030E048EC53E40F94EA4F30
:10E0B00087FD06C0C12CD12C88ECE82E83E4F82E15
:10E0C000CC8EDD8EEE8EFF8EBE016F5F7F4FCE0158
:10E0D0004C960E9489F085E50E94F731882309F467
:10E0E00059C00E94CD316B017C0120E030E0A901D4
:10E0F000C701B6010F943C5987FF04C0F7FAF094AA
:10E10000F7F8F094F7FAF094F7F8F094C982DA820D
:10E11000EB82FC8244E061E0CE0101960E942B5824
:10E1200020E030E0A901C501B4010F943C59181654
:10E130005CF580E090E0A0EAB0E489839A83AB8349
:10E14000BC83A50194016091EE0F7091EF0F809157
:10E15000F00F9091F10F0F94DB566B017C0120E0E2
:10E1600030E0A9010F943C5918161CF0C12CD12C99
:10E170007601CC8EDD8EEE8EFF8EBE016F5F7F4FFF
:10E18000CE014C960E9489F0109206050E94E08410
:10E190000C94DC5D28E01202F0011124ED53FA4FDB
:10E1A000C080D180E280F380A0CF81E0809304081A
:10E1B0001092021360E083E50E94BA3381110C943F
:10E1C000DC5D0F9459270C94DC5D83E50E94F731E8
:10E1D000882341F00E94B9318093CB050E94D73348
:10E1E0000C94DC5D0E94404888E292E10E94F23685
:10E1F0008091CB050E94C9380C94DC5D0E94F771B8
:10E200000C94DC5D1091F1040F946E326093410820
:10E21000709342088093430890934408112311F4AB
:10E220000C94DC5D812F0E94F1D40C94DC5D83E5BD
:10E230000E944532882309F458C80E94C9314FC84A
:10E2400083E50E944532182F811107C082E50E94A4
:10E250004532082F882309F453C80E94C9310C9411
:10E26000FE6283E50E944532882311F40C94BB6260
:10E270000E9497278B010C94BB6283E50E94453274
:10E28000882311F40C94DC5D0E94C93105C983E533
:10E290000E944532182F811107C082E50E94453245
:10E2A000882311F40C94DC5D0E94C9311CC9DF92F3
:10E2B000EF92FF920F931F93CF93DF93EC01E090C7
:10E2C0004F08F09050088AE0D82E6AE070E0CE0146
:10E2D0000F94315A8C01009711F0FC011082CE018D
:10E2E0000E940A2D81E00E94445C0115110519F07D
:10E2F000E801D992EACFC701DF91CF911F910F9129
:10E30000FF90EF90DF900C940A2D4F925F926F92E6
:10E310007F928F929F92AF92BF92CF92DF92EF92B5
:10E32000FF920F931F93CF93DF93CDB7DEB77C019E
:10E330004DB65EB660904F08709050088DB69EB690
:10E340006AE070E0C7010F94254F6C018C010E1933
:10E350001F09892B21F4C7010F94374F8C01C80185
:10E3600001962DB73EB7281B390B0FB6F8943EBF68
:10E370000FBE2DBF8DB79EB701965C01A801B701F6
:10E380000F94584FF501E00FF11F1082C5010E9454
:10E390000A2D81E00E94445CC114D10451F0760141
:10E3A0009FEFE91AF90A0FB6F8949EBE0FBE8DBE14
:10E3B000C5CF0FB6F8949EBE0FBE8DBEC3010E949E
:10E3C0000A2D0FB6F8945EBE0FBE4DBEDF91CF9101
:10E3D0001F910F91FF90EF90DF90CF90BF90AF9083
:10E3E0009F908F907F906F905F904F9008954F9285
:10E3F0005F926F927F928F929F92AF92BF92CF92D5
:10E40000DF92EF92FF920F931F93CF93DF93CDB7DD
:10E41000DEB7C059D1090FB6F894DEBF0FBECDBF2D
:10E420000E94E533882369F083E50E94F731882351
:10E4300001F120E040E070E060E08AE095E80E94B1
:10E440007A81C057DF4F0FB6F894DEBF0FBECDBF45
:10E45000DF91CF911F910F91FF90EF90DF90CF90C0
:10E46000BF90AF909F908F907F906F905F904F90F4
:10E47000089583E40E94F731882319F00E94FF84F5
:10E48000E0CF8090410990904209A0904309B0905C
:10E49000440980914A0980FF05C090919C0F9860C3
:10E4A00090939C0F869581708093980980E29FE0FD
:10E4B0000E9485718091D0089091D1089E012F5FB4
:10E4C0003F4F7901009799F09F938F9387E19FE0E9
:10E4D0009F938F933F932F930F94814FC7010E9477
:10E4E00057710F900F900F900F900F900F90809199
:10E4F000CE089091CF08009799F09F938F938EE06C
:10E500009FE09F938F93FF92EF920F94814FC701EB
:10E510000E9457710F900F900F900F900F900F90D7
:10E520006E0131E8C30ED11C6091AD087091AE0848
:10E530008091AF089091B008860123E041E00F94EC
:10E54000B74A9F938F938CEF9EE09F938F93FF9298
:10E55000EF920F94814FC7010E94577184EF9EE0A4
:10E560000E94857187E08093BF078093AE050F906E
:10E570000F900F900F900F900F908091C9088823F3
:10E58000F9F06091CA087091CB088091CC08909105
:10E59000CD0823E041E00F94B74A9F938F938BEE11
:10E5A0009EE09F938F93FF92EF920F94814FC7014C
:10E5B0000E9457710F900F900F900F900F900F9037
:10E5C0008091D2088823A1F01F928F931F921F92EF
:10E5D0008EED9EE09F938F93FF92EF920F94814F69
:10E5E000C7010E9457710FB6F894DEBF0FBECDBFB2
:10E5F0008091D3088823A9F01F928F931F9281E006
:10E600008F938EED9EE09F938F93FF92EF920F94E6
:10E61000814FC7010E9457710FB6F894DEBF0FBE3D
:10E62000CDBF4090D4085090D5086090D608709027
:10E63000D70820E030E0A901C301B2010F94EA4FEE
:10E64000811104C080914A0982FF20C0860121E027
:10E6500041E0C301B2010F94B74A9F938F93809119
:10E660004A0982FB882780F91F928F9381ED9EE0F3
:10E670009F938F93FF92EF920F94814FC7010E9457
:10E6800057710FB6F894DEBF0FBECDBF60919F08E3
:10E690007091A0088091A1089091A2088E010F5856
:10E6A0001F4F23E041E00F94B74A782E692E609106
:10E6B0009B0870919C0880919D0890919E0886010E
:10E6C00023E041E00F94B74A6F927F929F938F931C
:10E6D00080EC9EE09F938F93FF92EF920F94814F77
:10E6E000C7010E9457716091A3087091A40880919E
:10E6F000A5089091A60823E041E00F94B74A85EB66
:10E700009EE00E948571DF92CF928BEA9EE09F93FC
:10E710008F93FF92EF920F94814FC7010E94577120
:10E720008091AC088F938091AB088F9384EA9EE030
:10E730009F938F93FF92EF920F94814FC7010E9496
:10E7400057716091A7087091A8088091A9089091CD
:10E75000AA0823E041E00F94B74A9F938F938AE978
:10E760009EE09F938F93FF92EF920F94814FC7018A
:10E770000E9457718CE0E1EBF8E0AEE8B8E0019060
:10E780000D928A95E1F78CE0EDEBF8E0A2E8B8E0B5
:10E7900001900D928A95E1F780E00E94C8EE81E039
:10E7A0000E94C8EE82E00E94C8EE809149098093E1
:10E7B000630881E08093CB050E94D73388ED98E011
:10E7C0009F938F938CEB97E39F938F93FF92EF929E
:10E7D0000F94814F0FB6F894DEBF0FBECDBFC701B7
:10E7E0000E945771809148098F93809147098F93B8
:10E7F000809146098F93809145098F93BF92AF9284
:10E800009F928F928CE89EE09F938F93FF92EF925E
:10E810000F94814FC7010E9457710FB6F894DEBF65
:10E820000FBECDBF0ECE4F925F926F927F928F92AE
:10E830009F92AF92BF92CF92DF92EF92FF920F938F
:10E840001F93CF93DF9300D000D01F921F92CDB7BC
:10E85000DEB783E50F948D2A863028F083E19EE0B1
:10E860000E94F2363FC0833009F464C1B0F48130B5
:10E8700021F1823009F450C080E09EE00E94F2361F
:10E880000E94A9358823A1F08091E50F0E94C93824
:10E890000E944A380E9480F925C0843009F490C152
:10E8A000853051F780E00E94AE340E949E34F2CF52
:10E8B00082EF9DE00E94F236EDCF0E949E341092CE
:10E8C0000E0210920D028091FF04811125C08EE48A
:10E8D0000E94F73181111DC080EE9DE09093C20728
:10E8E0008093C10728960FB6F894DEBF0FBECDBF48
:10E8F000DF91CF911F910F91FF90EF90DF90CF901C
:10E90000BF90AF909F908F907F906F905F904F904F
:10E91000089586EE9DE0E2CF80910D0290910E0267
:10E9200097FF03C087EB9DE09BCF009709F0A8C03D
:10E930001D821E821F8218868DEC9CECACE4BEE327
:10E9400089839A83AB83BC83BE016B5F7F4FCE010B
:10E9500001960E9489F080910D0290910E028931FA
:10E9600091050CF0B3C021E0209338029C012F5F89
:10E970003F4F30930E0220930D0265E00F949D5699
:10E9800080FF03C024E0291B922F24E09202F001B3
:10E990001124E354FA4E80809180A280B38094E0E9
:10E9A0008902F0011124E755FA4E408051806280BF
:10E9B00073808DEC9CECACE4BEE38D839E83AF83CF
:10E9C000B88719821A821B821C82CE0101966C01C3
:10E9D000E12CF12C00EA10E4A3019201C501B4017D
:10E9E0000E94D1EF19821A821B821C82B601CE01CD
:10E9F00005960E9489F08092E60F9092E70FA09210
:10EA0000E80FB092E90F4092EA0F5092EB0F60923C
:10EA1000EC0F7092ED0F1092FF0400910D02109117
:10EA20000E0289E1E82EF12C093111050CF4780170
:10EA3000B70180E59DE00E94FD3D69E170E08BE457
:10EA40009DE00E94FD3D8AE00E94B9361016110635
:10EA50000CF020CF1F9289E18F93FF92EF9284E315
:10EA60009DE09F938F9382E49DE09F938F931F92ED
:10EA70000E946EB30FB6F894DEBF0FBECDBF0ACFB3
:10EA8000815065E00F949D5680FF03C024E0291B50
:10EA9000922F25E09202F0011124E80FF11D87FD6D
:10EAA000FA95EE0FFF1FEE0FFF1FE453FA4F809110
:10EAB000EE0F9091EF0FA091F00FB091F10F8083C6
:10EAC0009183A283B3831092380245CF80E090E017
:10EAD000A0EAB0E48093EE0F9093EF0FA093F00FB5
:10EAE000B093F10F84E792E00E94B6EF0E94EADC57
:10EAF0008FEF9FEF90930E0280930D0283EA9DE0CB
:10EB00000E94F23681E99DE00F94D93F63E972E0FB
:10EB100084E690E00E94747E6AEB72E084E690E006
:10EB20000E94747E8BE89DE00E94857181E00E94C6
:10EB3000AE3471CF89E40E944532882371F00E947F
:10EB4000C931182F853068F064E070E088E79DE0F7
:10EB50000E94FD3D85E79DE083CE8AE40E94B437A4
:10EB6000C1CE8AE40E9445328823B9F30E94C9319C
:10EB7000082F853048F064E070E082E69DE00E9456
:10EB8000FD3D8FE59DE06CCE8AE50E9445328823ED
:10EB9000A9F00E94CD3125E01202F0011124E00F0E
:10EBA000F11D07FDFA95EE0FFF1FEE0FFF1FE45357
:10EBB000FA4F60837183828393836CCE8AE5CECFD4
:10EBC0008AE50E9445328823C9F30E94CD316093C3
:10EBD00030067093310680933206909333065ACEF6
:10EBE000CF93DF93C091E410C0935D0981E6C89F85
:10EBF000E0011124CA51DF4E80919C0F80FF05C0B7
:10EC00000E944048CE010E94C036CE010E940A2DCB
:10EC100080E0DF91CF910C94445C6091350270915B
:10EC20003602072E000C880B990B0F94F14F2AE047
:10EC300037ED43E25CE30F9450502091B7053091DB
:10EC4000B8054091B9055091BA050F9450506093A2
:10EC5000790270937A0280937B0290937C020895EC
:10EC6000E0912C08E23030F4F0E0EA57F64F809162
:10EC70002208808308958091D1158823C1F08150A6
:10EC80008093D115EBEFF5E1882351F08150990B7A
:10EC90002BE1289FF001299FF00D1124EF5CF94E24
:10ECA0008BE1A6E1B6E101900D928A95E1F7209102
:10ECB000D115211105C08091DC1580628093DC158F
:10ECC00081E090E0A0E0B0E0211103C080E090E09E
:10ECD000DC0180931A0890931B08A0931C08B09342
:10ECE0001D0810921F0881E08093190883E080932B
:10ECF00078020895CF93DF93EC01CB01BA010F9412
:10ED0000F14F29EC38EC48EC5EE30F94D65720E045
:10ED100030E040E05FE30F94DC560F944F58688377
:10ED2000DF91CF910895E0912C0886E0E802F00190
:10ED30001124EB5FF74F8091220890E09583848344
:10ED40000895CF93DF93EC01CB01BA010F94F14FFB
:10ED500020E030E0A9010F94DC560F944F586883EF
:10ED6000DF91CF9108958F929F92AF92BF92CF92F1
:10ED7000DF92EF92FF92CF936B017C0120E030E0B5
:10ED8000A9010F94EA4F87FD9FC06DEB77E386E002
:10ED900095E3A70196010F94DC566B017C0120E0FE
:10EDA00030E040E251E40F94505020E030E048EC75
:10EDB00052E40F9450504B015C0120E030E0A90177
:10EDC000C701B6010F94EA4F20E030E040EA50E47A
:10EDD00087FF04C020E030E040EA50ECC501B401F8
:10EDE0000F94DC5620E030E040E251E40F94D65717
:10EDF0000F9448586B017C018BE2F7FE09C0F09438
:10EE0000E094D094C094C11CD11CE11CF11C8DE293
:10EE10008093A605C701B60120E137E240E050E04B
:10EE20000F9450568AE0882E912CA12CB12CCA0147
:10EE3000B901A50194010F945056605D6093A70538
:10EE4000C701B60128EE33E040E050E00F94505681
:10EE5000CA01B901A50194010F945056605D6093F9
:10EE6000A805C701B60124E630E040E050E00F9469
:10EE70005056CA01B901A50194010F945056605D26
:10EE80006093A9058EE28093AA05C701B601A5018A
:10EE900094010F945056C62FCA01B901A5019401DF
:10EEA0000F945056605D6093AB05C05DC093AC0598
:10EEB00086EA95E0CF91FF90EF90DF90CF90BF90E2
:10EEC000AF909F908F9008956DEB77E386E095EB80
:10EED00060CF8F929F92AF92BF92CF92DF92EF92CC
:10EEE000FF92CF936B017C0120E030E0A9010F94E9
:10EEF000EA4F87FDAAC06DEB77E386E095E3A701B3
:10EF000096010F94DC566B017C0120E030E0A901F2
:10EF10000F94EA4F87FF9EC0C701B601905820E0CA
:10EF200030E040E251E40F94505020E030E040E205
:10EF300051E40F94505020E030E040EA50E40F9448
:10EF4000DC5620E030E040E251E40F94D6570F94B5
:10EF500048586B017C0180E28093A60560E280E165
:10EF6000C81687E2D806E104F1048CF0C701B601A7
:10EF700020E137E240E050E00F945056CA01B90159
:10EF80002AE030E040E050E00F945056605D60931E
:10EF9000A70560E288EEC81683E0D806E104F10414
:10EFA0008CF0C701B60128EE33E040E050E00F944A
:10EFB0005056CA01B9012AE030E040E050E00F9419
:10EFC0005056605D6093A80560E284E6C816D104DF
:10EFD000E104F1048CF0C701B60124E630E040E022
:10EFE00050E00F945056CA01B9012AE030E040E0E9
:10EFF00050E00F945056605D6093A9058AE0882E1A
:10F00000912CA12CB12CC701B601A50194010F943C
:10F010005056C62FCA01B901A50194010F9450564C
:10F02000605D6093AA058EE28093AB05C05DC093DE
:10F03000AC0586EA95E0CF91FF90EF90DF90CF90FE
:10F04000BF90AF909F908F9008956DEB77E386E02F
:10F0500095EB55CF20E030E040E251E4C701B60126
:10F0600062CFCF93DF93EC01CB01BA010F94F14F44
:10F0700020E030E040E251E40F94D65720E030E049
:10F08000A9010F94DC56688379838A839B83DF917F
:10F09000CF910895CF93DF93EC01CB01BA010F9488
:10F0A000F14F20E030E040E251E40F94D65720E0E9
:10F0B00030E0A9010F94DC56688379838A839B83AF
:10F0C000DF91CF9108950F94F14F20E030E040E2BE
:10F0D00051E40F94D65720E030E0A9010F94DC569C
:10F0E0000C946977CF93DF93EC01CB01BA010F94B5
:10F0F000F14F2AE037ED43E25DE30F94D65720E06D
:10F1000030E0A9010F94DC560F944F58688379833F
:10F110008A839B83DF91CF910895CF93DF93EC0196
:10F12000CB01BA010F94F14F2AE037ED43E25DE3E2
:10F130000F94D65720E030E0A9010F94DC56688385
:10F1400079838A839B83DF91CF910895CF93DF9357
:10F15000EC01CB01BA010F94F14F20E030E0A9019E
:10F160000F94DC56688379838A839B83DF91CF91E8
:10F170000895CF93DF93EC01CB01BA010F94F14FC7
:10F1800020E030E0A9010F94DC56688379838A83FC
:10F190009B83DF91CF910895CF93DF93EC01CB0157
:10F1A000BA010F94F14F20E030E048EC52E40F94A4
:10F1B000D65720E030E0A9010F94DC5668837983AC
:10F1C0008A839B83DF91CF910895CF93DF93EC01E6
:10F1D000CB01BA010F94F14F20E030E048EC52E44B
:10F1E0000F94D65720E030E0A9010F94DC566883D5
:10F1F00079838A839B83DF91CF9108950F94F14F98
:10F2000020E030E048EC52E40F94D65720E030E0A4
:10F21000A9010F94DC560C94B376CF93DF93EC01E5
:10F22000CB01BA010F94F14F20E030E0A9010F9417
:10F23000DC560F94485879836883DF91CF91089505
:10F24000CF93DF93EC01CB01BA010F94F14F20E093
:10F2500030E0A9010F94DC56688379838A839B830D
:10F26000DF91CF910895CF93DF93EC01CB01BA01E9
:10F270000F94F14F20E030E04AE754E40F94D65762
:10F2800020E030E0A9010F94DC56688379838A83FB
:10F290009B83DF91CF9108952CEA35EC47E25EE342
:10F2A00060919405709195058091960590919705D0
:10F2B0000F94D6576093291570932A1580932B15B8
:10F2C00090932C1508952CEA35EC47E25EE36091AB
:10F2D00098057091990580919A0590919B050F94DE
:10F2E00050506093251570932615809327159093A1
:10F2F000281508952CEA35EC47E25EE36091940509
:10F300007091950580919605909197050F94D65729
:10F310006093291570932A1580932B1590932C15C3
:10F3200008952CEA35EC47E25EE360919805709110
:10F33000990580919A0590919B050F945050609388
:10F3400025157093261580932715909328150895F9
:10F350008091220890912308A0912408B09125085B
:10F360008093510290935202A0935302B09354029F
:10F370000895E0918D05E63010F581E08E0F8093C1
:10F380008D0540911A0850911B0860911C087091DE
:10F390001D0890911F088091180828E0E29FF00155
:10F3A0001124E25BFA4F2091681530916915318381
:10F3B0002083428353836483758396838783089570
:10F3C000FC01A081B1811C92A281B3818C918F5FDD
:10F3D0008C930280F381E02D90818CE0989F800DCA
:10F3E0001124EAE6F5E113AE84AF0895CF92DF92DF
:10F3F000EF92FF92CF93DF9300D01F92CDB7DEB78D
:10F400006B017C0120E030E0A9010F94EA4F87FDF9
:10F410001CC06DEB77E386E095E3A70196010F949E
:10F42000DC5669837A838B839C8360E2CE010196EC
:10F430000E949FFD0F900F900F900F90DF91CF9142
:10F44000FF90EF90DF90CF9008956DEB77E386E02B
:10F4500095EBE3CF0F94F14F20E030E04AE754E41E
:10F460000F94D65720E030E0A9010F94DC560C949D
:10F47000F679CF92DF92EF92FF926B017C0120E050
:10F4800030E0A9010F94EA4F87FD26C06DEB77E3CA
:10F4900086E095E3A70196010F94DC566B017C0191
:10F4A00020E030E0A9010F94EA4F20E030E040E096
:10F4B0005FE387FF04C020E030E040E05FEBC7017E
:10F4C000B6010F94DC560F944858CB01FF90EF9093
:10F4D000DF90CF900D949B006DEB77E386E095EB8A
:10F4E000D9CF0F94F14F20E030E0A9010F94DC5602
:10F4F0000C94397A0F94F14F20E030E0A9010F9479
:10F50000DC560F944858CB010D949B000F94F14F9B
:10F5100029EC38EC48EC5EE30F94D65720E030E05D
:10F5200040E05FE30F94DC560F944F58862F0D9404
:10F53000F2000D947A320D947A326FEF80912208A6
:10F540000D94983061E373EB82E00D94BF4166E364
:10F5500073EB81E00D94BF416BE373EB80E00D949E
:10F56000BF416CEE70EB83E00D94BF41CF92DF9210
:10F57000EF92FF92CF93DF9300D01F92CDB7DEB70B
:10F580006B017C0120E030E0A9010F94EA4F87FD78
:10F590001BC06DEB77E386E095E3A70196010F941E
:10F5A000DC5669837A838B839C83CE0101960E940B
:10F5B0003BFE0F900F900F900F90DF91CF91FF9037
:10F5C000EF90DF90CF9008956DEB77E386E095EBB9
:10F5D000E4CF0F94F14F20E030E040E251E40F948B
:10F5E000D65720E030E0A9010F94DC560C94B67A8F
:10F5F0008091421590914315891B8F7011F40C94E2
:10F60000123681E0089580917802882351F060914C
:10F6100092057091930530E020E041E081E00C9488
:10F620006B2A089584E00D946B2F83E00D946B2F6B
:10F6300082E00D946B2F0F94F14F20E030E0A90190
:10F640000F94DC560F944F58862F0D94D000909154
:10F65000E50F81E089270C94AE3461E082E298E006
:10F660000C94C9340F949A270C94D8F080E090E061
:10F67000A0E8B0E48093EE0F9093EF0FA093F00F0B
:10F68000B093F10F87ED92E00E94B6EFE0919D05F7
:10F6900080E090E0A6E1B3E4E43009F44AC080E001
:10F6A00090E0A0EBB1E48093E60F9093E70FA09376
:10F6B000E80FB093E90F8093EA0F9093EB0FA093BC
:10F6C000EC0FB093ED0FEE0FFF0BE954FD4F80816F
:10F6D00091818330910549F184309105D9F10297E8
:10F6E00061F480E090E0ABE8B3E48093E60F9093A0
:10F6F000E70FA093E80FB093E90F8FEB92E00E9421
:10F70000B6EF1092EE0F1092EF0F1092F00F1092D2
:10F71000F10F87ED92E00E94B6EF80919D058F5F1B
:10F720008530ECF480939D05089580E090E0ABE88F
:10F73000B3E48093E60F9093E70FA093E80FB093A4
:10F74000E90F8093EA0F9093EB0FA093EC0FB09327
:10F75000ED0FD3CF80E090E0ABE8B3E4F2CF1092AE
:10F760009D050895CF93DF9300D01F92CDB7DEB7EC
:10F770000F944F580F94EF4F69837A838B839C8348
:10F78000CE0101960E941CFD0F900F900F900F90DC
:10F79000DF91CF9108950F94F14F2AE037ED43E2C6
:10F7A0005DE30F94D65720E030E0A9010F94DC56BA
:10F7B0000C94B27BCF92DF92EF92FF92CF93DF93C4
:10F7C00000D01F92CDB7DEB76B017C0120E030E0A6
:10F7D000A9010F94EA4F87FD1BC06DEB77E386E02C
:10F7E00095E3A70196010F94DC5669837A838B8396
:10F7F0009C83CE0101960E941CFD0F900F900F90EC
:10F800000F90DF91CF91FF90EF90DF90CF90089510
:10F810006DEB77E386E095EBE4CF0F94F14F2AE0B0
:10F8200037ED43E25DE30F94D65720E030E0A901C5
:10F830000F94DC560C94DA7B0F94F14F20E030E00B
:10F84000A9010F94DC560C94DA7BCF92DF92EF92F1
:10F85000FF926B017C0120E030E0A9010F94EA4F98
:10F8600087FD26C06DEB77E386E095E3A70196015F
:10F870000F94DC566B017C0120E030E0A9010F946D
:10F88000EA4F20E030E040E05FE387FF04C020E083
:10F8900030E040E05FEBC701B6010F94DC560F94F7
:10F8A0004858CB01FF90EF90DF90CF900C94F1FF80
:10F8B0006DEB77E386E095EBD9CF0F94F14F20E025
:10F8C00030E0A9010F94DC560C94257CCF92DF9296
:10F8D000EF92FF92CF93DF9300D01F92CDB7DEB7A8
:10F8E0000F94F14F20E030E048EC52E40F94D657EB
:10F8F00020E030E0A9010F94DC566B017C0120E090
:10F9000030E0A9010F94EA4F2DEB37E346E055E3D1
:10F9100087FF04C02DEB37E346E055EBC701B60186
:10F920000F94DC5669837A838B839C83CE01019686
:10F930000E94B7FE0F900F900F900F90DF91CF9124
:10F94000FF90EF90DF90CF9008950C94C6DC0C945C
:10F95000C6DC0C94C6DC0C94C6DC0C9478DC0C94ED
:10F9600078DC0C9478DC0C9478DCCF92DF92EF9208
:10F97000FF92CF93C82F0F946E326B017C0124EA63
:10F9800030E74DE75FE36091250270912602809198
:10F990002702909128020F94EA4F87FD18C08AEF42
:10F9A00090E0A0E0B0E08C0D9D1DAE1DBF1D8093CA
:10F9B000380590933905A0933A05B0933B05C09361
:10F9C0001E02CF91FF90EF90DF90CF90089580E0DE
:10F9D00090E0DC01E8CFCF92DF92EF92FF920F939D
:10F9E0001F930F946E320091090510910A05209122
:10F9F0000B0530910C056B017C01C01AD10AE20A9B
:10FA0000F30A9701860137FD11C020910805209562
:10FA1000209308056A547C4F8F4F9F4F60930905D0
:10FA200070930A0580930B0590930C0581E09091EB
:10FA30000805911101C080E01F910F91FF90EF9098
:10FA4000DF90CF9008950F940B4010924C081092C5
:10FA50006C020E943D36882351F08091DC1582FDB6
:10FA600006C08BE09EE19093C2078093C10761E0DE
:10FA700084E09EE10E94BA370C94CFFC4F925F92D3
:10FA80006F927F928F929F92BF92CF92DF92EF926E
:10FA9000FF920F931F93CF93DF9300D000D01F925C
:10FAA0001F92CDB7DEB77C016A014901FB0190814D
:10FAB0008CE0989F800D1124982FF7012081822FD0
:10FAC000880F820F880F8093A5159093A615411576
:10FAD000510571F1FA82E9827C836B83011121C0A7
:10FAE000AE014B5F5F4FB401C6010E94A7276C01B6
:10FAF0006D817E818F8198856115710581059105E4
:10FB0000B9F00E940829F70180818F5F80838531D9
:10FB100038F3CE0101960E94E079E2CFB12C860144
:10FB200029C08A01B12C26C0452846284728B1F7AC
:10FB300028960FB6F894DEBF0FBECDBFDF91CF91F0
:10FB40001F910F91FF90EF90DF90CF90BF909F900B
:10FB50008F907F906F905F904F900895B39407C0FF
:10FB6000B1102EC001151105C9F20F5F1F4F01150D
:10FB70001105A9F2AE014B5F5F4FB401C6010E94AF
:10FB8000A7276C014D805E806F80788441145104FA
:10FB900061047104A9F0F0E24F165104610471048C
:10FBA000F9F2D301C2018D97A109B1090297A1050C
:10FBB000B10530F04BE2441651046104710471F652
:10FBC000F7018081482F4B0D5527551F46315105B0
:10FBD00034F0853020F0CE0101960E94E07981E07A
:10FBE000411451046104710409F480E0B80EF70176
:10FBF00080818B0D8083BB2009F496CFBA94AE012F
:10FC00004B5F5F4FB401C8010E94A7278C016D8133
:10FC10007E818F8198850E940829EDCFEF92FF9217
:10FC20000F931F93CF93DF9300D000D000D01F928B
:10FC30001F92CDB7DEB77C0120912008422F022E03
:10FC4000000C550B80912108833099F1843051F1DB
:10FC50008AE991E25F932F939F938F938E010F5FB9
:10FC60001F4F1F930F930F94814FC7010E946CDCAD
:10FC70004FE350E0B80183EC97E00F94515A0F9096
:10FC80000F900F900F900F900F902B960FB6F89447
:10FC9000DEBF0FBECDBFDF91CF911F910F91FF90BF
:10FCA000EF90089586EA91E227FDD4CF81E991E2B1
:10FCB000D1CF8FEA91E2CECFE0912C0885E1E80226
:10FCC000F0011124E85EFA4E868197810C940E7E35
:10FCD000E0912C0886E0E802F0011124EB5FF74F79
:10FCE000808191810C940E7E0F931F93CF93DF93AD
:10FCF0008C01EB019091561520915715921305C078
:10FD00000F94D8010E94DAF0F5CF8091551534E0B8
:10FD1000839FF0011124E85AFA4E11830083D383A4
:10FD2000C2839F5F909356158F5F281739F0809399
:10FD30005515DF91CF911F910F9108951092551590
:10FD4000F8CF63E972E084E690E00E94747E6AEB8B
:10FD500072E084E690E00C94747E81110C94A17E94
:10FD600068EB71E084E190E00C94747E0E94BAD854
:10FD70000C94AD7E0F9495120C94AD7E0E9494FA73
:10FD80000C94A17ECF93DF93CDB7DEB720E24885F8
:10FD900059856F818E810F94412CDF91CF91089509
:10FDA000282F10922A0880911A0890911B08A09180
:10FDB0001C08B0911D08B7FF08C010921A081092D5
:10FDC0001B0810921C0810921D088091A50588231D
:10FDD00031F080911A0880931E08109219088091C2
:10FDE00018081816FCF4082E000C990B821B9109B8
:10FDF00020911E08022E000C330B2817390794F0AF
:10FE000097FF02C090E080E080931E08092E000C4E
:10FE1000AA0BBB0B80931A0890931B08A0931C0895
:10FE2000B0931D0880911E086623A9F090911F08C9
:10FE3000891714F480931F0820911F08022E000CCC
:10FE4000330B2C5F3F4F482F082E000C550B241707
:10FE500035071CF4845080931F0808955F926F92B9
:10FE60007F928F929F92AF92BF92CF92DF92EF924A
:10FE7000FF920F931F93CF93DF9361E081E00E9485
:10FE8000D07EC0911F0885E0982E9C0ED1E09DEE9B
:10FE9000E92E91E2F92E882483947D2E7C1A6C2E13
:10FEA00061942FECC22E21E2D22E12E01C1B33E013
:10FEB000532E44E2A42E42E2B42EC11141C0DD23F0
:10FEC000D9F080911E081816BCF040911A08509184
:10FED0001B0860911C0870911D084F5F5F4F6F4FAA
:10FEE0007F4F40931A0850931B0860931C0870932F
:10FEF0001D088F5F80931E0880917802882341F04F
:10FF000030E020E041E068EF71E2862D0E946B2A2C
:10FF100080914A08882309F487C0C23051F4809147
:10FF20001E08823009F445C08091780281115AC0C0
:10FF3000D0E0CF5F9C12C1CF83E08093180818C037
:10FF4000C13031F790911E08913031F080917802E4
:10FF500081111EC0D0E0DCCF8091170810921708E5
:10FF60008823A1F3C0934B0880911908882371F36B
:10FF7000DF91CF911F910F91FF90EF90DF90CF9085
:10FF8000BF90AF909F908F907F906F905F900895FB
:10FF90001F92FF92EF927F9281E0913009F080E012
:10FFA0008F930E94C27E0F900F900F900F900F9032
:10FFB000D1CF8091170810921708882309F4B4CF85
:10FFC0008091550288258093550250927802A114A1
:10FFD000B10411F00E94242280911908882309F4A9
:10FFE000A3CFC6CF81E090911E08923009F080E047
:10FFF000909155022CED31E2911102C028ED31E2D1
:020000021000EC
:1000000001E04FED51E2612F0E94662B91CF80916C
:10001000170810921708882371F0C0934B0880913D
:100020001908882341F0A4CFC23009F082CF909103
:100030001E08923061F380917802882309F478CF0A
:100040001F92DF92CF921F9381E0923009F080E0FF
:100050008F930E94C27E0F900F900F900F900F9081
:1000600067CF2F923F924F925F926F927F928F92C3
:100070009F92AF92BF92CF92DF92EF92FF920F9337
:100080001F93CF93DF934C010F94374F0196840158
:10009000080F191FC8010F94374F01966801C80E49
:1000A000D91EF8016080C1E0611001C0C0E0F60116
:1000B0003080D1E0311001C0D0E0AA24A3946110B7
:1000C000A12C60E085E00E94D07E50901F08752C26
:1000D0009EE0E92EF12C252C21948A2D90E00196AA
:1000E0005C01AC0EB11CAD0EB11C71101DC0809135
:1000F00078028823A1F0E0912402E25068E072E2E5
:10010000E33038F4F0E0EE0FFF1FE152FD4F608165
:10011000718130E020E043E0822D0E946B2AD1E023
:10012000611013C0D2E011C0D2E06110D1E0D7114C
:100130000CC080917802882341F030E020E041E05B
:10014000B4018D2F85190E946B2AC1E0CD0F472C79
:100150004518662079F0C7110BC08091780288237A
:1001600039F030E020E041E0B801842D0E946B2A94
:10017000C2E0CD0F332071F0C7110BC0809178021F
:10018000882339F030E020E041E0B601842D0E9460
:100190006B2ACF5FF3E0AF16B1040CF4CF5FC71149
:1001A00062C080917802882309F45AC030E020E0D0
:1001B00042E065E172E2842D0E946B2AD09106052F
:1001C00093EF9E0D909305058EEF8E0D80932B0877
:1001D0002091A2152E151F0411F00CF041C02091A2
:1001E000A4159217E8F59EE39093A5158093A615A4
:1001F00065E470E080E090E00E94082961E36D0F03
:10020000062E000C770B880B990B0E94082960E2E0
:1002100070E080E090E00E94082980911C15909188
:100220001D150F949B000E94E32A6FE270E080E0AE
:1002300090E00E9408290E94EB7C811109C085E0B2
:100240008D9FF0011124ED5BF94F8481811108C06D
:1002500080911E1590911F150F949B000E94E32A18
:1002600092E090937802ECE0EE0EF11C7394FAE4C5
:10027000EF16F10409F039CFCF5FC0931808DF9172
:10028000CF911F910F91FF90EF90DF90CF90BF9093
:10029000AF909F908F907F906F905F904F903F9026
:1002A0002F90089580E292E20C9431808DE292E2E8
:1002B0000C9431808FE492E20C9431808AEE92E2C9
:1002C0000C94318085EA92E20C94318082ED92E2C6
:1002D0000C94318085E293E20C94318088E093E2C3
:1002E0000C94318088E892E20C94318089E692E2A5
:1002F0000C9431808F929F92AF92BF92EF92FF92B7
:100300000F931F93CF93DF93EC018B01E42EF22E1A
:1003100080916815909169158C179D0709F43EC06E
:100320002091FE0427FD1092FE0424EBC730D20773
:1003300009F03FC08B519D4B71F40F946E326E519A
:100340007B4F8F4F9F4F60938E0570938F058093E7
:10035000900590939105D0936915C093681530E08E
:1003600020E000931A0810931B0820931C08309378
:100370001D08E0921F08F0921808CB51DD4B21F4C4
:100380001092070510928D0582E08093780281E03B
:10039000809319081092A20510929C05DF91CF91CD
:1003A0001F910F91FF90EF90BF90AF909F908F9013
:1003B00008952DEBCB31D20771F68750944B19F08D
:1003C000CBE1DDEBC8CF0F946E3280908E0590901C
:1003D0008F05A0909005B0909105681979098A0958
:1003E0009B0997FFEDCF8091BF078770873041F75A
:1003F000C9E0D2E8B0CFCF93DF93EC010E94B97986
:1004000020E040E070E060E0CE01DF91CF910C94FD
:100410007A8120E040E070E060E085EF9FEA0E9492
:100420007A8181E08093070510924808109247086E
:10043000089520E040E070E060E081EB9AE70C94E2
:100440007A8180919809811114C080917D029091E8
:100450007E02019720911C1530911D152817390730
:1004600044F420E040E070E060E080E09CEB0C941D
:100470007A810C94198221E020930705FC01808188
:100480009181A281B3818093250290932602A0934B
:100490002702B093280220E040E070E060E0809105
:1004A0001508909116080C947A81CF93DF9300D0B1
:1004B0001F92CDB7DEB78DEC9CECACECBCE389832E
:1004C0009A83AB83BC83CE0101960E943B820F903E
:1004D0000F900F900F90DF91CF910895CF93DF93FE
:1004E00000D01F92CDB7DEB78DEC9CECACECBDE339
:1004F00089839A83AB83BC83CE0101960E943B82A1
:100500000F900F900F900F90DF91CF910895CF93A0
:10051000DF9300D01F92CDB7DEB780E090E0A0E877
:10052000BFE389839A83AB83BC83CE0101960E948B
:100530003B820F900F900F900F90DF91CF91089515
:10054000CF93DF9300D01F92CDB7DEB780E090E06D
:10055000A0E2B1E489839A83AB83BC83CE01019688
:100560000E943B820F900F900F900F90DF91CF91E0
:1005700008958FEF8093220820E040E070E060E073
:1005800086E197E90C947A8181E0809307051092C7
:10059000BF071092AE0520E040E070E060E08BEF16
:1005A00092E80E947A8189E696E29093C20780934E
:1005B000C107089581E0809307058091BF07877088
:1005C000873051F01092BF071092AE0589E696E28F
:1005D0009093C2078093C1078091E50F80939E0599
:1005E00080E00E94AE3420E040E070E060E08CE407
:1005F00094E80C947A8180917802882341F030E06D
:1006000020E041E06DE370E282E00E946B2A80917D
:10061000AE058770873041F420E040E070E060E094
:100620008EE293E80C947A81089520E040E070E037
:1006300060E085E493E80E947A8181E08093FF0482
:1006400080919F05811107C082E290E29093C207DA
:100650008093C107089588E290E2F8CF80917802F4
:10066000882341F030E020E041E06EE270E281E07A
:100670000E946B2A8091170810921708882321F096
:1006800010929F050C94158308950F931F93CF9399
:10069000DF9300D000D000D01F92CDB7DEB780919D
:1006A00078028823F1F01F9289E18F9380919F0552
:1006B00090E001969F938F938AE190E29F938F93AE
:1006C0008E010F5F1F4F1F930F930F94814FB8013F
:1006D0008FE090E20E94E72A0FB6F894DEBF0FBECB
:1006E000CDBF84E0809378028091FF04811108C01F
:1006F00020E040E070E060E08BE893E80E947A81BF
:100700002A960FB6F894DEBF0FBECDBFDF91CF9112
:100710001F910F910895CF92DF92EF92FF92CF93A6
:10072000DF9300D01F92CDB7DEB7809117081092EB
:100730001708882331F180919F058F5F80939F0573
:100740008931E0F081E08093FF0420E040E070E038
:1007500060E080E493EB0E947A8189E090E29093DC
:10076000C2078093C1070F900F900F900F90DF91F9
:10077000CF91FF90EF90DF90CF9008950E94158366
:10078000F2CF60911A0870911B0880911C0890911B
:100790001D08611571058105910509F43EC00F948E
:1007A000F14F2DEC3CEC4CEC5CE30F94505020915D
:1007B000EE0F3091EF0F4091F00F5091F10F0F9429
:1007C000DC566B017C0120E030E040E850EC0F94F7
:1007D000EA4F87FD53C020E030E040E850E4C70115
:1007E000B6010F943C5918160CF44FC0C092EE0F8E
:1007F000D092EF0FE092F00FF092F10F87ED92E0C0
:100800000E94B6EF82E08093780210921A0810924C
:100810001B0810921C0810921D08809178028823F2
:1008200009F4A1CFC090EE0FD090EF0FE090F00F41
:10083000F090F10F20E030E0A901C701B6010F945C
:10084000EA4F27E137EB41ED58E387FF04C027E18A
:1008500037EB41ED58EBC701B6010F94DC566983C5
:100860007A838B839C836BE2CE0101960E949FFD6D
:10087000BC0182E090E20E94E72A75CFC12CD12C06
:1008800090E8E92E90ECF92EB1CFC12CD12C80E864
:10089000E82E80E4F82EAACF80917802882341F0D8
:1008A00030E020E041E06DE370E282E00E946B2ADC
:1008B0008091AE058770873079F410929D0520E015
:1008C00040E070E060E082ED9CEB0E947A8181E084
:1008D00080939C050C94367B08952F923F924F9203
:1008E0005F926F927F928F929F92AF92BF92CF92C0
:1008F000DF92EF92FF920F931F93CF93DF9300D07D
:1009000000D0CDB7DEB71C017A8369832B833C838B
:100910004D835E832701380181E0809319080E948E
:10092000B97983E08093780230928C0520928B0510
:1009300089819A8190938A05809389058B819C8116
:10094000AD81BE818093850590938605A093870530
:10095000B09388054092810550928205609283058C
:1009600070928405F12CE12CC0921A08D0921B08D9
:10097000E0921C08F0921D08B0926915A0926815CB
:100980009092800580927F058C8D80937E052696BF
:100990000FB6F894DEBF0FBECDBFDF91CF911F9190
:1009A0000F91FF90EF90DF90CF90BF90AF909F900E
:1009B0008F907F906F905F904F903F902F90089511
:1009C00020E040E070E060E08BE19DEB0C947A81E8
:1009D0000E9474360E943BD50C94E08485E598E033
:1009E0000F94D33D0E94E0840D940B400E94E0845C
:1009F00085EB94E29093C2078093C10708950E940B
:100A0000CF330F94103F81E08093D2150F94523F63
:100A10000C94E0846F927F928F929F92AF92BF92DC
:100A2000CF92DF92EF92FF920F931F93CF93DF93BA
:100A300081E08093070561E00E94D07EC0911F088D
:100A400085E0882E8C0ED1E00FEF14E89BEBE92EA9
:100A500094E2F92E82E0982E9C1A26EFC22E24E80A
:100A6000D22E36ECA32E34E2B32E7D2E7C1A6C2EC1
:100A70006194C11130C0DD23D9F080911E08181691
:100A8000BCF040911A0850911B0860911C087091AD
:100A90001D084F5F5F4F6F4F7F4F40931A08509371
:100AA0001B0860931C0870931D088F5F80931E08BD
:100AB00080917802882341F030E020E041E063ED4E
:100AC00074E2862D0E946B2ACF5F8C12D2CF83E016
:100AD0008093180823C0C13081F580911E088130B1
:100AE00089F080917802882309F444C0DF92CF9284
:100AF000BF92AF927F9281E090911E08913089F170
:100B000080E02FC08091170810921708882349F3BE
:100B10000E94F68480911908882319F3DF91CF9100
:100B20001F910F91FF90EF90DF90CF90BF90AF900B
:100B30009F908F907F906F900895C23029F680919A
:100B40001E088230C9F080917802882399F01F93A3
:100B50000F93FF92EF929F9281E090911E08923046
:100B600079F68F930E94C27E0F900F900F900F9096
:100B70000F900F90D0E0A8CF80911708109217081F
:100B8000882309F30E94FF84809119088823D9F2F1
:100B9000C5CF611160932402409306058C3008F0A4
:100BA0003AC0E82F880FFF0B8827E652FA478F4F8D
:100BB0000D94D3560D86E685F1851086F485F7856C
:100BC000FA850686FD850B860086038686E591E814
:100BD00021E02093070520E040E070E060E00C9405
:100BE0007A818EE591E8F4CF82E691E8F1CF86E64E
:100BF00091E8EECF8AE691E8EBCF8EE691E8E8CF78
:100C000082E791E8E5CF86E791E8E2CF10924B08C2
:100C10008EE29FE7DDCF0C94E08482E591E8D8CFA7
:100C20008AE591E8D5CFCF930E9494FA0E94BAD872
:100C3000C82F882319F080E00F94790B8C2F0E9425
:100C4000AD7ECF910C94E0840F931F93CF93DF93ED
:100C5000CDB7DEB76E970FB6F894DEBF0FBECDBF2F
:100C6000282F082E000C330B90911F024091200278
:100C70008F3F39F0F901EE0FFF1FEF5DFD4F9081BF
:100C800041814F939F933F938F9384E49EE19F9381
:100C90008F938E010F5F1F4F1F930F930F94814F00
:100CA0004FE350E0B80183EC97E00F94515A0E9453
:100CB000E0840FB6F894DEBF0FBECDBF6E960FB6C0
:100CC000F894DEBF0FBECDBFDF91CF911F910F9182
:100CD00008958FEF0C94248680912C080C94248620
:100CE000E0918D05EE2389F0E150E0938D0588E0D9
:100CF000E89FF0011124E25BFA4F62817381278142
:100D00004681808191810C947A810C94E0842F92A9
:100D10003F924F925F926F927F928F929F92AF928B
:100D2000BF92CF92DF92EF92FF920F931F93CF93D8
:100D3000DF9300D01F92CDB7DEB761E081E00E9463
:100D4000D07E80911F088B83382E8B5F898388E04B
:100D500083198A8397E093199C8386E0782E731811
:100D600085E0682E631884E0582E531882E0482EE0
:100D70004318232C21948B8181115BC080911E0824
:100D8000882399F180917802882359F081E090912D
:100D90001E08911180E024E04CEF56E2622D0F9482
:100DA000412C80918609809322089B81953009F01F
:100DB0009EC010922C0880911E08853009F458C1FD
:100DC00080917802882309F4FEC111E080911E0809
:100DD000853009F010E0809122080F94F20000E0C5
:100DE0009C0149ED56E2662D7FC080911708109254
:100DF0001708882339F20E94708680911908882389
:100E000009F4C0CF0F900F900F900F90DF91CF910A
:100E10001F910F91FF90EF90DF90CF90BF90AF9018
:100E20009F908F907F906F905F904F903F902F900A
:100E300008959B819130B1F580911E088130D9F0E1
:100E400080917802882309F4ACCF11E080911E08CC
:100E5000813009F010E080916E0290916F020F9442
:100E60009B0061E0631900E09C0146EF56E2812F90
:100E70000E94662B96CF809117081092170888233E
:100E8000F9F210E000E027EE33E04AE050E06EE6D1
:100E900072E086EF96E20F942E2E80911908882337
:100EA00079F2B0CF8B81823009F06AC180911E083F
:100EB000823009F44CC0809178028823C1F011E09F
:100EC00080911E08823009F010E060913006709128
:100ED000310680913206909133060E94F67900E047
:100EE0009C0140EF56E2642D812F0E94662B809179
:100EF0008709809322088B81863009F0E3C081E066
:100F000080932C0880911E08863009F4C6C0809119
:100F10007802882391F011E080911E08863009F054
:100F200010E0809122080F94F20000E09C0149ED4E
:100F300056E2672D812F0E94662B9B819F5F9B83CA
:100F40008981981318CF89E0809318085BCF80912E
:100F5000170810921708882309F4ADCF20E030E07D
:100F60004AE754E460913006709131068091320670
:100F7000909133060F94505020E030E0A9010F9477
:100F8000DC5620E030E04AE754E40F94DC560F943E
:100F90004F581F92912C812C83EAA82E8FEAB82EED
:100FA0006B0110EDE12E17E0F12E00E010E028E1DA
:100FB0003CEF4FEF5FEF60E376E080EF96E20E9458
:100FC0006D840F9080911908882309F474CF1ACF8B
:100FD00080911E088330C1F080917802882309F443
:100FE00086CF11E080911E08833009F010E08091D7
:100FF0001E1590911F150F949B0063E0631900E08C
:101000009C0149EE56E233CF8091170810921708E1
:10101000882311F30F94B62C0BE91AE723EB31E088
:1010200050E040E06EE175E189EE96E20F942E2EDD
:1010300080911908882381F2E5CE809117081092DB
:101040001708882309F4A8C00F94B62C0BE417ECFA
:101050002CE830E050E040E06EE678E085EE96E285
:101060000F942E2E80911908882309F495C0CACEBA
:101070008091170810921708882309F4A1CE0F94C5
:10108000B62C60E376E789ED96E20F94272F8091E6
:101090001908882309F494CEB5CE809117081092D0
:1010A0001708882309F433CF0F94B62C60E376E752
:1010B00089ED96E20F94272F80911908882309F46F
:1010C00026CFA0CE9B81973091F580911E08873066
:1010D000B9F080917802882309F42FCF11E0809134
:1010E0001E08873009F010E0809135029091360299
:1010F0000F949B0000E09C0144ED56E26C811ACFF6
:101100008091170810921708882319F30DE016E74D
:1011100027EE33E04AE050E065E372E084ED96E2CA
:101120000F942E2E80911908882399F26BCE8B8113
:10113000883009F002CF80911E08883091F08091AC
:101140007802882309F4F9CE81E090911E08983046
:1011500009F080E023E049EC56E26A810F94412CCB
:10116000ECCE8091170810921708882341F389E08C
:1011700092E80E94FB8180911908882301F342CEF6
:101180009B81933009F424CF943009F00ACE8091EA
:101190001E08843009F451CF80917802882309F425
:1011A000A6CE11E080911E08843009F010E08091F5
:1011B0006E0890916F080F949B0000E09C0145EE33
:1011C00056E2652D54CE8091870980932208B5CED2
:1011D0005F926F927F928F929F92AF92BF92CF92C7
:1011E000DF92EF92FF920F931F93CF93DF93FF2431
:1011F000F39480911E1590911F15892B09F4F12C01
:1012000061E081E00E94D07EC0911F088C2E95E0A5
:10121000992E9C0EAA24A39484E0E82EEC1A83E075
:10122000D82EDC1A82E0C82ECC1A7A2C7C1A6C2EAE
:10123000619487E0B82EBC1AC111B8C080911E0815
:10124000882309F495C080917802882359F081E0C1
:1012500090911E08911180E024E044EC56E2662D46
:101260000F94412C8091870980932208C430E9F4BF
:10127000A0922C0880911E08843009F445C1809109
:101280007802882391F0D1E080911E08843009F023
:10129000D0E0809122080F94F20000E09C014DEA1A
:1012A00056E26E2D8D2F0E94662B10E000E0D5E0F7
:1012B0005C2E581800932208CD131FC0F801EE0FC2
:1012C000FF1FED54F04C8591949190932E088093DC
:1012D0002D0880911E088C1709F42BC1809178028B
:1012E000882359F081E090911E089D1380E023E04F
:1012F00043EA56E2652D0F94412C8D2F0F5F1F4F4F
:10130000D6E08630B9F680916E0890916F08892BEF
:1013100019F4FF2009F42DC1C73009F580911E088A
:10132000873009F417C1809178028823C1F088EED4
:1013300094E89F938F938AE996E29F938F93BF924D
:1013400081E090911E08973009F080E08F930E9411
:10135000C27E0F900F900F900F900F900F9088E02B
:10136000FF24F394CF5FC91167CF809318080EC094
:101370008091170810921708882309F464CF0E94FF
:10138000708680911908882309F45DCFDF91CF9191
:101390001F910F91FF90EF90DF90CF90BF90AF9093
:1013A0009F908F907F906F905F900895C13009F06B
:1013B0005FC080911E08813009F43FC0809178029F
:1013C000882309F44FCFD1E080911E08813009F0C5
:1013D000D0E080911E1590911F150F949B0000E0A6
:1013E0009C014DEB56E2672D8D2F0E94662B80915C
:1013F000860980932208C33009F034CF10922C085C
:1014000080911E08833009F46AC080917802882395
:1014100009F44BCFD1E080911E08833009F0D0E071
:10142000809122080F94F20000E09C014DEA56E200
:101430006D2D8D2F0E94662B15CF8091170810926D
:101440001708882309F4BACF0F94B62C09E91AE7D4
:1014500023EB31E050E040E06EE175E18DEB96E288
:101460000F942E2E80911908882309F4A7CF8ECFD0
:10147000C23009F0BCCF80911E088230B9F0809153
:101480007802882309F4EECED1E080911E088230E4
:1014900009F0D0E080916E0890916F080F949B0046
:1014A00000E09C0149EB56E26C2D9ECF809117081D
:1014B00010921708882319F30F94B62C0BE417EC3D
:1014C0002CE830E050E040E06EE678E089EB96E210
:1014D0000F942E2E80911908882389F257CF80917E
:1014E000170810921708882309F48FCF0F94B62C91
:1014F00060E376E78DEA96E20F94272F8091190832
:10150000882309F482CF42CF8091170810921708E0
:10151000882309F4B4CE0F94B62C60E376E78DEA05
:1015200096E20F94272F80911908882309F4A7CEFB
:101530002DCF8091170810921708882309F4CECE7A
:101540008BEB9AE80E94FB8180911908882309F4AB
:10155000C5CE1CCF8091170810921708882309F474
:10156000E2CE0E94E88480911908882309F4DBCE3A
:101570000DCF87E0F7CE4F925F926F927F928F925E
:101580009F92AF92BF92CF92DF92EF92FF920F9312
:101590001F93CF93DF930091220861E081E00E94C6
:1015A000D07EC0911F0810E0000F111F0D54104C89
:1015B00095E0592E5C0E20E8E22E26E2F22ED3E0D2
:1015C000DC1B3DE9C32E3AE7D32E42E7A42E46E2C8
:1015D000B42E82E0782E7C1A53EA852E56E2952EA0
:1015E00081E0682E6C1A4C2E4194C11137C0809155
:1015F0001E088823B1F080917802882359F081E099
:1016000090911E08911180E024E04EE856E2642D8E
:101610000F94412CCF5F5C12E8CF84E080931808D0
:101620000CC08091170810921708882321F30E949C
:101630007086809119088823F1F2DF91CF911F9174
:101640000F91FF90EF90DF90CF90BF90AF909F9061
:101650008F907F906F905F904F900895C13059F5B3
:10166000F8018591949190932E0880932D08809194
:101670001E08813081F080917802882359F21F92F0
:101680009F928F926F9281E090911E08913009F4A1
:1016900074C080E072C080911708109217088823E8
:1016A00051F380912208682F0F9498308091190887
:1016B000882309F3C2CFC23009F042C0F8018591F6
:1016C000949190932E0880932D0880911E0882306B
:1016D000D1F080917802882309F49CCFDF92CF92D9
:1016E000BF92AF927F9281E090911E08923009F0F4
:1016F00080E08F930E94C27E0F900F900F900F900A
:101700000F900F9087CF80911708109217088823A9
:1017100001F30E949D7A809119088823D1F28DCF20
:1017200080911708109217088823C1F06091220851
:101730008FEF0F94983080911908882379F07DCF2E
:10174000C33009F067CFF8018591949190932E08EA
:1017500080932D0880911E08833011F380917802C8
:10176000882309F457CF1F92FF92EF92DF9381E015
:1017700090911E08933009F08CCF8F930E94C27E07
:101780000F900F900F900F900F9044CF9F92AF92B9
:10179000BF92CF92DF92EF92FF920F931F93CF935E
:1017A000DF9361E081E00E94D07EC0911F08CC2EC3
:1017B00085E0982E9C0E9AE2A92E96E2B92ED7E0EB
:1017C000DC1B16E01C1B05E00C1B84E0F82EFC1A49
:1017D00082E0E82EEC1A81E0D82EDC1AC11133C069
:1017E00080911E088823B9F080917802882361F0E7
:1017F0006C2D619581E090911E08911180E024E0AC
:101800004DE656E20F94412CCF5FC911E7CF88E037
:10181000809318080CC0809117081092170888232D
:1018200019F30E947086809119088823E9F2DF91EC
:10183000CF911F910F91FF90EF90DF90CF90BF90CD
:10184000AF909F900895C13011F580911E088130AE
:1018500079F0809178028823B9F281E090911E0896
:10186000913009F080E023E04BE85FE36D2DCACFB3
:101870008091170810921708882359F389E29DE890
:101880000E94FB8180911908882319F3D0CFC230C0
:1018900009F0BFC090911E08923071F080917802DB
:1018A000882309F4B1CF81E0923009F080E020E292
:1018B0004FE556E26E2DA6CF8091170810921708BB
:1018C000882361F329E636E23093C2072093C107EB
:1018D00080911908882311F3AACF90911E089330A4
:1018E00079F080917802882309F48ECF63E06C1937
:1018F00081E0933009F080E020E243E556E282CFB8
:101900008091170810921708882359F32AE536E2C8
:101910003093C2072093C10780911908882309F3E7
:1019200086CF90911E08943071F0809178028823C0
:1019300009F46ACF81E0943009F080E020E247E4C6
:1019400056E26F2D5FCF80911708109217088823F9
:1019500061F32EE436E23093C2072093C1078091F1
:101960001908882311F363CF90911E08953071F008
:1019700080917802882309F447CF81E0953009F0FF
:1019800080E020E24BE356E2602F3CCF80911708C5
:1019900010921708882361F322E436E23093C207DD
:1019A0002093C10780911908882311F340CF8091BB
:1019B0001E08863081F080917802882309F424CFB4
:1019C00081E090911E08963009F080E023E04EE21D
:1019D00056E2612F17CF80911708109217088823BD
:1019E00051F385E49EE80E94FB81809119088823C9
:1019F00011F31DCF80911708109217088823D9F092
:101A0000B092C207A092C10780911908882399F06B
:101A10000ECFC33009F461CFC43009F482CFC53092
:101A200009F4A2CFC63019F2C73009F0EDCE90917B
:101A30001E089730F9F280917802882309F4E4CEE9
:101A400081E0973009F080E020E249E156E26D2F15
:101A5000D9CEAF92BF92CF92DF92EF92FF920F93C7
:101A60001F93CF93DF9361E081E00E94D07EC0910D
:101A70001F0885E0C82ECC0ED5E0DC1B93E0D92EE4
:101A800014E01C1BBD2CBC1A82E0F82EFC1A81E06D
:101A9000E82EEC1AAC2EA194C1112BC080911E0827
:101AA000882381F080917802882369F181E0909108
:101AB0001E08911180E024E042E156E26A2D0F9465
:101AC000412C21C08091170810921708882351F3E8
:101AD0000E94708680911908882321F3DF91CF91AD
:101AE0001F910F91FF90EF90DF90CF90BF90AF903C
:101AF0000895C130A1F590911E08913059F0809160
:101B00007802811119C0CF5FCC11C6CF86E08093D7
:101B10001808E4CF8091170810921708882379F3EA
:101B2000809137028C2780933702D092780280917F
:101B30001908882321F3D2CF81E0913009F080E0A9
:101B40009091370221E036E2911102C02DEF35E28B
:101B500001E044E056E26E2D0E94662BD4CFC230E5
:101B600009F077C080911E08823079F08091780268
:101B7000882349F281E090911E08923009F080E0BC
:101B800023E04CEA5FE36F2D9ACF80911708109203
:101B90001708882359F38CEA9AE70E94FB81809109
:101BA0001908882319F39ACF80911E08833081F099
:101BB00080917802882309F4A6CF81E090911E08D5
:101BC000933009F080E023E045EA5FE36B2D77CFA7
:101BD0008091170810921708882351F387EA9AE733
:101BE0000E94FB8180911908882311F377CF80919F
:101BF0001E08843081F080917802882309F483CF15
:101C000081E090911E08943009F080E023E04EE9D5
